:020000040000fa
:080000000020040000000000d4
:020000040000fa
:04000800842500004b
:020000040000fa
:04000c008425000047
:020000040000fa
:040010008425000043
:020000040000fa
:04001400842500003f
:020000040000fa
:04001800842500003b
:020000040000fa
:04001c008425000037
:020000040000fa
:040020008425000033
:020000040000fa
:04002400842500002f
:020000040000fa
:04002800842500002b
:020000040000fa
:04002c008425000027
:020000040000fa
:040030008425000023
:020000040000fa
:04003400842500001f
:020000040000fa
:04003800842500001b
:020000040000fa
:04003c008425000017
:020000040000fa
:040040008425000013
:020000040000fa
:04004400842500000f
:020000040000fa
:04004800842500000b
:020000040000fa
:04004c008425000007
:020000040000fa
:040050008425000003
:020000040000fa
:0400540084250000ff
:020000040000fa
:0400580084250000fb
:020000040000fa
:04005c0084250000f7
:020000040000fa
:0400600084250000f3
:020000040000fa
:0400640084250000ef
:020000040000fa
:0400680084250000eb
:020000040000fa
:04006c0084250000e7
:020000040000fa
:0400700084250000e3
:020000040000fa
:0400740084250000df
:020000040000fa
:0400780084250000db
:020000040000fa
:04007c0084250000d7
:020000040000fa
:0400800084250000d3
:020000040000fa
:0400840084250000cf
:020000040000fa
:0400880084250000cb
:020000040000fa
:04008c0084250000c7
:020000040000fa
:0400900084250000c3
:020000040000fa
:0400940084250000bf
:020000040000fa
:0400980084250000bb
:020000040000fa
:04009c0084250000b7
:020000040000fa
:0400a00084250000b3
:020000040000fa
:0400a40084250000af
:020000040000fa
:0400a80084250000ab
:020000040000fa
:0400ac0084250000a7
:020000040000fa
:0400b00084250000a3
:020000040000fa
:0400b400842500009f
:020000040000fa
:0400b800842500009b
:020000040000fa
:0400bc008425000097
:020000040000fa
:0400c0008425000093
:020000040000fa
:0400c400842500008f
:020000040000fa
:0400c800842500008b
:020000040000fa
:0400cc008425000087
:020000040000fa
:0400d0008425000083
:020000040000fa
:0400d400842500007f
:020000040000fa
:0400d800842500007b
:020000040000fa
:0400dc008425000077
:020000040000fa
:0400e0008425000073
:020000040000fa
:0400e400842500006f
:020000040000fa
:0400e800842500006b
:020000040000fa
:0400ec008425000067
:020000040000fa
:0400f0008425000063
:020000040000fa
:0400f400842500005f
:020000040000fa
:0400f800842500005b
:020000040000fa
:0400fc008425000057
:020000040000fa
:040100008425000052
:020000040000fa
:04010400842500004e
:020000040000fa
:04010800842500004a
:020000040000fa
:04010c008425000046
:020000040000fa
:040110008425000042
:020000040000fa
:04011400842500003e
:020000040000fa
:04011800842500003a
:020000040000fa
:04011c008425000036
:020000040000fa
:040120008425000032
:020000040000fa
:04012400842500002e
:020000040000fa
:04012800842500002a
:020000040000fa
:04012c008425000026
:020000040000fa
:040130008425000022
:020000040000fa
:04013400842500001e
:020000040000fa
:04013800842500001a
:020000040000fa
:04013c008425000016
:020000040000fa
:040140008425000012
:020000040000fa
:04014400842500000e
:020000040000fa
:04014800842500000a
:020000040000fa
:04014c008425000006
:020000040000fa
:040150008425000002
:020000040000fa
:0401540084250000fe
:020000040000fa
:0401580084250000fa
:020000040000fa
:04015c0084250000f6
:020000040000fa
:0401600084250000f2
:020000040000fa
:0401640084250000ee
:020000040000fa
:0401680084250000ea
:020000040000fa
:04016c0084250000e6
:020000040000fa
:0401700084250000e2
:020000040000fa
:0401740084250000de
:020000040000fa
:0401780084250000da
:020000040000fa
:04017c0084250000d6
:020000040000fa
:0401800084250000d2
:020000040000fa
:0401840084250000ce
:020000040000fa
:0401880084250000ca
:020000040000fa
:04018c0084250000c6
:020000040000fa
:0401900084250000c2
:020000040000fa
:0401940084250000be
:020000040000fa
:0401980084250000ba
:020000040000fa
:04019c0084250000b6
:020000040000fa
:0401a00084250000b2
:020000040000fa
:0401a40084250000ae
:020000040000fa
:0401a80084250000aa
:020000040000fa
:0401ac0084250000a6
:020000040000fa
:0401b00084250000a2
:020000040000fa
:0401b400842500009e
:020000040000fa
:0401b800842500009a
:020000040000fa
:0401bc008425000096
:020000040000fa
:0401c0008425000092
:020000040000fa
:0401c400842500008e
:020000040000fa
:0401c800842500008a
:020000040000fa
:0401cc008425000086
:020000040000fa
:0401d0008425000082
:020000040000fa
:0401d400842500007e
:020000040000fa
:0401d800842500007a
:020000040000fa
:0401dc008425000076
:020000040000fa
:0401e0008425000072
:020000040000fa
:0401e400842500006e
:020000040000fa
:0401e800842500006a
:020000040000fa
:0401ec008425000066
:020000040000fa
:0401f0008425000062
:020000040000fa
:0401f400842500005e
:020000040000fa
:0401f800842500005a
:020000040000fa
:0401fc008425000056
:020000040000fa
:04300800d8230000c9
:020000040000fa
:04300c00202400007c
:020000040000fa
:04301000f8240000a0
:020000040000fa
:04301400682400002c
:020000040000fa
:04301800b0240000e0
:020000040000fa
:04301c008425000007
:020000040000fa
:043020003e25000049
:020000040000fa
:0430240084250000ff
:020000040000fa
:0430280084250000fb
:020000040000fa
:04302c0084250000f7
:020000040000fa
:0430300084250000f3
:020000040000fa
:043034002c2200004a
:020000040000fa
:0430380084250000eb
:020000040000fa
:04303c0084250000e7
:020000040000fa
:0430400084250000e3
:020000040000fa
:0430440084250000df
:020000040000fa
:0430480084250000db
:020000040000fa
:04304c0084250000d7
:020000040000fa
:0430500084250000d3
:020000040000fa
:0430540088220000ce
:020000040000fa
:04305800b2220000a0
:020000040000fa
:04305c0084250000c7
:020000040000fa
:0430600084250000c3
:020000040000fa
:0430640084250000bf
:020000040000fa
:0430680084250000bb
:020000040000fa
:04306c0084250000b7
:020000040000fa
:0430700084250000b3
:020000040000fa
:0430740084250000af
:020000040000fa
:0430780084250000ab
:020000040000fa
:04307c0084250000a7
:020000040000fa
:0430800084250000a3
:020000040000fa
:04308400842500009f
:020000040000fa
:04308800842500009b
:020000040000fa
:04308c008425000097
:020000040000fa
:043090008425000093
:020000040000fa
:04309400842500008f
:020000040000fa
:04309800842500008b
:020000040000fa
:04309c008425000087
:020000040000fa
:0430a000dc2200002e
:020000040000fa
:0430a40006230000ff
:020000040000fa
:0430a800842500007b
:020000040000fa
:0430ac008425000077
:020000040000fa
:0430b0008425000073
:020000040000fa
:0430b400842500006f
:020000040000fa
:0430b800842500006b
:020000040000fa
:0430bc008425000067
:020000040000fa
:0430c0008425000063
:020000040000fa
:0430c400842500005f
:020000040000fa
:0430c800842500005b
:020000040000fa
:0430cc008425000057
:020000040000fa
:0430d0008425000053
:020000040000fa
:0430d400842500004f
:020000040000fa
:0430d800842500004b
:020000040000fa
:0430dc008425000047
:020000040000fa
:0430e0008425000043
:020000040000fa
:0430e400842500003f
:020000040000fa
:0430e800842500003b
:020000040000fa
:0430ec008425000037
:020000040000fa
:0430f0008425000033
:020000040000fa
:0430f400842500002f
:020000040000fa
:0430f800842500002b
:020000040000fa
:0430fc008425000027
:020000040000fa
:043100008425000022
:020000040000fa
:04310400842500001e
:020000040000fa
:04310800842500001a
:020000040000fa
:04310c008425000016
:020000040000fa
:043110008425000012
:020000040000fa
:04311400842500000e
:020000040000fa
:04311800842500000a
:020000040000fa
:04311c008425000006
:020000040000fa
:043120008425000002
:020000040000fa
:0431240084250000fe
:020000040000fa
:0431280084250000fa
:020000040000fa
:04312c0084250000f6
:020000040000fa
:0431300084250000f2
:020000040000fa
:0431340084250000ee
:020000040000fa
:0431380084250000ea
:020000040000fa
:04313c0084250000e6
:020000040000fa
:0431400084250000e2
:020000040000fa
:0431440084250000de
:020000040000fa
:0431480084250000da
:020000040000fa
:04314c0084250000d6
:020000040000fa
:0431500084250000d2
:020000040000fa
:0431540084250000ce
:020000040000fa
:0431580084250000ca
:020000040000fa
:04315c0084250000c6
:020000040000fa
:0431600084250000c2
:020000040000fa
:0431640084250000be
:020000040000fa
:0431680084250000ba
:020000040000fa
:04316c0084250000b6
:020000040000fa
:043170003023000008
:020000040000fa
:043174005a230000da
:020000040000fa
:0431780084250000aa
:020000040000fa
:04317c0084250000a6
:020000040000fa
:0431800084250000a2
:020000040000fa
:04318400842500009e
:020000040000fa
:04318800842300009c
:020000040000fa
:04318c00ae2300006e
:020000040000fa
:043190008425000092
:020000040000fa
:04319400842500008e
:020000040000fa
:04319800842500008a
:020000040000fa
:04319c008425000086
:020000040000fa
:0431a0008425000082
:020000040000fa
:0431a400842500007e
:020000040000fa
:0431a800842500007a
:020000040000fa
:0431ac008425000076
:020000040000fa
:0431b0008425000072
:020000040000fa
:0431b400842500006e
:020000040000fa
:0431b800842500006a
:020000040000fa
:0431bc008425000066
:020000040000fa
:0431c0008425000062
:020000040000fa
:0431c400842500005e
:020000040000fa
:0431c800842500005a
:020000040000fa
:0431cc008425000056
:020000040000fa
:0431d0008425000052
:020000040000fa
:0431d400842500004e
:020000040000fa
:0431d800842500004a
:020000040000fa
:0431dc008425000046
:020000040000fa
:0431e0008425000042
:020000040000fa
:0431e400842500003e
:020000040000fa
:0431e800842500003a
:020000040000fa
:0431ec008425000036
:020000040000fa
:0431f0008425000032
:020000040000fa
:0431f400842500002e
:020000040000fa
:0431f800842500002a
:020000040000fa
:0431fc008425000026
:020000040000fa
:104000000f4421000eff27000e0188000000000071
:10401000000020000000e00002003200000120004b
:104020002002880014000700b90207000000e00029
:1040300003003a0000232f00010020000200370097
:104040000000200001002000810f700001003200fc
:1040500014000700000020000000e0000200320011
:10406000000002000000000032f902000000000021
:104070000040da000000fe004440a900c0682200b1
:104080000000e000030032000020200090018800c2
:104090004440a800000006008a1f78008b1f7800ab
:1040a00000000600a1028800800478000000eb00f8
:1040b0001f003700e284440054a0b4009905ba0000
:1040c000e284440054a0b4009906ba00e28444009b
:1040d00054a0b4000006eb00476fde00fd07b200fd
:1040e000ae018800636ce10003003a00eaff0700bc
:1040f0000000eb000e003700606ce10008003a00a1
:10410000004deb000a05e800020039003420ec0005
:104110000af0a0008b05e900f9ff3e00040037001b
:104120006168e100010032000086eb000b0007002f
:1041300019c7ba001905ba000e04e00003003a00de
:104140000a00e000dbff3a0000000600fe07b200b4
:10415000ae0288008a047800f5ff37000cd0a30077
:10416000e20f4d001c00390089027800354dba007d
:104170000a05e800020039003420ec000af0a00033
:104180008b05e9000f003200254dba000a05e80052
:10419000020039003420ec000af0a0008b05e90091
:1041a000080032000c00e0000600320015cdba0015
:1041b0000a05e800020039003420ec000af0a000f3
:1041c0008b05e9008984e80054a0b4000b00e000ee
:1041d000e2ff3a00000006009902ba00055d78008f
:1041e0008b05e900f7ff3200c82ade00055d780084
:1041f0008b05e900f3ff32000c00e000f1ff320014
:1042000019ddba00eeff37004cf804000000000092
:10421000b8f3040000000000f27704000000000082
:104220005e78040000000000cc790400000000006b
:10423000d4770400000000008c7904000000000026
:104240003e830400000000008282040000000000a1
:1042500062820400000000001c78040000000000de
:104260000881040000000000f26f0400000000005c
:10427000e07a040000000000d87404000000000090
:10428000fe6f0400000000005a7a040000000000e5
:104290002e79040000000000e87604000000000011
:1042a000347004000000000054bd04000000000051
:1042b0009ad3040000000000d6cb040000000000e8
:1042c000a8cc04000000000054d30400000000004b
:1042d00094cb040000000000d4d2040000000000d1
:1042e00084cb0400000000006cca04000000000041
:1042f000d8da040000000000a4da04000000000086
:10430000dadb04000000000008dc0400000000000c
:104310009ed704000000000022d704000000000027
:10432000c2d5040000000000bcd40400000000005e
:10433000c6b40400000000005aae040000000000f3
:104340007ebc040000000000d6b4040000000000a1
:1043500038b8040000000000fcae040000000000bb
:1043600008b8040000000000eab7040000000000e4
:104370003eae0400000000006ab604000000000029
:1043800042b6040000000000fcb50400000000007c
:104390001cad040000000000eab5040000000000ad
:1043a0005cb50400000000003ebb040000000000fb
:1043b0008ab404000000000020b4040000000000e3
:1043c0003ab304000000000080ac040000000000cc
:1043d00018b30400000000005cb2040000000000fc
:1043e0000eb4040000000000aab1040000000000a8
:1043f000c2ae040000000000d2af040000000000c4
:10440000f0b004000000000024b10400000000002f
:104410008cae040000000000acba040000000000f4
:10442000e0ad040000000000a8ad040000000000a2
:1044300066ad040000000000d2ac040000000000e3
:104440009aac0400000000006e2c04000000000084
:104450002e310400000000003600f800809fbe00ee
:10446000829fbe00849fbe00869fbe003200f8007f
:104470003400f80010002000a00188000020200077
:104480009001880040408000514080006100400061
:10449000e08048004040880051408800c4802000ef
:1044a000144278000404e0000f0032000000eb002a
:1044b000e11c21004301dd00610179000200e00000
:1044c000060032004301dd00e6014100e181790090
:1044d00002814000660141000309e8000000e80095
:1044e000804f5200f3ff3e006000b8000c660700ea
:1044f0003400f9003200f9004f03be004f02be0045
:104500004f01be004f00be003600f900004006001b
:104510003600f800809fbe00829fbe00849fbe00d0
:10452000869fbe003200f8003400f8001000200022
:10453000a001880000202000900188000040eb00ce
:10454000b86007003400f9003200f9004f03be00e4
:104550004f02be004f01be004f00be003600f90002
:10456000004006003600f800809fbe00829fbe001b
:10457000849fbe00869fbe003200f8003400f80021
:1045800010002000a0018800002020009001880079
:104590000040eb007c6007003400f9003200f900b5
:1045a0004f03be004f02be004f01be004f00be00d1
:1045b0003600f900004006003600f800809fbe007b
:1045c000829fbe00849fbe00869fbe003200f8001e
:1045d0003400f80010002000a00188000020200016
:1045e0009001880010c0b3008e6007003400f9000d
:1045f0003200f9004f03be004f02be004f01be0063
:104600004f00be003600f900004006003600f800fa
:10461000809fbe00829fbe00849fbe00869fbe001a
:104620003200f8003400f80010002000a0018800db
:10463000002020009001880010c0b30052600700e5
:104640003400f9003200f9004f03be004f02be00f3
:104650004f01be004f00be003600f90000400600ca
:104660003600f800809fbe00829fbe00849fbe007f
:10467000869fbe003200f8003400f80010002000d1
:10468000a0018800002020009001880020c0b30015
:10469000646007003400f9003200f9004f03be00e7
:1046a0004f02be004f01be004f00be003600f900b1
:1046b000004006003600f800809fbe00829fbe00ca
:1046c000849fbe00869fbe003200f8003400f800d0
:1046d00010002000a0018800002020009001880028
:1046e00020c0b300286007003400f9003200f90050
:1046f0004f03be004f02be004f01be004f00be0080
:104700003600f900004006003600f800809fbe0029
:10471000829fbe00849fbe00869fbe003200f800cc
:104720003400f80010002000a001880000202000c4
:104730009001880030c0b3003a6007003400f900ef
:104740003200f9004f03be004f02be004f01be0011
:104750004f00be003600f900004006003600f800a9
:10476000809fbe00829fbe00849fbe00869fbe00c9
:104770003200f8003400f80010002000a00188008a
:10478000002020009001880030c0b300fe5f0700c9
:104790003400f9003200f9004f03be004f02be00a2
:1047a0004f01be004f00be003600f9000040060079
:1047b0003600f800809fbe00829fbe00849fbe002e
:1047c000869fbe00889fbe008a1f78003200f800d6
:1047d0003400f80010002000a00188000020200014
:1047e000900188008020a90080c0b3004d630700bd
:1047f000b606a9000005eb00883e200009352c0014
:1048000008007800196907000a05e800890f5500bb
:10481000fbff3a007b5d07003400f9003200f9002d
:104820004f0578004f04be004f03be004f02be008c
:104830004f01be004f00be003600f90000400600e8
:104840003600f800809fbe00829fbe00849fbe009d
:10485000869fbe00889fbe008a1f78003200f80045
:104860003400f80010002000a00188000020200083
:10487000900188008060a90090c0b3002963070000
:10488000b606a9000005eb00883e200009352c0083
:1048900008007800f56807000a05e800890f550050
:1048a000fbff3a00575d07003400f9003200f900c1
:1048b0004f0578004f04be004f03be004f02be00fc
:1048c0004f01be004f00be003600f9000040060058
:1048d0003600f800809fbe00829fbe00849fbe000d
:1048e000869fbe00889fbe008a1f78003200f800b5
:1048f0003400f80010002000a001880000202000f3
:10490000900188008040a900a0c0b30005630700a3
:10491000b606a9000005eb00883e200009352c00f2
:1049200008007800d16807000a05e800890f5500e3
:10493000fbff3a00335d07003400f9003200f90054
:104940004f0578004f04be004f03be004f02be006b
:104950004f01be004f00be003600f90000400600c7
:104960003600f800809fbe00829fbe00849fbe007c
:10497000869fbe00889fbe008a1f78003200f80024
:104980003400f80010002000a00188000020200062
:10499000900188008080a900b0c0b300e1620700e8
:1049a000b606a9000005eb00883e200009352c0062
:1049b00008007800ad6807000a05e800890f550077
:1049c000fbff3a000f5d07003400f9003200f900e8
:1049d0004f0578004f04be004f03be004f02be00db
:1049e0004f01be004f00be003600f9000040060037
:1049f0003600f800809fbe00829fbe00849fbe00ec
:104a0000869fbe00889fbe008a1f78003200f80093
:104a10003400f80010002000a001880000202000d1
:104a200090018800c0c0b300be620700b606a900ae
:104a30000005eb00883e200009352c0008007800b6
:104a40008a6807000a05e800890f5500fbff3a0055
:104a5000ec5c07003400f9003200f9004f057800e3
:104a60004f04be004f03be004f02be004f01be0008
:104a70004f00be003600f900004006003600f80086
:104a8000809fbe00829fbe00849fbe00869fbe00a6
:104a9000889fbe008a1f78003200f8003400f800ba
:104aa00010002000a0018800002020009001880054
:104ab000d0c0b3009b620700b606a9000005eb005a
:104ac000883e200009352c00080078006768070040
:104ad0000a05e800890f5500fbff3a00c95c070092
:104ae0003400f9003200f9004f0578004f04be0091
:104af0004f03be004f02be004f01be004f00be007c
:104b00003600f900004006000040da000000fe0018
:104b10000000050003f0a200889fbe008a9fbe002f
:104b20008c1f7800b2000700b90033006450e10028
:104b30004f0032006420e1005200320003826c001a
:104b400007003b000905d0000306d000820f540087
:104b50000c065d0002003900020032008901780075
:104b6000030678008582550004003d000003fd0027
:104b70008103fd008502ea008b854200840f7200ec
:104b800002003b0060001000e08018006011b800d7
:104b90000005eb007a28e1000a00390006007800e1
:104ba000c75ddd00f707b200878075002d00370074
:104bb000828171000a017800610560008180d10066
:104bc0000080d3008502e900f9ff3b0006044000a5
:104bd0008784480002003b0060041400e0841c004d
:104be0000988a300070032008a8171008281710068
:104bf000610164008904d1000884d3008b05e800ba
:104c0000170037000978a30013003a000b00e000fa
:104c1000130034008b05e9000804440089844c002b
:104c20000a4474000978a3000d003a000b00e0006c
:104c3000070034008b05e9000804440089844c0017
:104c400001003a000b0020000978a300f7ff3200b2
:104c50000001eb0002003700828171000a01780038
:104c6000280007000cf0a70001f0a0007100370039
:104c70006420e10002003a00838f6c007100330071
:104c80000801be000200be006a0037000001be003d
:104c9000420007000470a70003f0a10003f8a3007e
:104ca00013003a006509b100100032000900350018
:104cb0006928e1000200350001002800000005001d
:104cc00000004000818048008502e900fcff3a00b6
:104cd00000000600f88f4200050035008100d10079
:104ce0000080d3008502e800fcff3a0000000600c7
:104cf0008000eb00000005004f89de008201780093
:104d00002f01370081002000618055000b003d001d
:104d10000b00200061fe2f000100e1001d003400a7
:104d200082817100610164008904d1000884d3008c
:104d30000000e800faff3a00710020006100640002
:104d400003007000020060000900320061044400aa
:104d5000e0844c000988a500050032008b05e800be
:104d60006808e10002003a008904d1000884d300f9
:104d7000f20f20000258e10005003d00c75ddd0094
:104d8000f907b2008980750008007800000006006d
:104d90000bf827008b00780000000500c70ade0032
:104da000f107b200f50fb20008003200e1cf420077
:104db000020032000170a00024000500810f700085
:104dc000010032000408050044000500810f700056
:104dd00002003a00140005008502e90000004000ce
:104de00081c04800fcff3b000170a00024000500ca
:104df0000004be00e9ff07000003be000405be007a
:104e00000200be00e5ff0700844f750000000600a9
:104e10000200be006450e100050036006420e1009d
:104e2000020036000968a30001003a000800be0035
:104e30000160a0004f0678004f05be004f04be0081
:104e400000000600f0ff2f00f1ff2700f9ff3700f8
:104e5000889fbe008a9fbe008c9fbe00870007000f
:104e6000850478000005be006420e10049003e0092
:104e70006220e10003003200090035000bf8a300b6
:104e8000440032000bf8a30008003200100220009a
:104e900090408800f0ff2f00f1ff27003d00370011
:104ea00001f82f00000020003a0037003d00070005
:104eb00018ff07000006be000a00be00324f2000a7
:104ec00053f32300bc000700060034000c00be00b2
:104ed000340007000fff07000006be000a00be00f6
:104ee000020037008904e9000c00be002d00070015
:104ef0002e0007002b00070007ff07000001be007f
:104f00000c00be006a0007000005be000001be00e4
:104f1000260007000006be00a2f32300430d2c006c
:104f2000fdfe0700809fbe000c00be00d2e32700fc
:104f3000d3f02b001d0007004f01be005c000700ee
:104f40000006be000a01be00180007000a01be00ec
:104f5000f1fe07000006be006148b90066ff0700c9
:104f60000005be0032082800e3952b000f00070063
:104f70000c01be00e8fe07000006be000a00be00ed
:104f80000200280013f32300080007000c01be00f4
:104f9000e1fe07004f06be004f05be004f04be00f5
:104fa0000000060003f0230002000500889fbe00f9
:104fb0008a9fbe008c1f78008dff070094ff33008e
:104fc00003866c006450e100240032006420e1009c
:104fd000270032006150e100220032006120e10030
:104fe000210032008b854200eb07b1000134b8008c
:104ff000003ab8000804420089844a00013ab80027
:105000000030b8008880400009014a0004003300e5
:105010000000400081804800020149008b05e90042
:10502000c909dd0083017000010032001300200077
:10503000c814de004814dd004709de001200b2008b
:10504000c808de00088470002eff070001f0a100f0
:105050000cf0a70001f0a00076ff37006120e1000e
:1050600078ff32000801be000200be00f7ff3700e3
:105070006150e100fcff3a0072ff37000003be0000
:1050800046ff07006220e100020032000600be0079
:1050900005000500e507b100f107b20004f02300a8
:1050a0008480700007f0a70001f0a0002400050034
:1050b000889fbe008a9fbe008c1f78004cff0700af
:1050c00053ff330003866c006450e1002e00320071
:1050d0006420e100330032006150e1002f00320013
:1050e0006120e1003100320085855500eb07b000fa
:1050f00009002000080420000500370008044400cf
:1051000089844c000a0031000603430087834b006a
:105110000001530081815b00f8ff33000203be00f1
:105120000800a0000804440089844c00f6ff390000
:10513000c639dd0083017300010032001300200036
:105140008904d1000884d3000998a3000500320027
:105150000800a7000300a0008904d1000884d30040
:105160008b05e8008904d1000884d3000001eb001e
:105170000281d200e3fe070001f0a1000cf0a700bd
:1051800001f0a0002bff37006420e1002dff32006a
:105190000801be000200be00f7ff37006120e100f9
:1051a00028ff32006000b800f3ff37000000200045
:1051b00001f82700f0ff3700f4ff2f003f00370011
:1051c000881f7800030478000300e00007003d001a
:1051d00060001000e080180060011900e0811900f3
:1051e00002003b0001f02d0003003700040007001f
:1051f00008f0a70001f0a0004f04780000000600ae
:10520000889fbe008a9fbe00008270000402710069
:1052100004827100260032000004be000200be00bd
:105220006011b8006b092000950220000182cf00b8
:105230000a0039000541b1000082cf0007003900a3
:105240000541b1000982cf00040039000541b100d9
:105250000882cf00010039000541b100054252002b
:10526000120032000a003b0082817100610164007b
:105270008100d1000080d3008984d3000884d3004a
:105280008b05e8000442e800f7ff3a00070037000a
:105290000804440089844c000000480081804800d4
:1052a0008b05e9000442e900f9ff3a0095fe07008a
:1052b0004f05be004f04be0000000600889fbe00e0
:1052c0008a9fbe00841f7800c9fe07004f00780047
:1052d00011003300f0ff2f00838f6c0006003b00ad
:1052e000040565000a00a7000800370009f0a600c1
:1052f0001000200008003700820f5400838f5c00ec
:10530000030039001000200001003e0000002000d2
:1053100009f0a7000000ea004f05be004f04be00e0
:105320000000e00000000600800078001106b100d7
:10533000030035009101b10001003c000050a100c4
:10534000000006000900370030427800b1417800c3
:10535000834f52000400320010002000060031008c
:105360000080eb00000006000201e9000200e000fe
:10537000f5ff3a000000eb00000006000002780094
:10538000808f50000c00310082814000830f50005c
:10539000090031008200400002003700c36078003d
:1053a0000201e9000200e000fcff3a0000000600f4
:1053b000315a78000201e9000200e000fcff3a00e7
:1053c0000000060080017800020037008159780053
:1053d0000201e9000200e000fcff3a0000000600c4
:1053e000020037000204e0000b0032008101780067
:1053f0000002780030417800b14f5100f9ff3200cf
:105400001000200014427800934f52000300310036
:105410000080eb00000006000000eb00000006002a
:1054200000017800b1417800035978000304e000de
:10543000fcff3a00000006008000780001017800bf
:105440003104e000fdff3a000000510000000600ba
:105450008001780002003700845978000201e900d9
:105460000200e00006003200314278000404e0004f
:10547000f9ff3a00020037008059eb000201e90011
:105480000200e000fcff3a0000000600889fbe001a
:1054900081047800194478000804e0000e0032000e
:1054a00006003700d24178000304e0000a00320011
:1054b000d1cf1100fbff32000000e8008800fb00a4
:1054c000550307000000e0000300320009017800e6
:1054d00080007800f3ff37004f04be000000060094
:1054e000889fbe00810478000000e00002003a00be
:1054f000e8a1800001003700000478000800be0029
:1055000078050700000444001804e00004003a0095
:10551000a0432100e0a188000004eb000700370051
:105520000800be005e050700000044001004e00013
:10553000010032000058eb00e0a18800080078006c
:105540004f04be0000000600e4874700889fbe00ad
:105550008a9fbe008c1f78008e1f7800000578009f
:1055600001077800020678000e00e00001003a0012
:105570006e8757008a0578008b04780089057800cb
:105580003b4478000800fb00140307000000e00023
:10559000f9ff3a00d0c2b300804f5400030032003c
:1055a00000c0e900804f540002003a008904e8007e
:1055b00001003700004478000c0178008e0078006c
:1055c00009007800290007009e8f540001003a006e
:1055d0000a0f78009e0f550003003a00e00f5000bc
:1055e000e08f58000f003a00b2c2b300824f54005f
:1055f00004003a00e00f5000e08f580015003d0015
:1056000008003700d2c2b300824f540011003a00a4
:105610000200200003002800820f5000838f5800f2
:105620000a0036002002200090408800f0ff2f0082
:10563000f1ff2700d2c2b300824f540005003a00a8
:105640000000200001002800020037006000100068
:10565000e08018004f0778004f0678004f05be0025
:105660004f04be004f00b10000000600ee87470067
:10567000889fbe008a9fbe008c9fbe008e1f780050
:10568000f0b79f00010678008205780000047800da
:10569000080578000a047800b84678000d00fb0081
:1056a000ce0207000000e000f9ff3a00d0c2b300cc
:1056b00080cf56000300320000c0e90080cf5600c2
:1056c00002003a000a05e800010037008046780031
:1056d0000b00e00005003500e18f550003003200ab
:1056e00040022000808f5500060034006044b8005e
:1056f0000c00e000720032007fb09700000e7800ce
:10570000480037000b00e0000e003200f08f55001b
:105710001a003a0000c3b3009a4f100017003a0075
:105720001a40900081c7b300814f5000030032003f
:1057300081c5b300814f500010003a000a85e8008f
:105740000e003700ab00200000c3b3009a4f1000da
:105750000a003a001a40900081c7b300814f500000
:10576000040032008b00200081c5b300814f50003f
:1057700002003a000a85e8000b0120000a007800c8
:10578000000278000400780001c3b300b0cf10001d
:10579000fbff3200040778006044b800b4b79f00f4
:1057a0000d0037008132210081405000c1ef9f0081
:1057b0006159b9000800be00920c07004fea97003b
:1057c0000401fb00cf91de00c8b79f00d9b79f004e
:1057d00002044000838448008e0278003e00fb00f3
:1057e00085bf9f00850207000b01780080007800cc
:1057f00080322100990407008fba97000000e00072
:10580000e8ff3a003fb29700850f550007003a00c5
:105810006044b8000c00e00029003200ffb297009d
:10582000050e78006044b80025003700048252005d
:10583000d034210060c07d000000fb000002520057
:105840001700330011003a004fe997000200fb00f7
:10585000cf80de000000540081805c00800f540087
:10586000818f5c00090039006159b90085bf9f0034
:10587000510c07008fba97004fb19700dfb1970026
:10588000820f5000838f5800050032002002200054
:10589000904088000084eb008084eb000500370016
:1058a000d0c2b30080cf560002003a00600414005a
:1058b000e0841c000c00e00001003200050e7800be
:1058c0000800be004f0778004f06be004f05be001f
:1058d0004f04be00ef00b10000000600889fbe002c
:1058e000000478001800900082047800808f540033
:1058f0000100360080047800180078000901780063
:1059000060040700188c44001800900089045000bf
:1059100019049800080078004f04be00000006003b
:105920000400fa000100e00003003a000f80e900e3
:10593000e0bf9f0002003700e0bf9f008100e90048
:10594000f1bf9f00e4805700e0c62200040007007a
:10595000efb897008048eb000080fa0000000600d6
:105960006200fa00889fbe008a1f78000005780058
:1059700081047800020478008300780080f92f0009
:105980000f004000330207009a979f00a9979f00dd
:105990000000eb00b09f9f001885fb008a04fb000d
:1059a0000a05ea004f55de0050022000808f5400a7
:1059b0000d003200e10f55000b003a000a0178009b
:1059c000880078002f9097009f91970003000100b6
:1059d000a0979f000000e0008e0032003f989700e3
:1059e0000000e800b09f9f000a044400500220001d
:1059f000808f5400040032000900e000e6ff3a0006
:105a00003f989700840037000000eb00909f9f00b4
:105a1000809f9f00f0979f00e0979f00d0979f0086
:105a2000c0979f0007003700613c21000100500033
:105a300000004000a13b210061007800df98970042
:105a400001007000d09f9f0088047800090478004e
:105a5000384578008a00fb00603c2100ee01070019
:105a60000000e000f0ff3a00a1c2b300814f5500f2
:105a70000e003a00cf8897000180e900c08f9f0098
:105a800010007800c09f9f000000e00005003d006e
:105a90000000ea00c09f9f005f9897000020a000d0
:105aa000d09f9f000904e8000f003700c09f9f00af
:105ab0000000eb0005003700f2ff2700820f5000c6
:105ac000020032006a01b900028040000904780037
:105ad00088047800b900fb000103b100e98f500091
:105ae000f5ff3600c09f9f00e0c2b300984f100042
:105af000020032000080eb0019003700a0c2b300a2
:105b0000d84f100007003a00cf8897000180e900c5
:105b1000c08f9f0010007800a09f9f000804e8003d
:105b2000100037000000eb00a09f9f008800780065
:105b300005003700f3ff2700830f500002003200fa
:105b40006a02b9000400410001047800880078006e
:105b50003101fb000203b100e90f5100f5ff3600ef
:105b6000a09f9f00984478008900fb00203b210003
:105b7000a90107000000e000020032000804e8006c
:105b8000010037008044eb00c97f9f0080c6b3004e
:105b900080cf540004003a0098cf14000a003a0065
:105ba0006640500006003700c0c6b30080cf5400e6
:105bb00005003a0098cf140003003a006540400009
:105bc000c07f9f000804e800e3fb2f008f814100a5
:105bd0001841780081f92f008f804000a0f92f0034
:105be0000f004000100007000000e00009003a002c
:105bf000e1fb2f008f804000a0f92f000f00400034
:105c00001a0707000000e000020035000804e80061
:105c100061ff37000080eb004f0578004f04be00a5
:105c20000080fa0000000600889fbe008a1f7800ee
:105c300000047800824478000305780070c6b30041
:105c400080cf540021003c0000c0e90080cf540008
:105c5000d5003d007240500080cf54003c0132001e
:105c60000d003c006c40500080cf54004f013c00c0
:105c700000c0e90080cf5400cb003d0050c2b3000b
:105c800080cf5400460132007c40400080cf540059
:105c900046013a00c400370010c6b30080cf54005c
:105ca000c100320004003c006940500080cf540025
:105cb0003e013a006900370030c6b30080cf54007f
:105cc000180032000040e8000900370000c7b300a8
:105cd00080cf54001001320008003c0000c0e900f1
:105ce00080cf5400d90032005c003c006540500079
:105cf00080cf54002d013a000f00370050c7b30089
:105d000080cf5400550032006340400080cf5400e3
:105d1000520032006540500080cf540023013a0009
:105d20000b0137001181e9008208780078009000ab
:105d3000127578002301370028609000c2c6b300b6
:105d4000824f500007003a001101780064005100b2
:105d5000800878001000be004f89de0082017800c4
:105d60001400370012c7b300824f500003003a00fe
:105d7000110278006800520005003700a2c6b30087
:105d8000824f500006003a0091027800688052006d
:105d9000800878005001be004000be0005003700ba
:105da0001180e9008008780010007800cf80de00c4
:105db0006109b900009cbe000294be0028629000f8
:105dc00085c6b300854f52000d00320025c6b300d2
:105dd000854f520004003a000000fb00cf80de0037
:105de0006109b9000800370045c7b300854f52006c
:105df00003003200e6c24200854f520004003a0020
:105e0000cf80de006109b900009cbe000294be0094
:105e10003802be002803be0078009000d1c2b30053
:105e2000e00f5200e08f5a00e00f5b00e08f5b0054
:105e300008003500881090000118a300020032000d
:105e4000b1c2b300030037000108a30051003200c3
:105e500001c2b300017578004c0037002860900043
:105e6000c2c6b300824f500008003a001103780008
:105e700064005300800878001002be006033b80050
:105e80000400be000601be001400370012c7b300b4
:105e9000824f500003003a0091027800688052005f
:105ea00005003700a2c6b300824f500006003a003a
:105eb0001103780068005300800878005001be008c
:105ec0004000be00050037001180e900800878001e
:105ed000100078008000eb006011b800009cbe004c
:105ee0000294be002862900085c6b300854f520020
:105ef0000d00320025c6b300854f520004003a0061
:105f00000080fb008000eb006011b8000800370043
:105f100045c7b300854f520003003200e6c242007d
:105f2000854f520004003a008000eb006011b80079
:105f3000009cbe000294be00081090000038a30030
:105f4000140032003800be002801be00e00f5000ef
:105f5000e08f5800e00f5900e08f59000d0032002b
:105f600080c7b30080cf54000300320080c5b30067
:105f700080cf540007003a007800900001c3b300be
:105f8000017578000000e800097578000000e8005d
:105f90007004980078009000000545006a0498009d
:105fa000894078006700370028619000c0c4b300c2
:105fb000804f510006003a0091037800688053003a
:105fc000800878005001be004000be000500370088
:105fd0001101780064005100800878001000be00b4
:105fe000af090700009cbe000294be00b8009000fc
:105ff000780090000100e00002003d00d1c2b30033
:1060000008003700881090000118a3000200320039
:10601000b1c2b300030037000108a300040032003e
:1060200001c2b300017578000000e8007004980018
:1060300078009000000545006a04980089407800c7
:1060400008007800b7020700600037002861900060
:10605000c3c6b3001180e900834f51002200320013
:106060000a003c00e4c15100834f5100250032007a
:1060700083c1e800834f510013003200e8c1510092
:10608000834f51001e003a000a00370043c7b30097
:10609000834f51001b003200e6c14100834f510085
:1060a00018003200e9c15100834f510014003a003a
:1060b000050037008008780010007800485c9000e8
:1060c0000848780041003700800878001000780008
:1060d000680a9000cfa2de00612bb9000498be00d0
:1060e0000690be0039003700800878001000780064
:1060f00068099000cf91de000288be0033003700af
:106100001180e9008008780010007800680c900089
:10611000080878002d0037001180e9008008780019
:1061200010007800cf80de006109b900009cbe003d
:106130000294be0078009000000545006a049800b3
:1061400081c7b30008007800990407001f003700da
:106150001180e90080087800100578006a04980032
:10616000d80c90000900e00004003d000a0078000f
:10617000b1fc0700800478000700370009017800af
:106180008000eb000a007800340207000000e00005
:10619000010032008a045000190c98000b003700ef
:1061a00078009000097578000600370078009000ac
:1061b000000545000904e00001003a0059c2b3009f
:1061c000094d78000000e800700498000000eb0022
:1061d0004f0578004f04be00000006006900e10092
:1061e000040035006d00e100030034000002b1003e
:1061f000010032000000050010000500800078005a
:106200001104b100030035009101b10001003c0010
:106210000050a000000006000001eb000300370062
:106220000201e8000404e000070032006103b80046
:106230006112b8008601420066427a00814f520026
:10624000f7ff3a00010037008001eb0003007800ff
:10625000000006000108780000000600889fbe00cc
:10626000000478001800900082047800808f5400a9
:1062700001003600800478001800780009017800d9
:1062800000020700188c4400180090008904500098
:1062900019049800080078004f04be0000000600b2
:1062a0000400fa000100e00003003a000f80e9005a
:1062b000e0bf9f0002003700e0bf9f008100e900bf
:1062c000f1bf9f00ec8157002fb99700e480570081
:1062d000e012230004000700efb897008048eb00ad
:1062e0000080fa00000006006200fa00889fbe00ed
:1062f0008a1f780000057800810478000204780085
:106300008300780080f92f000f004000d1ff0700c4
:106310009a979f00a9979f000000eb00b09f9f00f5
:106320001885fb008a04fb000a05ea004f55de00d1
:1063300050022000808f54000d003200e10f550004
:106340000b003a000a017800880078002f9097002f
:106350009f91970003000100a0979f000000e000bc
:106360008e0032003f9897000000e800b09f9f0029
:106370000a04440050022000808f540004003200c0
:106380000900e000e6ff3a003f98970084003700dc
:106390000000eb00909f9f00809f9f00f0979f0060
:1063a000e0979f00d0979f00c0979f00070037009d
:1063b000013e21000100500000004000413d21004d
:1063c00061007800df98970001007000d09f9f0067
:1063d0008804780009047800384578008a00fb00ba
:1063e000003e21008cff07000000e000f0ff3a00b3
:1063f000a1c2b300814f55000e003a00cf8897002c
:106400000180e900c08f9f0010007800c09f9f00ae
:106410000000e00005003d000000ea00c09f9f0072
:106420005f9897000020a000d09f9f000904e8001b
:106430000f003700c09f9f000000eb0005003700f1
:10644000f2ff2700820f5000020032006a01b900fb
:10645000028040000904780088047800b900fb003d
:106460000103b100e98f5000f5ff3600c09f9f0087
:10647000e0c2b300984f1000020032000080eb0031
:1064800019003700a0c2b300d84f100007003a002f
:10649000cf8897000180e900c08f9f00100078002e
:1064a000a09f9f000804e800100037000000eb00e8
:1064b000a09f9f008800780005003700f3ff2700a9
:1064c000830f5000020032006a02b900040041004c
:1064d00001047800880078003101fb000203b1005c
:1064e000e90f5100f5ff3600a09f9f009844780007
:1064f0008900fb00c03c210047ff07000000e000ce
:10650000020032000804e800010037008044eb007c
:10651000c97f9f0080c6b30080cf540004003a00ba
:1065200098cf14000a003a00664050000600370079
:10653000c0c6b30080cf540005003a0098cf1400c5
:1065400003003a0065404000c07f9f000804e80057
:106550001801fb00e3fb2f008f81410081f92f0020
:106560008f804000a0f92f000f00400010000700ae
:106570000000e00009003a00e1fb2f008f8040009e
:10658000a0f92f000f004000b80407000000e00051
:10659000020035000804e80061ff37000080eb00ce
:1065a0004f0578004f04be000080fa00000006008e
:1065b000889fbe008a1f780000047800e0c6b30000
:1065c000804f5100c100320015003c006b4050006c
:1065d000804f5100240032000a003c0070405000ff
:1065e000804f5100fa00320065404000804f51005a
:1065f0006800320050c2b300804f51000b013a00d6
:106600000701370040c6b300804f51001b00320025
:1066100065404000804f510004013a0017003700e8
:1066200030c7b300804f5100e900320007003c0042
:1066300064405000804f5100560032000040e80096
:10664000804f5100f9003a00d300370050c7b30023
:10665000804f51004f00320063404000804f510096
:10666000f2003a004b0037001181e90082087800ff
:106670007800900012417800ea003700286090000e
:10668000c4c6b300844f500007003a0011027800de
:1066900064005200800878001002be004fabde009c
:1066a000860378001100370014c7b300844f5000f0
:1066b00003003200a4c6b300844f500006003a0025
:1066c0001102780068005200800878003002be0095
:1066d0002003be00050037001180e9008008780023
:1066e00010027800cfa2de00612bb900049cbe002e
:1066f0000694be002860900081c6b300814f500010
:106700000d00320021c6b300814f500004003a0052
:106710000402fb00cfa2de00612bb90008003700a5
:1067200041c7b300814f500003003200e6c0400073
:10673000814f500004003a00cfa2de00612bb90067
:10674000049cbe000694be003802be002803be00b2
:1067500078009000d1c2b300e00f5200e08f5a00e1
:10676000e00f5b00e08f5b000800350088109000b0
:106770000118a30002003200b1c2b30003003700c9
:106780000108a3004c00320001c2b30081717800ff
:106790004700370028609000c4c6b300844f500003
:1067a00006003a0011027800640052008008780068
:1067b0001002be006033b8001100370014c7b300e8
:1067c000844f500003003200a4c6b300844f500031
:1067d00006003a0011027800680052008008780034
:1067e0003002be002003be00050037001180e90022
:1067f00080087800100278008002eb006033b80057
:10680000049cbe000694be002860900081c6b300c0
:10681000814f50000d00320021c6b300814f50005f
:1068200004003a000482fb008002eb006033b800f1
:106830000800370041c7b300814f50000300320009
:10684000e6c04000814f500004003a008002eb0097
:106850006033b800049cbe000694be00081090008f
:106860000038a300140032003802be002803be0026
:10687000e00f5200e08f5a00e00f5b00e08f5b00fa
:106880000d00320080c7b300804f5100030032007a
:1068900080c5b300804f510007003a007800900097
:1068a00001c3b300817178000000e80082717800b4
:1068b0000000e8007004980078009000808141009a
:1068c00063049800824078003e0037002861900001
:1068d000c3c6b3001180e900834f5100220032008b
:1068e0000a003c00e4c15100834f510025003200f2
:1068f00083c1e800834f510013003200e8c151000a
:10690000834f51001e003a000a00370043c7b3000e
:10691000834f51001b003200e6c14100834f5100fc
:1069200018003200e9c15100834f510014003a00b1
:10693000050037008008780010007800485c90005f
:10694000084878004100370080087800100078007f
:10695000680a9000cfa2de00612bb9000498be0047
:106960000690be00390037008008780010007800db
:1069700068099000cf91de000288be003300370026
:106980001180e9008008780010007800680c900001
:10699000080878002d0037001180e9008008780091
:1069a00010027800cfa2de00612bb900049cbe006b
:1069b0000694be0078009000808141006304980036
:1069c00081c7b30008007800790207001f00370074
:1069d0001180e90080087800100578006a049800aa
:1069e000d80c90000900e00004003d000a00780087
:1069f00091fa070080047800070037000901780049
:106a00008000eb000a007800140007000000e0009e
:106a1000010032008a045000190c98000b00370066
:106a200078009000827178000600370078009000ae
:106a3000808141000204e00001003a0052c2b3002c
:106a4000824978000000e800700498000000eb0024
:106a50004f0578004f04be00000006000300370019
:106a6000b0cf1000050032000201e900800178007b
:106a70000200e000faff3a00000005000300780081
:106a8000000006008001780002003700b15978004c
:106a90000201e9000200e000fcff3a0000000600ed
:106aa000000178000700370086cf520002003a004c
:106ab0000080510000000600344378000604e00026
:106ac000f9ff3a0082017800b24278000504e00044
:106ad0000200320001027800f7ff37000080510009
:106ae00000000600000178000800370081027800ed
:106af000354378000604e00002003a0000805100af
:106b000000000600864f5200f9ff3a00820178002b
:106b1000324278000404e000f4ff3a0000805100a3
:106b200000000600cf04b000889fbe008a9fbe0010
:106b30008c9fbe008e1f780000067800814678008a
:106b40003c00be002c01be00d0979f00e1979f0043
:106b5000f2979f00839f9f0010c6b30080cf56001e
:106b60001200320010c4b30080cf56000f00320074
:106b70005c0890000000e00002003d006000200082
:106b8000090037000000e00008003a0070c6b300ba
:106b900080cf56000300320070c4b30080cf56008f
:106ba00002003a0010002000500e98008c0078007f
:106bb00080fa2f000f004000d3010700e20f5000c1
:106bc0000f003a0030002000100e9800e024210051
:106bd00011c6b30081cf560019003200e4c0400056
:106be00081cf560016003200202521008140e800a8
:106bf00081cf560012003a00e02421001000370037
:106c00000000e0001400340030002000100e980056
:106c10006025210011c6b30081cf56000800320064
:106c2000e4c0400081cf560005003200a0252100bd
:106c30008140e80081cf560001003a006025210024
:106c4000ec009000b0487800b06878001040780000
:106c500090409800a601370011c6b30081cf5600be
:106c60000300320011c4b30081cf56000e003a0079
:106c7000ec00900002c3b3008258780061069800cf
:106c800082c5b30013c6b30083cf560001003a009b
:106c900082c7b3008258780061069800fc0090001b
:106ca0008180e800710698000000e00005003a00cd
:106cb000c0979f008001eb0022fb2f000f014100d5
:106cc0008701370010c6b30080cf5600060032009f
:106cd00010c4b30080cf56009a003a00f12621007c
:106ce000d1b79f0002003700e2252100d2b79f00f4
:106cf0005c0890001b0220000000e000010035004d
:106d00008005e8000b05e8006022b8006033b80099
:106d10005f909700ef9097007f9197008f99970071
:106d2000a7050700000278003c00be002c01be0051
:106d30000400e00001003d0003f0a200d0979f0096
:106d4000e1979f00f2979f00839f9f00cf9197004c
:106d5000e4815100c3979f000040eb00a0779f00a3
:106d60003efb2f000f07470031003700c201200013
:106d700003002000a0fa2f000f004000d8030700f6
:106d80005f909700ef9097007f9197008f99970001
:106d900090b79f00a1b79f00b2b79f00c3b79f00f5
:106da0005e0607000004be00670555004240a900ca
:106db0000c003400850607000002be000203be007e
:106dc0001fb09700afb097003fb19700cfb19700c9
:106dd000f7060700d0979f00e1979f00f2979f006a
:106de000839f9f0067074700700020000500370061
:106df0006f676400cc48dd004444de000884700006
:106e0000c4ccde00e00f5400e08f5c0005003400cd
:106e10000000e900e10f4000f5ff3a0001003700f3
:106e20000067eb000000e900fdff3b00670747003b
:106e30000a00e000090034006022b8006033b800a6
:106e40005f909700ef9097007f9197008f99970040
:106e5000600507000000e000c4ff3c0032fb2f008b
:106e60000f014100020757008e0178008b0f570079
:106e7000010034008b0178000300e0002b00350096
:106e80000040eb008e8f51000a003d0082fa2f0077
:106e90000f01410003004100b0489000f0c0b30072
:106ea000e7cf500003003c000040eb00010037003a
:106eb000810178008300e90034fb2f000f024200bb
:106ec0000101420012427800804f5200f8ff320068
:106ed000ef4f500001003a000449e8000100e000d3
:106ee00007003d008301e8004f90970064004000d8
:106ef000c0979f0022fb2f000f01410002003700c6
:106f000032fb2f000f01410003007800050037001d
:106f1000e24078008100fb005fb29700e4c0780097
:106f2000017178000000e900f9ff3b005c08900067
:106f30000000e000ea003d000300e900500e980068
:106f4000e70037005f949700ef9497007f959700d4
:106f50008f9d97006022b8006033b8000800be0023
:106f60000a01be00160507000000e00005003d0014
:106f70000bf0a200d8979f00e9979f00fa979f0017
:106f80008b9f9f0070592700cf9097000088b90011
:106f9000026a2800130020006d05070064045000f9
:106fa000c8979f0015003b0063041400c0ff2f002a
:106fb000000464000800ea00c0979f005f909700fb
:106fc000ef9097007f9197008f9997000a282100f2
:106fd000070037000808a300030032003a02be0091
:106fe0002a03be00fc0507000884d100680545009f
:106ff0000800e000f7ff3c001a0037000800e0003e
:107000001c003200c0ff2f0000046400c8979f00de
:107010000a2821006000b8000200200003ff2300be
:10702000070037000808a300030032003a02be0040
:107030002a03be00e80507000884d1006805450062
:107040000800e000f7ff3c000002be000203be00a3
:107050005f909700ef9097007f9197008f9997002e
:10706000e1040700d0979f00e1979f00f2979f00ef
:10707000839f9f005c0f900060c6b30080cf5600d6
:10708000040032006000200061c4b30081cf5600cc
:1070900002003a00cf9097006a8040000e0740003f
:1070a000f30f5700010034003e01200000c3b3007d
:1070b000a0779f003bfb2f008f85450035003700f0
:1070c0005fb09700efb097007fb197008fb997003e
:1070d000920507000004be00680757004240a9005f
:1070e00010003400b90507000002be000203be0014
:1070f0005fb09700efb097007fb197008fb997000e
:107100002b0607006022b80046782d00771924006e
:10711000b1050700d0979f00e1979f00f2979f006d
:10712000839f9f00e88545008a0020000801be007b
:107130000c003700a400200005002000a0fd2f0057
:107140000f004000850207005fa89700efa8970096
:107150007fa997008fb1970004c3b30084654100f5
:107160000001be00e00f5100e08f5900060034001e
:107170000a05e900e10f4500eeff3a000200370082
:1071800000c3b300806578000a05e900fcff3b00fe
:10719000e88545000e00e0000d0034005f90970088
:1071a000ef9097007f9197008f999700d0b79f003d
:1071b000e1b79f00f2b79f0083bf9f006022b80035
:1071c0006033b800830407000000e000bcff3c000f
:1071d00031fb2f008f804000818555004f91970033
:1071e00067004100c0979f00020037008b05e9004f
:1071f0000000e900010178008200780003c3b300b9
:10720000b1cf1100f9ff3200c0979f00dc09900058
:1072100061c6b30081cf56000300320061c4b300e1
:1072200081cf560002003a000000e8000900370054
:107230001000200051c6b30081cf56000500320077
:107240000d40780050c4b2000080fb000000e9004f
:107250004f00de00830140008b8f5100010034009d
:107260008b0178000300e0001d00350000c3b3006f
:107270008b8f510006003d0062c2790069404000da
:1072800041c3b300814f520001003c0069405000ef
:107290008300e9008100410001003700840178008b
:1072a0000302e90001037800a142780080cf520078
:1072b000faff320091c3b300814f500001003a0041
:1072c000054be8000400e00005003d000201e90074
:1072d0008301e8004f9297000402e800c4979f00e2
:1072e0004f9297008d4078000c007800f70207005d
:1072f0004f0778004f06be004f05be004f04be008a
:10730000cf04b10000000600889fbe000004780092
:10731000e68440001900d0004500de00f27f200026
:10732000820f500010003a00000ceb009904780026
:107330006f816400200020001b003a0021019000b2
:107340000200e00018003a00110190000200e00085
:1073500015003a00100020001100e0001200320079
:1073600020002000100037000000e00004003a0078
:10737000010078000e0207000000e00008003c0059
:10738000f20028001901610001fe2300810c710048
:1073900021c02f00010c40000080eb0002003700ec
:1073a000000ceb000000eb004f04be0000000600e4
:1073b000fc874700889fbe008a9fbe008c9fbe004e
:1073c0008e1f78000006780080c5b30080cf500083
:1073d0000a0032007740400080cf50000a0032009f
:1073e0006940400080cf50000b003200303821004f
:1073f00080bf9f00ae0020000a0037002237210026
:1074000082bf9f00060037003338210083bf9f00f2
:107410008e002000030037003438210084bf9f0015
:107420000e0120003c02be002c03be000605be007b
:107430000404be0040c6b30080cf500003003200f9
:107440006540400080cf50000b003a00e00f520032
:10745000e08f5a00e00f5b00e08f5b0006003d000c
:107460006000b8006011b800040450008584580022
:107470000605590087855900e80f570004003200bf
:1074800040002000f00f570038003a00010037009c
:1074900030002000e00f5400e08f5c00e00f5d0042
:1074a000e08f5d0004003a00dc0890008d012000b0
:1074b0000100e000060032008e00e90088806000d4
:1074c0008fba9700e5c07800f1ef9f007d012000a2
:1074d000800078008100e900050033008b05d100b1
:1074e0000a85d3008984d3000884d300f9ff3700cc
:1074f000089ebe000a96be00120037008d06e90005
:107500008e00e900848060000fb99700e2c1780026
:1075100082fd2f000f01410003f17e008000780002
:107520008100e900050033008783d1000683d30082
:107530008582d3000482d300f9ff3700049ebe0089
:107540000696be003c02be002c03be00e00f5200b7
:10755000e08f5a00e00f5b00e08f5b008b0034008f
:107560000d00e000e5ff3c00880037002c60900033
:1075700081c6b300814f50000b00320006003c0072
:107580000004e00008003200e6c05000814f5000c7
:107590004e003a0004003700c1c6b300814f5000ce
:1075a0004a003a00210037000800e00004003a00d9
:1075b0005c0890008d0120000000e0000600320011
:1075c000110009000e84d8000fb99700e2c07800be
:1075d000f1ef9f007d012000110009000e84d8000a
:1075e0000a003700110009000e04d8008d06e900da
:1075f0000e81b900020454008fb8970061417c00ed
:1076000081fd2f008f80400082f07e000004780012
:107610000800e000020032000d00e000f1ff3c0035
:10762000cfc4de00614db90025003700e00f5400e3
:10763000e08f5c0004003a005c0890008d0120009f
:107640000000e000070032006171b9000800be00d0
:10765000e90407008fb99700e3417800f3ef9f003a
:107660007d0120006171b9000800be00d20407004e
:107670000b0037006171b9000800be00b4030700b9
:107680008d06e90000f1b900020454000fba97001a
:10769000e4427c0084fd2f000f02420005f27e00d0
:1076a0000004be00e00f5000e08f580002003200de
:1076b0000d00e000efff3c004fcdde008a057800b2
:1076c000089ebe000a96be0030003700e00f54004e
:1076d000e08f5c00e00f5d00e08f5d0004003a0089
:1076e0005c0890008d0120000000e00009003200dd
:1076f0006172b900612bb9000800be000a01be002a
:10770000660507000fba970064427800f4ef9f0007
:107710007d0120006172b900612bb9000800be0034
:107720000a01be00560507000d0037006172b9005e
:10773000612bb9000800be000a01be005b0507000e
:107740008d06e90000f2b900040454008fba9700d6
:1077500065427c0085fd2f008f82420084f27e000e
:10776000009ebe000296be003c04be002c05be007a
:10777000e00f5400e08f5c00e00f5d00e08f5d00e3
:10778000020034000d00e000e8ff3c00e80f570065
:1077900010003a000c1090000038a3000d003200d9
:1077a000f78f560006003e0085fd2f008f824200b5
:1077b000e5c07e0000c3b30080cf5000050032005a
:1077c0008d06e90002c3b30081fd2f008f804000c9
:1077d00082f07e0078811600120e98006c009000f6
:1077e00083fd2f008f8141008d804100a5fc0700a3
:1077f0001c089000dc089000810f500006003d003e
:1078000000805000000e98000c1090000040a10075
:10781000001698000f0037000100e0000d003d0049
:107820008c109000f4806000f08f500009003a0046
:107830007c099000fc009000810051000c09900030
:1078400082805000008050004240a90001003400b6
:10785000000e98004f0778004f06be004f05be008f
:107860004f04be00cf01b100000006000400fa0082
:10787000889fbe008a9fbe008c1f7800000478009d
:1078800001067800f80d9000780090008085550082
:1078900008089000808555001808900080855500e4
:1078a0002808900080855500380890008085550094
:1078b00048089000808555000002220090bf9f007c
:1078c00000032300a0bf9f00081090000028a30021
:1078d00015003a000b00e000130034000b0578009f
:1078e0008a047800e20f55000100360029002000cc
:1078f000c801900009017800ee8057005800900000
:1079000003000100500498000000e0008c003200e9
:107910006808900009004000600c980009055500b7
:107920004240a900eeff3c00780190000200e00018
:107930000c003400c80190008c00780058009000c2
:1079400003000100500498008080eb000000e0007c
:107950007c003200e8089000780090000080400031
:10796000600c9800880c90000900e00011003400c1
:1079700009057800e28f5400010036002a0020003b
:10798000c80190000a017800ec8057005800900070
:1079900003000100500498000000e000680032007d
:1079a000680890000a004000600c98008a84540027
:1079b000edff3700180990000200e0000c003400d1
:1079c000c8019000e80090005800900003000100fa
:1079d000500498008080eb000000e0005900320065
:1079e000e80890001808900000804000600c9800a3
:1079f000a80c90000900e00011003400090578008f
:107a0000e28f5400010036002a002000c8019000d7
:107a10000a017800ec805700580090000300010034
:107a2000500498000000e000450032006808900013
:107a30000a004000600c98008a845400edff370073
:107a4000380990000200e0000e003400e8009000c9
:107a50001808900080804000c801900058009000f5
:107a600003000100500498008080eb000000e0005b
:107a700034003200e8089000380890000080400090
:107a8000600c9800c80c90000900e0001100340060
:107a900009057800e28f5400010036002a0020001a
:107aa000c80190000a017800ec805700580090004f
:107ab00003000100500498000000e00020003200a4
:107ac000680890000a004000600c98008a84540006
:107ad000edff3700081090008000eb000028a300a5
:107ae000180032000b00e000160034008b04780010
:107af00009057800e28f5400010036002a002000ba
:107b0000c80190000a017800ee80570058009000ec
:107b100003000100500498000000e000080032005b
:107b2000680890000a004000600c98008a845400a5
:107b30004240a900eeff3c008000eb00010037004e
:107b40008080eb00010078004f0678004f05be00f2
:107b50004f04be000080fa0000000600881f780075
:107b60008a9fbe008c9fbe00000478000205be0004
:107b70000406be000401be000a00be007402070035
:107b8000008cbe000c01be009e03070000055500de
:107b900081855d002a0498003b0498000800780065
:107ba0004f06be004f05be004f04780000000600df
:107bb000e600400011017800050028008502610000
:107bc0006f0161008208780002003200120020007c
:107bd00011003700a0019000120020000300e00017
:107be0000d003a00900190000300e0000a003a0006
:107bf0001000e00008003a0036003700640340003f
:107c00009608780080017800530b7800900978007e
:107c10000408780070015100110278000400e000af
:107c2000f6ff3200130037006402400014037800ae
:107c30004f33de00838141008308730080017800a8
:107c4000d3037800cf3bde00140378000603430023
:107c5000068a7300130278000402420010037800c1
:107c60004f33de00860972009001780003884100de
:107c70000201e90091017800ef8f5100eaff360020
:107c80001000370080017800530378004f33dd0087
:107c90001002d100040873006402400094037800cd
:107ca000cf3bdd001303d1008689730011037800f8
:107cb0004f33dd009401d100030a73009108d10015
:107cc0000201e80091017800ff8f5100edff3e00b6
:107cd000ef886100918872000200780000000600c1
:107ce0000400fa00889fbe0000047800e604440007
:107cf000190078008000d000c508de00f47f200065
:107d0000848f50000e003a00ef0060002000200039
:107d10006b003a00a80090000100e00068003a0003
:107d2000980090000100e00065003a00100020007b
:107d30001800e000620032002000200060003700e0
:107d40000100e0000a003a0008007800c2bf9f006e
:107d5000d3bf9f0096ff0700800078000000eb0073
:107d60004fb99700dfb997000100e00054003c00d4
:107d70004f88de000281400083014800e07f200040
:107d8000800f5100e08f59000d0034001900e00011
:107d900004003d006000b8000200200003ff2f0037
:107da000030037006000b8000200200003ff270036
:107db000009cbe000294be0010002000400037006e
:107dc000e00f5100e08f5900050034004411dd0040
:107dd000f000280019006000800c710037003700a7
:107de0001900780004002800040260006f006000a1
:107df0000040a000800c7800d0fc2f00f1ff2f0085
:107e0000800f5100818f590006003d00840c7800de
:107e10000000eb002004980010049800000ceb0018
:107e2000270037006f014100060037000800780086
:107e3000500c7800e400440011087800990878009c
:107e4000800ceb00700051007001410001fe2f001a
:107e500082804000ef8f4000f4ff35000000ea0010
:107e6000150032008800780070011000d1027800ff
:107e7000822add00980178008019de00038c7200f0
:107e80006404440098027800822add0091017800a1
:107e90008019de0083887200990078000209dd00f5
:107ea000980078008008de00010c710099007800cd
:107eb0000008de00800c7800990c72000080eb0056
:107ec0004f04be000080fa0000000600f087470063
:107ed000889fbe008a9fbe008c9fbe008e1f7800c8
:107ee00000047800814478000205be000406780092
:107ef0000b00e00002003c001b002000ea432100d0
:107f000060c6b30080cf54000e00320060c4b300de
:107f100080cf54000b00320070c6b30080cf5400f5
:107f20000300320070c4b30080cf540099003a00bf
:107f3000e40f46007f00350058089000800f56007f
:107f40007c003d000c06e80060c6b30080cf540002
:107f50001000320060c4b30080cf54000d00320026
:107f6000081090000038a30004003a005808900060
:107f7000808f550001003d005b0c98005808900070
:107f80000c005000500c980002003b000000eb0079
:107f9000500c980018089000e80090000c00e000d9
:107fa00026003c0002c3b300827078000000e800a5
:107fb000100c9800d80890000100e00003003c007d
:107fc000881090000138a30005003200e8009000fe
:107fd000e2c2b300827078000000e800100c980044
:107fe000580890008c00ea00810f500001003d000d
:107ff0000006ea008c00ea00210c9800000646000a
:108000005c0c98008b0f5600010034000b067800c2
:108010003c0c9800e8009000180890000080400098
:108020000c0178008a00780096fa07005808900042
:108030000c0650004c0c9800be0037008c8f550089
:1080400018003d00008040000b0178008a00780095
:108050008cfa07001808900000804500100c98006a
:108060008b0556002b0c9800d80890000100e0000a
:1080700003003c00881090000138a3000600320085
:10808000e8009000e2c2b3008270780038089000e7
:108090000000e800300c980058089000400c980050
:1080a000a4003700008040000c0178008a007800ae
:1080b00074fa07001808900000004600100c9800a1
:1080c0008c855500d80890000100e00003003c00ba
:1080d000881090000138a30005003200e8009000ed
:1080e000e2c2b300827078000000e800100c980033
:1080f00058089000808f55000100340080057800fa
:10810000e800900018089000008040008c004500b6
:108110000b0178005bfa0700180890000b00400084
:10812000100c9800580890008b0550002b0c9800fc
:108130008000370070c6b30080cf540003003200c7
:1081400070c4b30080cf540012003a005808900069
:10815000808f550004003d00081090000038a300f7
:1081600001003a005b0c9800580890000000e900fc
:10817000500c980002003b000000eb00500c9800ef
:1081800070c6b30080cf540009003a0059c6b3004e
:108190000c00370010c6b30080cf54000600320038
:1081a00010c4b30080cf540006003a00040037002a
:1081b00059c4b3000300370009c7b30001003700fa
:1081c00009c5b30018089000e80090009a70780084
:1081d0000000e800100c9800d80890000100e000b2
:1081e00003003c00881090000138a3000500320015
:1081f000e8009000e2c2b300827078000000e8005e
:10820000100c9800580890000000e00010003400a6
:108210008b05e900808f550001003400800578004f
:10822000e800900018089000008040008a00e800f4
:108230000b01780013fa0700180890000b004000ab
:10824000100c9800580890008b0550002b0c9800db
:10825000e80090001808900000804000095878005d
:108260000005e8000c00e00004003500b1c2b300d6
:10827000014878008a06780004003700d1c2b300b4
:10828000014878008a0678000c06ea00fd85570050
:108290000007eb0009003700a20020008c007800e6
:1082a000728057003b0007007fb097008fb897009f
:1082b000816d7800000678000e07e8000c00e000f1
:1082c000f5ff3c00e10f570013003c0050c6b3001f
:1082d00080cf54000300320050c4b30080cf54005c
:1082e00003003a008a06780000c3b300805e78007d
:1082f0000e00e00008003a0000c3b300805e780082
:10830000050037000e07e900fc80570061407f0040
:1083100002c3b300825e40000e00e000f9ff3c00a3
:10832000e800900018089000008040008086560009
:108330003d0c98000810900074006000f00f500091
:108340000e003a00980890007800900000804000ed
:10835000a808900001004000b8089000010040000b
:10836000c808900001004000f8089000810f5000fc
:1083700002003d0000805000000c98004f0778007c
:108380004f06be004f05be004f04be000f01b100f6
:108390000000060080027800010378001100090047
:1083a0000203d80080017800830a78000299b9009e
:1083b00002015300920298000500780000000600b8
:1083c0008f1fd100160307008f87e9000000e0002f
:1083d00000000600809feb00110307008f87e90073
:1083e0000000e000000006002800fa00889fbe00a0
:1083f0008a9fbe008c9fbe0003866b008f00070023
:108400006400e100440032006408e1004a003200e8
:108410006100e100460032006108e10049003200dd
:10842000ec0647006000b8003d02be003d03be0000
:10843000f48657006011b8003d04be003d05be0043
:108440007d0320000b0037000000a0008d06e9002e
:10845000130032000402420085824a0006034b00ea
:1084600087834b00000040008180480002014900e2
:10847000838149000802520089825a000a035b0086
:108480008b835b00f0ff3b000802420089824a00b8
:108490000a034b008b834b008d06e900edff3a0089
:1084a0008482720086827200f707b20087827200af
:1084b00001003200150020001e0490003e0b9000c9
:1084c00006035400e63fb0000368a3000700320033
:1084d0000000a7000500a0008301d1000281d300a5
:1084e0008180d3000080d3000603e8008301d1001f
:1084f0000281d3008180d3000080d3000002eb0012
:108500000482d2002100070003f0a1000cf0a700b4
:1085100003f0a0005d003700640247006408e1003a
:10852000570032003400be003401be00f6ff3700b1
:108530006108e100520032006011b8006000b8002c
:10854000f1ff370003ff270002002000fbff370088
:10855000839f68000100e00002003d006000100001
:10856000e08018000300e00002003d0060011100ff
:10857000e0811900100107004f00e00002003b00fd
:1085800060001000e08018000000060018002000c5
:1085900057002000080453000d003d000600200095
:1085a00097fc2f000740e1001e0034008482720017
:1085b000610260008301d1000281d3008180d30079
:1085c0000080d3000804e800f8ff3a0047002000cc
:1085d0006104600005047400040464000d003200ae
:1085e00061004000e080480060014900e0814900ee
:1085f00003b8a500070032000603e8006538e10073
:1086000004003a008301d1000281d3008180d300ad
:108610000080d300f87f20000830e100030035001f
:10862000080378006000b8006011b8004433dd0032
:10863000f300b200830173000000060068044700e5
:108640000294be000094be00fc0447008694be0065
:108650008494be0009007800ba0207000800780080
:10866000b802070099007800814f70000b003b00b2
:108670000800be00930207004f00b100030037005e
:10868000f3ff2700f2ff2f006110b9004f06be0074
:108690004f05be004f04be000080fa000000060037
:1086a00081037800bdf107000001be006000b80042
:1086b0000478a30013003a006220e10015003e0098
:1086c0000d0039008301d1000281d3008180d300e5
:1086d0008301d1000281d3008180d3008301d100c6
:1086e0000281d3008180d3000538b000c42add00a8
:1086f000f300b2008381720007f0a70003f0a0002e
:1087000000000600f3ff2700f2ff2f006110b90000
:10871000fbff370003ff2700f7ff37001400fa00c4
:10872000889fbe008a9fbe008c9fbe000004be00d2
:108730000205be00680047000a90be000890be0017
:10874000800207000070a7000bf0a100304320005a
:108750009e02900080825200b0fe2f000028e100af
:1087600011003d00b0fc2f000028e100150034008e
:108770001e0990008e0890007e0090000501b00058
:108780000201d1008180d3000080d3008502e8007f
:10879000fbff3a000b00e000bcff3b006000100054
:1087a000e0801800b9ff3700f0ff2f00f1ff27002d
:1087b0000b00e000b5ff3b00010028000000200096
:1087c000b2ff37006000b800b0ff37004f89de000d
:1087d00082017800820237002800fa00889fbe00dc
:1087e0008a9fbe008c9fbe0003866b0093ff07002c
:1087f0000028a30064003a000128a30067003a00a3
:108800000008a30062003a000108a30065003a00d6
:108810001e009000be08900081064000ed3fb100b0
:10882000f4805700ee019000111ab8008e099000f4
:10883000311bb8009e099000311cb800511db800d2
:10884000f485570046000700fe0190003a0007003b
:108850008b85e8003e0007008e099000400007006d
:10886000ee019000340007008b85e8003800070017
:108870008e099000400007009e0990001b18b80068
:10888000890440000a854800fe019000340007007a
:108890008b85e80038000700ee01900030000700eb
:1088a0008e0990001b18b800890440000a85480012
:1088b0000a98a30008003a000402420085824a0098
:1088c00006034b0087834b0008044c0089844c004e
:1088d0000a054d008d06e90084827200850273004e
:1088e0004c3add00850272000100320015002000c4
:1088f000443ade001400b2004538de00cb45dd000e
:108900000b007000c540de00cb4ddd008b80700099
:108910004549de00cb55dd000b017100c551de007d
:108920000d03780019ff070003f0a1000cf0a70069
:1089300003f0a00055ff37001b18b8008502400067
:1089400006834800e0834b0060044c0007003700ba
:108950001b18b8000603400087834800faff370061
:108960001b18b8008703400008844800e0844c00ce
:1089700060054d00000006001b18b8000804400008
:1089800089844800faff37000108a3003cff3a0041
:108990005800be005801be00e3ff37000008a300e6
:1089a00037ff3a0009047800f9ff370000000000a3
:1089b00007f0a2001c0137006022b8000602200068
:1089c0000000d0008180d2000482d2008582d200d3
:1089d0000000a0000202520083825a00030031000e
:1089e0000202420083824a000000a1000603e9005f
:1089f000f3ff3a0000000600efff07000400be008e
:108a000000000600020ab900001bb9000200b8000d
:108a1000810042008100430000000600889fbe00e4
:108a20008a9fbe0030044200b0844a0030054b00eb
:108a300090854b006000b1000898be000a90be000f
:108a40000440e10005c8e10006d0e10007d8e100dc
:108a500002003100680040001008e8004f05be0029
:108a60004f04be0000000600889fbe008a9fbe0023
:108a70003004be002005be000418540005985c00b8
:108a800006185d0007985d00110020000440e10019
:108a900005c8e10006d0e10007d8e1000100390077
:108aa0008000eb00108810004f05be004f04be0090
:108ab000000006001200fa00889fbe008a9fbe00d8
:108ac0008c9fbe00e0b79f00f1b79f0082bf9f0060
:108ad00093bf9f000605be000404be000000eb002b
:108ae000d0b79f00c0b79f00b0b79f00a0b79f004e
:108af00090b79f000006eb005fb19700cfb09700e2
:108b0000820141003fb097000200e00004003d00f8
:108b1000370007007e805700c0ff070003003700c2
:108b2000330007007e805700cfff0700dfb69700b5
:108b30000d00e0000c0035006fb29700ffb2970007
:108b40000fbb97009fbb9700100020000100200082
:108b50006011b8000002720081827200020373008b
:108b6000838373001b0007000c06e800010420004b
:108b7000810f5600e0ff3a000d00e00004003d00c8
:108b80000802be000a03be007e805700a3ff070054
:108b90005fa897000000e00005003a001fb29700b0
:108ba000afb297003fb39700cfb39700090007001b
:108bb0006fb09700ffb097000fb997009fb997006b
:108bc0004f06be004f05be004f04be000080fa00f5
:108bd000000006000100070000000600a4b79f0087
:108be000b5b79f00c6b79f00d7b79f00000006002b
:108bf0004f09de0082817100b3b79f004f01de0094
:108c00008180400082807000a1b79f008fb09700e4
:108c10004f09de00000040000200700090b79f0086
:108c20007fa897004f01de008180400082807000a5
:108c300081b79f000d0007004f3ade0000004000a2
:108c400004007000f0af9f0008000700040242001b
:108c500085824a0006034b0087834b00dfff070035
:108c60000802be000a03be00000006002fb29700f3
:108c7000bfb297004fb39700dfb397000000060024
:108c8000881f780018002000881f780089ff0700df
:108c90008f87e9004f04780000000600801feb007a
:108ca00084ff07008f87e90000000600889fbe0050
:108cb0008a9fbe00e00f5000e08f5800e00f59007f
:108cc000e08f59000c003d006044b8006055b800ca
:108cd0000000540081805c0002015d0083815d0022
:108ce000180020001500070008003d0018000700cc
:108cf0000004eb00050037000004eb000f00070044
:108d000002003d001200070018002000dcff0700f1
:108d10000800e000060032006022b8006033b800ae
:108d20000000520081805a0002015b0083815b00d9
:108d30004f05be004f04be0000000600e00f5200c9
:108d4000e08f5a00e00f5b00e08f5b000000060040
:108d50006044b8006055b8000402540085825c008d
:108d600006035d0087835d0000000600889fbe004b
:108d70008a9fbe008c1f7800e00f5000e08f5800e3
:108d8000e00f5900e08f59000d003d006044b8002d
:108d90006055b8000000540081805c0002015d0055
:108da00083815d001c0020000820e10009a8e1008b
:108db0000ab0e1000bb8e1000d003d0008003700eb
:108dc0000006eb00e00f5200e08f5a00e00f5b005e
:108dd000e08f5b0006003d006044b8006055b800bd
:108de0000402540085825c0006035d0087835d00f9
:108df000aaff07000c00e000060032006022b80065
:108e00006033b8000000520081805a0002015b000c
:108e100083815b004f0678004f05be004f04be0003
:108e200000000600000000002800fa00889fbe0035
:108e30008a9fbe008c9fbe00070678008786690067
:108e40000c003b00030478008704780008f0a100c0
:108e500009f0a100840f5000858f5800860f59003b
:108e6000890f5c00030033000cf0a20001003a00ff
:108e70000cf0a100f1fd07006400e1005f0032008a
:108e8000780147006408e100610032006c0147008e
:108e9000748557003200be001201be003a04be00c5
:108ea0001a05be001e039000be0a90008503530001
:108eb00006003d000004fd008104fd000205fd00e8
:108ec0008305fd008703ea00050378000df8a30081
:108ed0000400320060041400e0841c0060051d00e2
:108ee000e0851d006022b8007d0320000d38e10000
:108ef0008006eb000b0039004433dd00f300b200c4
:108f00008301730039003700848272000d027800fb
:108f1000e10664008b85d1000a85d3008984d300e3
:108f20000884d3008703e900f7ff3b0008004000f6
:108f3000898048000a0149008b81490004003b00f8
:108f400060001000e080180060011900e081190045
:108f50000358a300090032008d82720084827200df
:108f6000610260008301d1000281d3008180d300bf
:108f70000080d3000603e8001b0037000348a3006d
:108f800017003a000600e000170034000603e9006d
:108f90000d00a30000004800818048000201490044
:108fa000838149000348a3000f003a000600e00057
:108fb000090034000603e9000000400081804800f9
:108fc000020149008381490001003a000003eb00df
:108fd0000348a300f5ff32006022b800020037000a
:108fe000848272006182660068fd070003f0a100c0
:108ff0000cf0a70003f0a000a4fd370064014700b7
:109000006408e10002003a000df8a3009cfd3a005c
:109010003200be001201be009cfd370000000000bf
:10902000889fbe008a9fbe008c9fbe000404be00c5
:109030000605be00809fbe00829fbe002f00070075
:10904000040678000800be000a01be002b000700dd
:10905000840678004f03be004f02be008d4f76009d
:109060007fb0970013003300f0ff2f008b8f6b0051
:1090700006003b000d0666000c00a7000a00370042
:1090800007f0a600100020000a003700880f5200e9
:10909000898f5a008a0f5b008b8f5b0003003900b9
:1090a0001000200001003e000000200007f0a70093
:1090b0000000ea004f06be004f05be004f04be0090
:1090c00000000600e48240001078a3000700320090
:1090d000640240001178a3003400be001401be00f9
:1090e000040032000330a700000006003500be0077
:1090f0001501be000330a0000000060005ff270098
:1091000005826100070032000428e10001003200fe
:10911000240005000600070001003a004400050095
:109120000408050002000700f9ff3a0014000500da
:109130006f826100810270008502710085027200f9
:1091400000000600800078005002be005003be0000
:109150004439de00f700b200f37f20000301610014
:10916000090032000218e10016003a008501720081
:1091700083017300838173000008200015003a000a
:109180004000200013003700850172008301730046
:109190008381730005003a0004a8be0006a8be0043
:1091a000100020000b0037000201e9000402420019
:1091b00085824a0006034b0087834b000748a300c3
:1091c000f9ff32000740a00004a8be0006a8be00b8
:1091d0002000200080009800920098000000060007
:1091e000881f7800030478000300e00007003d00ba
:1091f00060001000e080180060011900e081190093
:1092000002003b0001f02d000300370004000700be
:1092100008f0a70003f0a0004f047800000006004b
:10922000889fbe00008270000402710004827100f9
:109230002400320036432000c50020008383cf0085
:109240000a0039000541b1008283cf0007003900d0
:109250000541b1008183cf00040039000541b10010
:109260008083cf00010039000541b10085c3530060
:109270006022b800120032000a003b0084827200b3
:10928000610260008301d1000281d3008180d3009c
:109290000080d3000603e8008743e800f7ff3a00a8
:1092a00007003700000040008180480002014900ab
:1092b000838149000603e9008743e900f9ff3a008a
:0c92c000b2fc07004f04be0000000600d6
:020000040000fa
:1092cc007e7e00007e7e00007e7e00007e7e0000a2
:1092dc007e7e00007e7e00007e7e00007e7e000092
:1092ec007e7e00007e7e00007e7e00007e7e000082
:1092fc007e0d00000a000000426c00007565000045
:10930c00427500007320000046690000726d000079
:10931c0077610000726500003a20000025730000a0
:10932c000d0a000000540000727900002048000073
:10933c00454c0000502000006f720000203f0000e0
:10934c000d0a000000230000200000002000000097
:10935c00424f00004f5400004c4f000041440000ad
:10936c004552000000520000656200006f6f000063
:10937c00746900006e670000206900006e740000c4
:10938c006f200000626f00006f7400006c6f0000b3
:10939c0061640000657200000d0a000000420000cc
:1093ac0054000000434f00004e46000049470000a7
:1093bc000043000056430000004f00004e00000028
:1093cc00534500005420000048460000505f000048
:1093dc00434f00004e460000494700003d4f00003f
:1093ec004e2000004f4e0000204f00004e20000089
:1093fc004f4e0000204f00004e2000004f46000052
:10940c00460000004f460000460000005345000097
:10941c005420000048460000505f0000434f0000fd
:10942c004e460000494700003d4f000046460000f4
:10943c00204f00004e2000004f4e0000204f000037
:10944c0046460000204f00004e2000004f46000012
:10945c00460000004846000050000000484600004e
:10946c00503a0000204f00006e0d00000a00000072
:10947c0048460000503a0000204f0000666600008d
:10948c000d0a0000004c000049430000454e00004e
:10949c0053450000004100005054000058000000eb
:1094ac0025730000202500007320000025730000a8
:1094bc00202500007320000025730000004d0000e3
:1094cc0047410000494e00000042000054200000bb
:1094dc004d6900006320000047610000696e0000c8
:1094ec002053000065740000207400006f3a0000e7
:1094fc002025000030320000580d00000a0000004a
:10950c004d6900006320000047610000696e000097
:10951c0020270000253000003258000027200000d2
:10952c006f750000742000006f6600002072000050
:10953c00616e0000676500003a20000043300000b7
:10954c00202d000020440000360d00000a00000011
:10955c004d420000494100005300000053650000db
:10956c007420000074680000652000004d69000044
:10957c006320000042690000617300002047000076
:10958c00656e000065720000617400006f7200006f
:10959c00004d000050520000454100004d500000ad
:1095ac000053000065740000207400006865000022
:1095bc00204d00006963000020500000726500001f
:1095cc002d4100006d70000000520000454200006b
:1095dc004f4f000054000000504100004952000061
:1095ec00005500004e5000004149000052000000a0
:1095fc004e4100004d45000000500000494e000057
:10960c000056000045520000534900004f4e000028
:10961c00004700004554000000490000425500007e
:10962c00530000004c4300004d0000004552000068
:10963c0052000000547200006170000020430000d2
:10964c006f7500006e740000733a0000200d00006e
:10965c000a00000020200000202000004f730000b2
:10966c00636900006c610000746f000072200000e0
:10967c0046610000696c00007572000065730000a3
:10968c003a200000256400000d0a000000200000b4
:10969c00202000002041000064640000726500007e
:1096ac007373000020460000616900006c750000b7
:1096bc0072650000733a000020250000640d000064
:1096cc000a0000002020000020200000537400003d
:1096dc00616300006b20000046610000696c0000b3
:1096ec0075720000657300003a20000025640000cc
:1096fc000d0a00000020000020200000204d00007a
:10970c00617400006820000046610000696c000074
:10971c0075720000657300003a200000256400009b
:10972c000d0a00000020000020200000204e000048
:10973c00564d000020460000616900006c75000069
:10974c0072650000733a000020250000640d0000d3
:10975c000a000000202000002020000047650000c7
:10976c006e650000726100006c2000004661000014
:10977c00696c000075720000657300003a200000ef
:10978c00256400000d0a00000020000020200000cd
:10979c00204c000061730000742000005472000023
:1097ac00617000003a200000253000003278000083
:1097bc000d0a00000055000049000000554900004a
:1097cc00204d00006f640000653a0000204300004b
:1097dc0044350000330d00000a000000554900001c
:1097ec00204d00006f640000653a0000204e000020
:1097fc00617600006967000061740000696f000009
:10980c006e0d00000a00000055490000204d0000bc
:10981c006f640000653a0000204d000049440000d0
:10982c000d0a000000550000492000004d6f00009b
:10983c00646500003a2000004d49000044200000ff
:10984c002f2000004e610000766900006761000067
:10985c00746900006f6e00000d0a000000550000d6
:10986c00492000004d6f0000646500003a200000a4
:10987c0042750000736900006e6500007373000090
:10988c00204e0000617600006967000061740000e2
:10989c00696f00006e0d00000a00000055490000c1
:1098ac00204d00006f640000653a0000204e00005f
:1098bc006f7400002073000065740000206f0000be
:1098cc0072200000496e0000766100006c69000097
:1098dc00640d00000a000000444100004300000039
:1098ec00504300004d35000031320000323a000088
:1098fc002049000032530000535400004154000032
:10990c0020250000303200005820000028300000d4
:10991c007835000045290000205b0000256400001c
:10992c005d0d00000a000000504300004d350000a2
:10993c0031320000323a0000205000005752000033
:10994c005354000041540000202500003032000028
:10995c00582000002830000078370000362900001d
:10996c00205b0000256400005d0d00000a00000073
:10997c00504300004d35000031320000323a0000f7
:10998c00205600006f6c0000756d00006520000013
:10999c00636f00006e66000069670000757200005e
:1099ac0065640000207400006f200000253000006a
:1099bc00325800000d0a000000490000325300002c
:1099cc00005700004d38000038300000343a0000d9
:1099dc0020440000657600006963000065490000c2
:1099ec00443a0000202500003032000058250000c9
:1099fc00303200005820000052650000763a00001a
:109a0c0020250000640d00000a000000574d0000e6
:109a1c0038380000303400003a2000005350000069
:109a2c004453000054410000542000002530000035
:109a3c00325800002028000030780000304300002d
:109a4c00292000005b250000645d00000d0a000069
:109a5c00005700004d38000038300000343a000048
:109a6c00204900004e5400005354000041540000a3
:109a7c002025000030320000582000002830000063
:109a8c007830000042290000205b000025640000b3
:109a9c005d0d00000a00000050570000524f0000fe
:109aac004646000000410000757400006f2d000058
:109abc00506f000077650000722000004f660000b8
:109acc00663a0000204f00006e0d00000a000000f6
:109adc0041750000746f00002d5000006f7700007e
:109aec0065720000204f0000666600003a200000fe
:109afc004f660000660d00000a0000005649000089
:109b0c004e0000005665000068690000636c0000a0
:109b1c0065200000564900004e3a00002025000048
:109b2c0073250000642500006425000064250000f6
:109b3c0064250000640d00000a000000524500007e
:109b4c0053450000540000005452000041500000e6
:109b5c0053000000534500004e4400000053000029
:109b6c0045540000004300004f4d0000464f0000dc
:109b7c0052540000004200004c4900004e4b0000c3
:109b8c0045520000530000004c4f0000434b0000b6
:109b9c0000310000300000003230000000550000a1
:109bac004e4c00004f4300004b000000504f000093
:109bbc0053310000005000004f53000030000000f3
:109bcc0047410000494e0000004400005350000083
:109bdc00004900004e5000005554000000410000a8
:109bec004e4100004c4f000047000000444900006b
:109bfc0047490000544100004c00000031000000b7
:109c0c00320000003300000034000000350000007a
:109c1c00496e0000766100006c6900006420000051
:109c2c0055490000204d00006f64000065200000c5
:109c3c0073700000656300006966000069650000d0
:109c4c00640d00000a000000494700004e000000af
:109c5c00414c000057410000595300004f4e00008a
:109c6c00004c00004f470000005300005953000007
:109c7c00004900006e760000616c00006964000011
:109c8c002050000061720000616d000065740000de
:109c9c006572000073200000666f000072200000e7
:109cac0053450000542000004c4f0000470d0000ad
:109cbc000a000000544500004c000000544900000c
:109ccc004d450000004c00004f4300004b5300007a
:109cdc00004300004c4500004152000000520000bf
:109cec0045530000544f0000524500000030000066
:109cfc00003400003431000030300000004200001d
:109d0c006c75000065420000757300000053000084
:109d1c0065720000696100006c2000004e75000047
:109d2c006d620000657200003a200000257500008d
:109d3c000d0a000000420000756900006c64000010
:109d4c002044000061740000653a000020250000ea
:109d5c00642f0000256400000d0a0000004800007c
:109d6c00454c0000500000003f0000004176000010
:109d7c00616900006c610000626c000065200000ed
:109d8c00436f00006d6d0000616e00006473000095
:109d9c003a0d00000a0000002020000020200000e6
:109dac00424f00004f5400004c4f00004144000053
:109dbc0045520000202d000020520000656200007a
:109dcc006f6f000074200000696e0000746f00005b
:109ddc002074000068650000206200006f6f0000b6
:109dec00746c00006f61000064650000722000005c
:109dfc00696d00006d65000064690000617400000d
:109e0c00656c0000790d00000a00000020200000a5
:109e1c002020000042540000204300004f4e000060
:109e2c0046490000472000002d2000004765000037
:109e3c00742000007468000065200000424300009c
:109e4c003132000037200000436f00006e660000c6
:109e5c00696700007572000061740000696f000092
:109e6c006e0d00000a0000002020000020200000e1
:109e7c00425400002043000056430000204f0000d5
:109e8c004e2f00004f460000462000002d20000001
:109e9c00456e0000616200006c650000206f0000e0
:109eac00722000004469000073610000626c0000c5
:109ebc0065200000436c000065610000722000000a
:109ecc00566f0000696300006520000043610000cc
:109edc007074000075720000650d00000a0000002f
:109eec0020200000202000004254000020480000e8
:109efc0046500000204f00004e2f00004f4600003f
:109f0c00462000002d200000456e0000616200001c
:109f1c006c650000206f0000722000004469000096
:109f2c0073610000626c0000652000004846000070
:109f3c00502e0000204700006574000020740000c3
:109f4c0068650000204800004650000020530000c7
:109f5c0074610000747500007320000077690000c4
:109f6c00746800006f750000742000006120000010
:109f7c0070610000726100006d2e00000d0a00007f
:109f8c00002000002020000020420000542000008f
:109f9c004d470000414900004e2000007820000091
:109fac002d20000053650000742000007468000030
:109fbc00652000004d69000063200000676100000f
:109fcc00696e0000207400006f20000078200000f3
:109fdc0077680000657200006520000078200000a2
:109fec0069730000206f000063740000616c000056
:109ffc0020430000302d0000443600000d0a000004
:10a00c00002000002020000020420000542000000e
:10a01c004d50000052450000414d00005020000002
:10a02c004f4e00002f4f000046460000202d000030
:10a03c00204500006e610000626c0000652000008d
:10a04c0074680000652000006d69000063720000f8
:10a05c006f700000686f00006e65000020700000db
:10a06c00726500002d6100006d700000207300000f
:10a07c006f2000006e6f00006e2d00004f45000039
:10a08c00206d000069630000726f000070680000b2
:10a09c006f6e000065730000207700006f72000087
:10a0ac006b200000776500006c6c00000d0a00004e
:10a0bc00002000002020000020420000542000005e
:10a0cc005041000049520000202d000020450000a6
:10a0dc006e610000626c0000652000007061000081
:10a0ec0069720000696e0000672000006d6f00004f
:10a0fc00646500000d0a0000002000002020000014
:10a10c0020420000542000004e4100004d4500004c
:10a11c00203c00006e6100006d6500003e200000d8
:10a12c002d200000536500007420000074680000ae
:10a13c00652000006d6f0000647500006c65000008
:10a14c00206e0000616d0000652c00002075000081
:10a15c0070200000746f00002033000032200000db
:10a16c006368000061720000730d00000a000000bb
:10a17c00202000002020000042540000205000004d
:10a18c00494e0000203c0000706900006e3e00004b
:10a19c00202d000020530000657400002074000086
:10a1ac0068650000206d00006f640000756c000095
:10a1bc0065200000706900006e2c00002075000006
:10a1cc0070200000746f0000203400002064000038
:10a1dc006967000069740000730d00000a0000003c
:10a1ec0020200000202000004254000020520000db
:10a1fc00454200004f4f0000542000002d2000006d
:10a20c0052650000626f00006f7400002074000043
:10a21c006865000020420000433100003237000026
:10a22c000d0a000000200000202000002042000049
:10a23c0054200000554e00005041000049520000cf
:10a24c00202d0000205500006e7000006169000098
:10a25c0072200000616c00006c200000646500003e
:10a26c0076690000636500007320000066720000d0
:10a27c006f6d000020740000686500002042000033
:10a28c0043310000323700000d0a000000200000ae
:10a29c002020000020420000542000005645000001
:10a2ac0052530000494f00004e2000002d200000aa
:10a2bc0047650000742000007468000065200000f1
:10a2cc004243000031320000372000005665000088
:10a2dc0072730000696f00006e200000496e000070
:10a2ec00666f00000d0a0000002000002020000016
:10a2fc00204700004554000020440000414300006a
:10a30c00202d00002047000065740000206900002b
:10a31c006e6600006f200000667200006f6d00001a
:10a32c00207400006865000020500000434d0000c0
:10a33c00353100003232000020440000414300005f
:10a34c000d0a000000200000202000002047000023
:10a35c00455400002045000052520000202d000002
:10a36c002047000065740000207400006865000040
:10a37c0020450000727200006f7200002063000024
:10a38c006f7500006e740000657200000d0a00000d
:10a39c000020000020200000204700004554000051
:10a3ac002049000042550000532000002d200000e1
:10a3bc0047650000742000006465000062750000b1
:10a3cc0067200000696e0000666f000020660000c8
:10a3dc00726f00006d2000007468000065200000a2
:10a3ec0049420000757300000d0a000000200000b7
:10a3fc00202000002047000045540000205500009c
:10a40c00492000002d20000047650000742000004a
:10a41c007468000065200000637500007272000013
:10a42c00656e00007420000055490000204d0000ae
:10a43c006f640000650d00000a0000002020000081
:10a44c002020000047450000542000004932000045
:10a45c00532000002d2000005265000061640000b4
:10a46c002074000068650000205700004d38000083
:10a47c003830000034200000494e0000542f0000fa
:10a48c00535000004420000053740000617400001d
:10a49c00757300002072000065670000697300008e
:10a4ac0074650000727300000d0a000000200000ab
:10a4bc0020200000204700004554000020560000da
:10a4cc00494e0000202d0000205200006561000064
:10a4dc0064200000746800006520000073740000a4
:10a4ec006f72000065640000207600006568000053
:10a4fc00696300006c65000020560000494e0000a6
:10a50c000d0a000000200000202000002052000056
:10a51c00454200004f4f0000542000002d20000049
:10a52c0052650000626f00006f7400002074000020
:10a53c006865000020640000657600006963000017
:10a54c00650d00000a000000202000002020000003
:10a55c005345000054200000434f00004d460000be
:10a56c004f52000054200000424c0000494e0000a5
:10a57c004b4500005253000020780000202d0000b5
:10a58c002053000065740000207400006865000012
:10a59c00206300006f6d0000666f00007274000095
:10a5ac00206200006c6900006e6b00006572000098
:10a5bc007320000062650000747700006565000080
:10a5cc006e20000031200000616e0000642000004d
:10a5dc00380d00000a0000002020000020200000a0
:10a5ec005345000054200000434f00004d4600002e
:10a5fc004f520000542000004c4f0000434b000011
:10a60c0020780000202d0000204c00006f6300001b
:10a61c006b2000007468000065200000636100007e
:10a62c007220000061740000207400006865000056
:10a63c002067000069760000656e0000204b00006a
:10a64c004d2f0000682e000020310000302c00003f
:10a65c0020320000302000006f720000204f0000fc
:10a66c00464600000d0a00000020000020200000db
:10a67c002053000045540000204300004f4d0000c3
:10a68c00464f000052540000205500004e4c000074
:10a69c004f4300004b200000782000002d200000cc
:10a6ac00556e00006f6300006b20000074680000a2
:10a6bc0065200000636100007220000061740000de
:10a6cc0020740000686500002067000069760000b7
:10a6dc00656e000020690000676e00006974000060
:10a6ec00696f00006e200000706f0000736900003d
:10a6fc00746900006f6e00002e200000504f0000a7
:10a70c00533000002c200000504f0000533100004b
:10a71c00206f0000722000004f460000460d000024
:10a72c000a000000202000002020000053450000fb
:10a73c005420000044410000432000004741000029
:10a74c00494e000020780000782000002d200000e9
:10a75c005365000074200000746800006520000040
:10a76c00504300004d350000313200003220000013
:10a77c0067610000696e000020660000726f0000c7
:10a78c006d2000003078000030300000202d0000db
:10a79c0020300000784300004620000028680000ac
:10a7ac006967000068650000722000006973000092
:10a7bc00206c00006f77000065720000290d00000e
:10a7cc000a0000002020000020200000534500005b
:10a7dc00542000004453000050200000494e00005b
:10a7ec005055000054200000414e0000414c000028
:10a7fc004f4700002f440000494700004954000017
:10a80c00414c0000202d0000205300006574000016
:10a81c002074000068650000204300004420000004
:10a82c0043680000616e0000676500007220000044
:10a83c004453000050200000696e00007075000049
:10a84c00740d00000a0000002020000020200000f1
:10a85c005345000054200000494700004e200000e2
:10a86c004f4e00002f4f0000464600002f410000c5
:10a87c004c57000041590000534f00004e2000007f
:10a88c002d200000536500006e6400002074000051
:10a89c006865000020690000676e000069740000a4
:10a8ac00696f00006e20000073740000617400007a
:10a8bc0075730000206d000065730000736100006b
:10a8cc0067650000206f000072200000636f0000bd
:10a8dc006e6600006967000075720000652000005c
:10a8ec007468000065200000426c00007565000073
:10a8fc004275000073200000746f0000206100009e
:10a90c0073730000756d0000652000007468000012
:10a91c0065200000696700006e6900007469000022
:10a92c006f6e00002069000073200000616c000055
:10a93c007761000079730000206f00006e0d00003d
:10a94c000a000000202000002020000053450000d9
:10a95c00542000004c4f00004720000078200000dd
:10a96c004f4e00002f4f000046460000202d0000e7
:10a97c0020430000686100006e6700006520000045
:10a98c006c6f000067670000696e000067200000b4
:10a99c00666f000072200000782000002842000042
:10a9ac00542c00002049000042550000532c00009c
:10a9bc0020530000595300002c2000005549000082
:10a9cc00290d00000a0000002020000020200000bb
:10a9dc00534500005420000050570000524f000017
:10a9ec0046460000204f00004e2f00004f4600004e
:10a9fc00462000002d200000456e00006162000022
:10aa0c006c650000206f000072200000646900007b
:10aa1c0073610000626c000065200000617500002d
:10aa2c00746f0000207000006f77000065720000ea
:10aa3c00206f0000666600000d0a00000020000078
:10aa4c00202000002053000045540000205400003a
:10aa5c00454c0000204f00004e2f00004f460000d8
:10aa6c00462000002d200000456e000061620000b1
:10aa7c006c6500002f4400006973000061620000e7
:10aa8c006c650000206f000075740000707500008c
:10aa9c0074200000617300002074000068650000e1
:10aaac0020540000435500000d0a00000020000057
:10aabc0020200000205300004554000020540000ca
:10aacc00494d00004520000048480000204d000082
:10aadc004d2000002d200000536500007420000064
:10aaec007468000065200000494b00004520000000
:10aafc00546900006d6500000d0a00000020000084
:10ab0c002020000020530000455400002055000078
:10ab1c0049200000782000002d2000005365000023
:10ab2c007420000074680000652000005549000086
:10ab3c00207400006f200000782c000020770000ab
:10ab4c006865000072650000207800003a0d000076
:10ab5c000a0000002020000020200000202000001f
:10ab6c0020200000782000003d200000312e000045
:10ab7c002043000044350000332000002842000030
:10ab8c0075730000696e000065730000732000008f
:10ab9c0052610000646900006f2900000d0a00007a
:10abac0000200000202000002020000020200000b9
:10abbc0020780000203d0000203200002e200000f4
:10abcc00424d000042540000202800004e6100005d
:10abdc007669000067610000746900006f6e000008
:10abec00290d00000a000000202000002020000099
:10abfc002020000020200000782000003d200000d4
:10ac0c00332e0000204d0000494400002028000095
:10ac1c004d7500006c740000692d0000496e000039
:10ac2c00666f00002044000069730000706c000027
:10ac3c0061790000290d00000a00000020200000ae
:10ac4c0020200000202000002020000078200000a0
:10ac5c003d200000342e0000204200004d42000038
:10ac6c00542000002f2000004d490000440d00002e
:10ac7c000a000000202000002020000020200000fe
:10ac8c0020200000782000003d200000352e000020
:10ac9c002042000075730000696e000065730000af
:10acac00732000004e6100007669000067610000af
:10acbc00746900006f6e00000d0a00000020000097
:10accc00202000002052000045530000544f00008b
:10acdc0052450000202d000020460000756c00003d
:10acec006c79000020520000657300006574000050
:10acfc002074000068650000204200006c750000a4
:10ad0c006542000075730000206100006e64000055
:10ad1c002042000043310000323700002074000054
:10ad2c006f20000066610000637400006f72000009
:10ad3c00792000006465000066610000756c0000fd
:10ad4c00747300000d0a0000002000002020000099
:10ad5c002056000045520000534900004f4e0000a1
:10ad6c00202d0000204700006574000020740000b6
:10ad7c0068650000204200006c7500006542000010
:10ad8c0075730000204800006172000064770000b9
:10ad9c0061720000652f0000536f000066740000a4
:10adac00776100007265000020560000657200009b
:10adbc00736900006f6e0000730d00000a00000044
:10adcc00436f00006d6d0000616e00006420000098
:10addc006e6f000074200000666f0000756e00003e
:10adec00642e0000205400007279000020480000fe
:10adfc00454c0000502000006f720000203f000006
:10ae0c000d0a000023200000004f00004b0d000035
:10ae1c000a23000020000000425400003a200000e9
:10ae2c00536500006e640000204300006f6d00004d
:10ae3c006d6100006e640000202700002573000087
:10ae4c0027000000564f00004c5500004d450000f7
:10ae5c002025000064200000257300000054000031
:10ae6c004f4e0000452000002573000000540000e8
:10ae7c004f470000474c0000455f00005652000051
:10ae8c002025000064000000425400003a2000001d
:10ae9c00556e0000616200006c65000020740000bb
:10aeac006f200000544f0000474700004c45000045
:10aebc005f560000522000002d2000004846000084
:10aecc00502000006c6900006e6b000020750000c3
:10aedc006e6f0000706500006e650000640000007d
:10aeec00534500005420000055410000525400000e
:10aefc005f4300004f4e000046490000473d0000f4
:10af0c00256c00006c7500002025000073200000eb
:10af1c002564000000530000455400002050000040
:10af2c00524f0000464900004c450000533d0000c4
:10af3c002564000020300000202500006420000063
:10af4c003020000025640000202500006420000053
:10af5c0031200000312000003020000030200000a3
:10af6c003120000030000000534500005420000048
:10af7c00504900004e3d00002573000000530000b6
:10af8c0045540000204e0000414d0000453d00009e
:10af9c00257300000053000045540000204e0000b3
:10afac00414d0000455f0000534800004f52000027
:10afbc00543d000025730000005300004554000070
:10afcc00204d000055530000494300005f4d000028
:10afdc0045540000415f0000444100005441000012
:10afec003d4f000046460000005300004554000051
:10affc00204d000055530000494300005f4d0000f8
:10b00c0045540000415f00004441000054410000e1
:10b01c003d4f00004e00000053450000542000003e
:10b02c00434f000044450000433d000025640000f0
:10b03c002025000073000000534500005420000040
:10b04c00425400005f5600004f4c00005f4300006c
:10b05c004f4e000046490000473d000025580000b7
:10b06c00202500006420000025640000202500003d
:10b07c0064000000534500005420000042540000be
:10b08c005f53000054410000544500005f43000032
:10b09c004f4e000046490000473d0000256400006b
:10b0ac0020250000640000005345000054200000df
:10b0bc0041550000544f0000434f00004e4e00001d
:10b0cc003d250000640000005345000054200000a2
:10b0dc0041550000444900004f5f00004449000006
:10b0ec0047490000544100004c3d0000257300000e
:10b0fc00202500007320000025730000202500008f
:10b10c00732000004f46000046000000534500002d
:10b11c005420000041550000444900004f5f0000de
:10b12c00414e0000414c00004f4700003d250000ff
:10b13c00642000002564000020250000642000002d
:10b14c00257300000053000045540000204100000e
:10b15c0055440000494f00003d25000064200000cc
:10b16c0025640000004f0000504500004e200000f8
:10b17c00257300002025000073000000434c0000e4
:10b18c004f5300004520000025640000004d0000d6
:10b19c0055530000494300002025000064200000a6
:10b1ac00504c00004159000000420000543a00008d
:10b1bc00205500006e610000626c000065200000ec
:10b1cc00746f0000205000004c410000592000001a
:10b1dc002d2000004156000052430000502000007a
:10b1ec006c6900006e6b0000207500006e6f000033
:10b1fc00706500006e650000640000004d55000095
:10b20c00534900004320000025640000205000003a
:10b21c00415500005345000000420000543a000024
:10b22c00205500006e610000626c0000652000007b
:10b23c00746f000020500000415500005345000081
:10b24c00202d000020410000565200004350000009
:10b25c00206c0000696e00006b200000756e000011
:10b26c006f700000656e000065640000004c00000b
:10b27c0049530000540000004c49000043450000b5
:10b28c004e530000450000004c49000043450000af
:10b29c004e5300004520000025730000004c0000b8
:10b2ac0049430000454e0000534500002025000096
:10b2bc00733d000025730000004100005652000051
:10b2cc00435000005f4d000045540000415f0000fa
:10b2dc00444100005441000020250000640000009f
:10b2ec00425400003a200000556e000061620000dc
:10b2fc006c650000207400006f2000006765000082
:10b30c00742000004d650000746100006461000051
:10b31c0074610000202d00002041000056520000f6
:10b32c0043500000206c0000696e00006b20000090
:10b33c00756e00006f700000656e000065640000a3
:10b34c00004e0000414d0000452000002573000018
:10b35c00004d00005553000049430000202500001b
:10b36c0064200000464600005f520000454c00007f
:10b37c00454100005345000000420000543a0000d3
:10b38c00205500006e610000626c0000652000001a
:10b39c00746f000020530000454500004b20000056
:10b3ac00464f00005257000041520000442000005c
:10b3bc002d20000041560000524300005020000098
:10b3cc006c6900006e6b0000207500006e6f000051
:10b3dc00706500006e650000640000004d550000b3
:10b3ec005349000043200000256400002046000063
:10b3fc00465f00005052000045530000530000000f
:10b40c004d55000053490000432000002564000006
:10b41c00204600004f5200005741000052440000eb
:10b42c0000420000543a0000205500006e610000fc
:10b43c00626c000065200000746f00002046000064
:10b44c004f5200005741000052440000202d0000d4
:10b45c00204100005652000043500000206c0000b8
:10b46c00696e00006b200000756e00006f700000ac
:10b47c00656e00006564000000420000545f00002f
:10b48c005354000041540000452000002573000077
:10b49c00202500007300000025730000004300000d
:10b4ac00564300005f430000464700002025000083
:10b4bc007300000043560000435f00004346000049
:10b4cc0047200000257300002025000064200000a8
:10b4dc0025640000004e00004200000032320000e3
:10b4ec0038300000203000003030000030200000e8
:10b4fc0031410000303000002025000030320000c7
:10b50c005830000030200000303000003030000097
:10b51c002025000030320000582500003032000099
:10b52c005820000030300000303000002030000087
:10b53c00303000003020000030300000303000008f
:10b54c00203000003030000030200000303000008f
:10b55c00303000002030000030320000302000007d
:10b56c003030000030300000202500003032000068
:10b57c0058250000303200005800000057420000ef
:10b58c00003200003238000034200000303000005f
:10b59c00303000002031000041300000302000002d
:10b5ac002530000032580000303000002030000000
:10b5bc0030300000302000002530000032580000f0
:10b5cc0025300000325800002030000030300000e0
:10b5dc0030200000303000003030000020300000ff
:10b5ec0030300000302000003030000030300000df
:10b5fc0020300000303000003020000030300000df
:10b60c0032300000203000003030000030200000cc
:10b61c002530000032580000253000003258000060
:10b62c00004f000046460000004f00004e00000096
:10b63c00434100004c4c0000202500006420000019
:10b64c00524500004a4500004354000000430000ee
:10b65c00414c00004c2000002564000020450000f7
:10b66c004e44000000430000414c00004c20000000
:10b67c0025640000204100004e5300005745000097
:10b68c00520000004d5500005349000043200000bb
:10b69c002564000020520000455700005f52000056
:10b6ac00454c00004541000053450000004d000092
:10b6bc005553000049430000202500006420000081
:10b6cc0052450000575f00005052000045530000e7
:10b6dc00530000004d55000053490000432000006a
:10b6ec002564000020420000414300004b5700003d
:10b6fc004152000044000000413200004450000060
:10b70c000041000056520000435000000048000069
:10b71c00465000000020000000420000543a000097
:10b72c002025000073000000415600005243000029
:10b73c00505f00004d4500004449000041000000ee
:10b74c0054490000544c0000453a000000410000f0
:10b75c005254000049530000543a000000410000cc
:10b76c004c420000554d00003a00000042540000cd
:10b77c003a20000074690000746c0000653d000004
:10b78c00257300002c6100007274000069730000c6
:10b79c00743d0000257300002c6100006c620000f9
:10b7ac00756d00003d25000073000000415600003f
:10b7bc0052430000505f0000504c00004159000003
:10b7cc0000420000543a0000205000006c61000060
:10b7dc00796900006e6700000041000056520000bd
:10b7ec00435000005f5000004155000053450000dd
:10b7fc0000420000543a0000205000006175000027
:10b80c0073650000640000004132000044500000e9
:10b81c005f53000054520000454100004d5f000092
:10b82c0053540000415200005400000042540000e8
:10b83c003a200000506c000061790000696e000035
:10b84c00672000005b4100003244000050200000e3
:10b85c005374000072650000616d000020530000fd
:10b86c0074610000727400005d0000004132000041
:10b87c00445000005f53000054520000454100004a
:10b88c004d5f00005355000053500000454e000022
:10b89c0044000000425400003a20000050610000b7
:10b8ac007573000065640000205b000041320000ed
:10b8bc0044500000205300007472000065610000c9
:10b8cc006d2000005375000073700000656e000061
:10b8dc00645d000000430000414c00004c5f000020
:10b8ec00414300005449000056450000004300004d
:10b8fc00414c00004c5f0000454e0000440000002d
:10b90c00434100004c4c00005f4900004e430000d6
:10b91c004f4d0000494e000047000000434100001d
:10b92c004c4c00005f4f000055540000474f000086
:10b93c00494e0000470000004c4900004e4b0000ef
:10b94c0000420000543a0000204e000065770000d1
:10b95c00204100006374000069760000652000003f
:10b96c00446500007669000063650000005000002b
:10b97c004c410000594900004e47000000420000b5
:10b98c00543a00002050000061690000726500000c
:10b99c0064200000446500007669000063650000c7
:10b9ac002025000073000000434c00004f530000a2
:10b9bc00455f00004f4b000000420000543a00006d
:10b9cc00204300006c6f00007365000064200000d1
:10b9dc006c6900006e6b00002025000073000000f5
:10b9ec004f500000454e00005f4f00004b00000020
:10b9fc00425400003a2000004f700000656e0000b9
:10ba0c002025000073200000666f000072200000eb
:10ba1c004944000020250000730000004f50000036
:10ba2c00454e00005f450000525200004f5200008e
:10ba3c00004e0000414d0000450000004254000043
:10ba4c003a2000004e650000772000005061000095
:10ba5c0069720000696e00006720000050720000df
:10ba6c006f660000696c0000652000002573000003
:10ba7c00202d00003e200000257300000042000035
:10ba8c00756900006c6400003a000000425400002c
:10ba9c003a200000426f00006f7400002043000049
:10baac006f6d0000706c0000657400006500000094
:10babc00534300004f5f00004f500000454e000004
:10bacc0000530000434f00005f4300004c4f000048
:10badc005345000000530000544100005445000041
:10baec00004300004f4e00004e4500004354000040
:10bafc00414200004c4500005b4f00004e5d0000d1
:10bb0c00004300004f4e00004e450000435400001f
:10bb1c00414200004c4500005b4f000046460000cf
:10bb2c005d00000044490000534300004f560000e4
:10bb3c0045520000414200004c4500005b4f0000a4
:10bb4c004e5d00000044000049530000434f0000cc
:10bb5c005645000052410000424c0000455b00007d
:10bb6c004f460000465d000000420000543a0000c1
:10bb7c00204700006f740000205300007461000027
:10bb8c007475000073200000257300002025000050
:10bb9c0073000000425400003a200000525800008c
:10bbac0020510000756500007565000020540000f0
:10bbbc00696d0000656f00007574000000000000e6
:10bbcc005379000073740000656d00002050000074
:10bbdc006f77000065720000204400006f77000052
:10bbec006e21000000480000616e0000646c0000d3
:10bbfc00657200003a200000436500006e7400007e
:10bc0c00726100006c2000004c6f0000636b000040
:10bc1c0073200000756e00006c6f0000636b0000f9
:10bc2c006564000000480000616e0000646c000058
:10bc3c00657200003a200000436500006e7400003d
:10bc4c00726100006c2000004c6f0000636b000000
:10bc5c00732000006c6f0000636b000065640000d3
:10bc6c0000480000616e0000646c0000657200000a
:10bc7c003a20000041740000746500006d700000f3
:10bc8c00746900006e670000207400006f200000d3
:10bc9c0072650000736f00006c7600006520000078
:10bcac007061000069720000696e0000672000007e
:10bcbc0065720000726f00007200000048610000a5
:10bccc006e6400006c650000723a000020410000b8
:10bcdc0032440000502000006c6900006e6b0000c4
:10bcec00206300006c6f000073650000642000008e
:10bcfc002d2d00002041000074740000656d0000c3
:10bd0c0070740000696e000067200000746f000002
:10bd1c00206300006f6e00006e650000637400000d
:10bd2c000041000032440000500000004861000057
:10bd3c006e6400006c650000723a00002047000041
:10bd4c0069760000696e00006720000075700000c5
:10bd5c00206f00006e2000004254000020630000a1
:10bd6c006f6e00006e65000063740000696f000068
:10bd7c006e000000486100006e6400006c650000fd
:10bd8c00723a0000204e00006f2000004465000055
:10bd9c007669000063650000202d00002d20000056
:10bdac0041740000746500006d7000007420000088
:10bdbc00636f00006e6e0000656300007469000024
:10bdcc006f6e000000480000465000000048000064
:10bddc00616e0000646c0000657200003a20000087
:10bdec004e6f000074200000636f00006e6e000048
:10bdfc0065630000746900006e6700002074000029
:10be0c006f2000006e650000772000006465000064
:10be1c0076690000636500002025000064200000a6
:10be2c00256400002025000064000000445300003d
:10be3c00502000004465000074650000637400002d
:10be4c0065640000004700005420000044650000b9
:10be5c00746500006374000065640000004c000011
:10be6c00434d000020440000657400006563000031
:10be7c0074650000640000004d490000442000007f
:10be8c004465000074650000637400006564000084
:10be9c0000440000657400006563000074650000d8
:10beac00642000004d490000442000002f200000b9
:10bebc00424d000042540000205500004900000093
:10becc004465000074650000637400006564000044
:10bedc00204d00004944000020550000490000009e
:10beec00424d0000425400002044000065740000e4
:10befc00656300007465000064000000524100009e
:10bf0c004420000044650000746500006374000068
:10bf1c0065640000004d0000464c0000204f0000fe
:10bf2c0046460000004d0000464c0000205000002a
:10bf3c005245000053530000004d0000464c0000d9
:10bf4c00204800004f4c000044000000546f0000db
:10bf5c00676700006c65000020560000520000006e
:10bf6c00476f000074200000564900004e3a000054
:10bf7c0020250000732500006425000064250000c6
:10bf8c006425000064250000640000004465000086
:10bf9c0074650000637400006564000020560000a6
:10bfac00494e000020430000686100006e670000ed
:10bfbc00653a000020250000732500006425000070
:10bfcc006425000064250000642500006400000066
:10bfdc00466100006c6c000062610000636b000045
:10bfec00207400006f200000434400003533000033
:10bffc0000480000616e0000646c00006572000077
:10c00c003a200000556e00006b6e00006f77000048
:10c01c006e2000005665000068690000636c00002b
:10c02c006520000044650000746500006374000026
:10c03c006564000000440000657400006563000046
:10c04c0074650000642000004e650000772000003d
:10c05c005665000068690000636c000065200000f4
:10c06c0054790000706500003a200000453400004f
:10c07c00362f00005a3400000044000065740000a4
:10c08c006563000074650000642000004e650000cc
:10c09c00772000005665000068690000636c0000a2
:10c0ac006520000054790000706500003a20000003
:10c0bc0045330000382f000045330000392f0000b5
:10c0cc0045350000332000002d2000004c6f00008f
:10c0dc00772000004f420000430000004465000040
:10c0ec00746500006374000065640000204e00005d
:10c0fc006577000020560000656800006963000049
:10c10c006c6500002054000079700000653a000056
:10c11c0020450000333800002f4500003339000063
:10c12c002f45000035330000202d00002048000072
:10c13c0069670000682000004f42000043000000c7
:10c14c00486100006e6400006c650000723a0000eb
:10c15c002044000069730000616200006c650000ff
:10c16c00206300006f6e00006e65000063740000b9
:10c17c002d610000626900006c6900007479000098
:10c18c00004200004d5700004330000031530000c6
:10c19c0000440000657400006563000074650000d5
:10c1ac0064200000424d0000425400002055000065
:10c1bc0049000000424d0000574d00003031000096
:10c1cc0053000000446500007465000063740000b7
:10c1dc00656400002042000075730000696e000069
:10c1ec0065730000732000004e6100007620000093
:10c1fc0055490000005500006e610000626c0000a3
:10c20c0065200000746f0000206900006465000068
:10c21c006e7400006966000079200000475400002d
:10c22c00204f0000533a000020250000730000004e
:10c23c00466100006c6c000062610000636b0000e2
:10c24c00207400006f2000004344000035330000d0
:10c25c002055000049000000486100006e64000099
:10c26c006c650000723a000020530000656e0000ff
:10c27c00642000004344000043200000737400005d
:10c28c00617400007573000020700000726500007e
:10c29c00656d00007074000069760000656c00002c
:10c2ac0079000000486100006e6400006c650000bd
:10c2bc00723a000020490000676e000069740000ab
:10c2cc00696f00006e2000004f6e000000560000e9
:10c2dc0020300000204e00002043000036200000db
:10c2ec004c20000034000000486100006e64000027
:10c2fc006c650000723a000020520000657100006d
:10c30c007565000073740000204c0000434d000064
:10c31c002052000065640000756e0000646100002e
:10c32c006e74000020440000617400006100000085
:10c33c00486100006e6400006c650000723a0000f9
:10c34c00205300006574000020540000656c000050
:10c35c0065700000686f00006e65000020560000dc
:10c36c006f6c0000756d0000653a00002025000020
:10c37c006400000041320000445000000041000005
:10c38c0056520000435000000000000048460000d8
:10c39c0050000000c0e10000c5e10000cbe100004e
:10c3ac00cce100005061000069720000696e000071
:10c3bc00673a0000204f00006e0000005061000042
:10c3cc0069720000696e0000673a0000204f00009f
:10c3dc0066660000004300006c650000617200009e
:10c3ec002050000061690000726900006e67000057
:10c3fc007300000042610000636b00000044000009
:10c40c00657600006963000065730000005300004e
:10c41c0065740000746900006e6700007300000012
:10c42c004d6500006e7500003a2000004d61000063
:10c43c00696e0000004d0000656e0000753a00004a
:10c44c002044000061730000686200006f6100000e
:10c45c0072640000004d000065740000616400000f
:10c46c0061740000613a000020500000617200000d
:10c47c0074790000004d00006574000061640000d8
:10c48c0061740000613a00002043000068750000f0
:10c49c006e6b0000004d00006574000061640000cc
:10c4ac0061740000613a0000204f000066660000d5
:10c4bc0000540000656d0000707300003a2000000d
:10c4cc004f66000066000000546500006d700000af
:10c4dc00733a0000204300006f6f00006c61000095
:10c4ec006e74000000530000657400007469000055
:10c4fc006e670000732000003e20000055490000cc
:10c50c000044000061730000686200006f6100006d
:10c51c0072640000004d0000616900006e20000094
:10c52c004d6500006e750000004100007574000040
:10c53c006f7000006c610000793a0000204f000021
:10c54c006666000000410000757400006f7000000a
:10c55c006c610000793a0000204f00006e00000072
:10c56c00566f00006c7500006d6500003a200000ed
:10c57c002d2500006464000042000000566f00008e
:10c58c006c7500006d6500003a2000002b32000035
:10c59c003464000042000000566f00006c7500000f
:10c5ac006d6500003a20000030640000420000007d
:10c5bc00566f00006c7500006d6500003a2000009d
:10c5cc002b2500006464000042000000445300006e
:10c5dc00503a0000204400006967000069740000b4
:10c5ec00616c000000440000535000003a20000031
:10c5fc00416e0000616c00006f670000005300008a
:10c60c0065740000746900006e6700007320000000
:10c61c003e20000041750000646900006f000000be
:10c62c00486100006e6400007366000072650000d3
:10c63c00653a0000204f00006666000000480000cc
:10c64c00616e000064730000667200006565000096
:10c65c003a2000004f6e0000004d0000696300009e
:10c66c002042000069610000733a0000204f000076
:10c67c0066660000004d0000696300002042000067
:10c68c0069610000733a0000204f00006e0000004a
:10c69c004d6900006320000047610000696e0000d6
:10c6ac003a2000002569000064420000005300009d
:10c6bc0065740000746900006e6700007320000050
:10c6cc003e200000436100006c6c0000696e0000ad
:10c6dc006700000025640000004c00006f63000040
:10c6ec006b3a000020310000306b00006d2f000011
:10c6fc00680000004c6f0000636b00003a200000e3
:10c70c00323000006b6d00002f680000004c000000
:10c71c006f6300006b3a0000204f0000666600005b
:10c72c00005500006e6c00006f6300006b3a000057
:10c73c00205000006f7300002031000000550000f5
:10c74c006e6c00006f6300006b3a0000205000001c
:10c75c006f73000020300000005500006e6c00006c
:10c76c006f6300006b3a0000204f0000666600000b
:10c77c00004200006c6900006e6b000065720000e6
:10c78c00733a0000202500006400000043610000a3
:10c79c00723a000020450000337800002f4500005d
:10c7ac003533000000430000617200003a200000a5
:10c7bc0045340000362f00005a34000000430000be
:10c7cc00617200003a200000556e00007365000095
:10c7dc00740000005365000074740000696e000062
:10c7ec0067730000203e0000204300006f6d0000c6
:10c7fc00666f000072740000002d0000204e0000d7
:10c80c006f740000205000006c610000796900001a
:10c81c006e670000202d0000005500006e6b0000bc
:10c82c006e6f0000776e00002054000069740000e9
:10c83c006c650000005500006e6b00006e6f000010
:10c84c00776e0000204100007274000069730000d4
:10c85c0074000000556e00006b6e00006f770000d6
:10c86c006e200000416c0000627500006d0000003d
:10c87c004e6f0000204400006576000069630000e4
:10c88c006500000025640000630000007c7c000053
:10c89c00004200006c750000657400006f6f0000b2
:10c8ac0074680000003e00002000000042540000ac
:10c8bc002020000000250000732000002d20000027
:10c8cc0025730000202d00002025000073000000bf
:10c8dc004e4f000020540000415000004500000065
:10c8ec004e4f000020430000440000004e4f00005b
:10c8fc00204400004953000043000000465700004c
:10c90c003a20000025730000004200007569000009
:10c91c006c7400003a200000256400002f250000f4
:10c92c0064000000532f00004e3a00002025000048
:10c93c00750000005365000074740000696e0000ff
:10c94c0067730000203e000020410000626f000071
:10c95c007574000000200000202000002000000062
:10c96c00416200006f75000074000000417500000a
:10c97c00646900006f000000436100006c6c0000f3
:10c98c00696e000067000000436f00006d660000d8
:10c99c006f72000074000000554900000000000098
:10c9ac000d0a000049420000757300003a20000097
:10c9bc005241000044200000502f00004e3a00006d
:10c9cc00202500006425000064250000642500007b
:10c9dc00642500006425000064250000642000002c
:10c9ec00485700003a200000253000003264000057
:10c9fc0020530000573a0000202500006425000059
:10ca0c006420000042750000696c0000643a00006c
:10ca1c002025000064250000642f00002564000020
:10ca2c00256400000d0a0000000d00000a490000fa
:10ca3c0042750000733a0000204c00004d200000ad
:10ca4c00444900003a200000256400002043000007
:10ca5c00493a000020250000640d00000a00000087
:10ca6c004c69000067680000742000004d6f0000e6
:10ca7c00647500006c6500003a2000004c4d00000d
:10ca8c0045330000380000004c6900006768000066
:10ca9c00742000004d6f0000647500006c65000090
:10caac003a2000004c4300004d0000004c6900008f
:10cabc0067680000742000004d6f00006475000072
:10cacc006c6500003a2000004c4300004d5f0000f4
:10cadc00410000004c6900006768000074200000f1
:10caec004d6f0000647500006c6500003a2000007a
:10cafc004c4300004d5f000049490000004c000011
:10cb0c006967000068740000204d00006f6400002d
:10cb1c00756c0000653a0000204c0000434d00008d
:10cb2c005f49000049490000004c000069670000a3
:10cb3c0068740000204d00006f640000756c0000ec
:10cb4c00653a0000204c0000434d00005f49000096
:10cb5c00560000004c69000067680000742000005b
:10cb6c004d6f0000647500006c6500003a200000f9
:10cb7c004c5300005a0000004c690000676800002c
:10cb8c00742000004d6f0000647500006c6500009f
:10cb9c003a2000004c5300005a5f000032000000a5
:10cbac000d0a000049420000757300003a20000095
:10cbbc0047540000205000002f4e00003a20000087
:10cbcc002563000025630000256300002563000039
:10cbdc00256300002563000025630000204400004d
:10cbec00493a00002025000064200000485700004e
:10cbfc003a2000002564000020530000573a000042
:10cc0c00202500006420000042750000696c0000c3
:10cc1c00643a00002025000063250000632f00000b
:10cc2c0025630000256300000d0a00000049000088
:10cc3c0042750000733a0000205500006e61000040
:10cc4c00626c000065200000746f0000206400001e
:10cc5c00656300006f640000652000006e610000d9
:10cc6c007669000067610000746900006f6e000057
:10cc7c002074000079700000650000005b25000046
:10cc8c006c6c0000755d00002045000052520000e5
:10cc9c004f5200003a20000049420000757300001a
:10ccac003a20000052580000204900006e76000027
:10ccbc00616c000069640000204c0000656e00008f
:10cccc0067740000682000005b25000064200000f1
:10ccdc002d20000025300000325800005d3a000085
:10ccec002000000025300000325800002000000019
:10ccfc000d0a0000005b0000256c00006c75000044
:10cd0c005d2000004445000042550000473a0000f9
:10cd1c002049000042750000733a000020520000c8
:10cd2c00585b0000256400005d3a00002000000004
:10cd3c005b530000454c0000465d000000490000bc
:10cd4c0042750000733a00002025000030320000cc
:10cd5c00582000002d3e000020250000303200003d
:10cd6c00582000004c6500006e67000074680000dd
:10cd7c003a20000025640000202d0000204900000e
:10cd8c006e760000616c00006964000020430000b6
:10cd9c0068650000636b0000737500006d00000097
:10cdac005b2500006c6c0000755d000020450000e8
:10cdbc00525200004f5200003a200000494200003d
:10cdcc00757300003a200000525800002042000009
:10cddc007566000066650000722000005469000052
:10cdec006d6500006f750000742000005b2500006d
:10cdfc00645d00003a200000005b000023ef00009f
:10ce0c00263300005bc30000ef2600003321000036
:10ce1c0042020000200c000000880000010c000001
:10ce2c00000b0000010c000000410000010c000090
:10ce3c0000400000010c000000430000010c000049
:10ce4c0000420000010c0000000b0000010000007b
:10ce5c00574d000038380000585800002052000090
:10ce6c0065730000706f00006e6400006564000064
:10ce7c002077000069740000682000002564000021
:10ce8c00005700004d3800003858000058200000b2
:10ce9c0052650000737000006f6e00006465000046
:10ceac0064200000776900007468000020250000f1
:10cebc006420000064750000726900006e67000059
:10cecc00206900006e69000074690000616c00004c
:10cedc00697a000061740000696f00006e00000048
:10ceec00574d000038380000585800002052000000
:10cefc0065730000706f00006e64000065640000d4
:10cf0c00207400006f200000506f00006c6c00005b
:10cf1c00005700004d380000385800005820000021
:10cf2c0066610000696c00006564000020740000fc
:10cf3c006f2000007365000074200000504c00004e
:10cf4c004c4300004c4b0000205b000025640000ab
:10cf5c005d000000574d00003838000058580000a4
:10cf6c0020660000616900006c6500006420000010
:10cf7c00746f0000207300006574000020530000e3
:10cf8c00504400004d4f000044450000205b000061
:10cf9c00256400005d000000574d0000383800008b
:10cfac005858000020660000616900006c650000a4
:10cfbc0064200000746f0000207300006574000092
:10cfcc00205400005853000052430000205b000026
:10cfdc00256400005d000000574d0000383800004b
:10cfec005858000020660000616900006c65000064
:10cffc0064200000746f0000207300006574000052
:10d00c00204100004946000054580000205b0000fd
:10d01c00256400005d000000574d0000383800000a
:10d02c005858000020660000616900006c65000023
:10d03c0064200000746f0000207300006574000011
:10d04c00204100004946000052580000205b0000bf
:10d05c00256400005d000000574d000038380000ca
:10d06c005858000020660000616900006c650000e3
:10d07c0064200000746f00002073000065740000d1
:10d08c00205000004c4c00005f4e0000205b000064
:10d09c00256400005d000000574d0000383800008a
:10d0ac005858000020660000616900006c650000a3
:10d0bc0064200000746f0000207300006574000091
:10d0cc00206600006972000073740000206200008a
:10d0dc0069740000206f000066200000504c0000b6
:10d0ec004c5f00004b2000005b250000645d0000dd
:10d0fc00005700004d380000385800005820000040
:10d10c0066610000696c000065640000207400001a
:10d11c006f20000073650000742000007365000030
:10d12c00636f00006e6400002062000069740000f0
:10d13c00206f000066200000504c00004c5f000087
:10d14c004b2000005b250000645d000000570000d0
:10d15c004d3800003858000058200000666100006f
:10d16c00696c000065640000207400006f200000f2
:10d17c007365000074200000746800006972000080
:10d18c006420000062690000742000006f660000db
:10d19c00205000004c4c00005f4b0000205b000056
:10d1ac00256400005d000000574d00003838000079
:10d1bc005858000020660000616900006c65000092
:10d1cc0064200000746f0000207300006574000080
:10d1dc002053000050440000525800003120000041
:10d1ec005b250000645d0000005700004d38000016
:10d1fc00385800005820000066610000696c00007f
:10d20c0065640000207400006f200000706f000047
:10d21c0077650000722000006f6e0000205b00003c
:10d22c00256400005d00000000480000465000002e
:10d23c003a2000004f6e00000048000046500000ed
:10d24c003a2000004f660000660000004d650000ab
:10d25c00746100003a2000005061000072740000fc
:10d26c00790000004d650000746100003a20000058
:10d27c0043680000756e00006b00000041750000f3
:10d28c00746f0000706c0000617900003a2000009f
:10d29c004f6e000000410000757400006f700000bc
:10d2ac006c610000793a0000204f000066660000b7
:10d2bc0000430000617200003a200000453300007a
:10d2cc00382f000045330000392f00004535000091
:10d2dc003300000043610000723a0000204500005a
:10d2ec00343600002f5a0000340000004f54000068
:10d2fc00204200006c6900006e6b00003a200000b8
:10d30c00330000004f540000204200006c69000004
:10d31c006e6b00003a200000350000004f540000f6
:10d32c00204200006c6900006e6b00003a20000087
:10d33c0031000000436f00006d6600006f7200004a
:10d34c00742000004c6f0000636b0000733a000007
:10d35c00204f00006e000000436f00006d6600005f
:10d36c006f720000742000004c6f0000636b0000b3
:10d37c00733a0000204f0000666600000050000069
:10d38c00726500007373000020530000617600008a
:10d39c0065000000436c0000656100007220000015
:10d3ac005061000069720000696e00006773000034
:10d3bc00004200006c750000657400006f6f000087
:10d3cc00746800000053000065740000746900006c
:10d3dc006e67000073000000446500007669000071
:10d3ec00636500007300000042610000636b000085
:10d3fc000045000064690000740000003c2000003f
:10d40c002020000000200000202000003e00000032
:10d41c0020200000200000004e6f0000204400007f
:10d42c006576000069630000657300002041000010
:10d43c0076610000696c0000616200006c650000a0
:10d44c0000200000436f00006e00000043610000ec
:10d45c00723a0000205500006e73000065740000e5
:10d46c00002000003e0000005061000075730000b9
:10d47c0065640000007c00007c200000002500009a
:10d48c00732000002d20000025730000206f000089
:10d49c006e200000257300000025000073200000a2
:10d4ac002d200000257300000025000073200000d3
:10d4bc006f6e000020250000730000002573000033
:10d4cc00003e000020200000004d000065740000ac
:10d4dc0061000000536500007474000000690000d6
:10d4ec006e67000073000000446500007669000060
:10d4fc000063000065730000200000005061000014
:10d50c006972000000200000202000002020000094
:10d51c0020200000202000002020000020200000ff
:10d52c00202000002020000020200000200000000f
:10d53c005061000069720000696e000067200000f5
:10d54c004f66000066000000506100006972000028
:10d55c00696e0000672000004f6e00000053000051
:10d56c006176000065000000556e000070610000df
:10d57c0069720000656400000053000061760000d1
:10d58c006564000000000000426c0000756500003e
:10d59c00746f00006f7400006800000025730000b9
:10d5ac00202d000020250000732000006f6e00006d
:10d5bc00202500007300000025730000202d0000c2
:10d5cc00202500007300000025730000206f000070
:10d5dc006e20000025730000002500007300000081
:10d5ec00486100006e640000736600007265000004
:10d5fc00653a0000204f00006666000000480000fd
:10d60c00616e0000647300006672000065650000c6
:10d61c003a2000004f6e0000004d000065740000c1
:10d62c00613a000020500000617200007479000023
:10d63c00004d000065740000613a000020430000ba
:10d64c00687500006e6b00000041000075740000ee
:10d65c006f7000006c610000793a0000204f0000f0
:10d66c006666000000410000757400006f700000d9
:10d67c006c610000793a0000204f00006e00000041
:10d68c0043610000723a000020450000333800006e
:10d69c002f450000333900002f45000035330000c2
:10d6ac0000430000617200003a2000004534000085
:10d6bc00362f00005a340000004300006172000055
:10d6cc003a200000556e00007365000074000000e5
:10d6dc004f540000204200006c6900006e6b00008b
:10d6ec003a200000330000004f540000204200009c
:10d6fc006c6900006e6b00003a20000035000000e1
:10d70c004f540000204200006c6900006e6b00005a
:10d71c003a20000031000000436f00006d660000ed
:10d72c006f720000742000004c6f0000636b0000ef
:10d73c00733a000020300000004300006f6d0000c1
:10d74c00666f000072740000204c00006f630000d4
:10d75c006b7300003a20000031000000436c0000a5
:10d76c0065610000722000005061000069720000c9
:10d77c00696e0000677300000050000072650000c5
:10d78c00737300002032000000500000617500002f
:10d79c0073650000640000004e6f00002044000020
:10d7ac0065760000696300006500000045640000b8
:10d7bc0069740000005500006e7000006169000083
:10d7cc007265000064000000536100007665000083
:10d7dc0064000000436f00006e6e00006563000083
:10d7ec00746900006e670000004300006f6e00005b
:10d7fc006e65000063740000656400000053000057
:10d80c0065740000746900006e670000730000000e
:10d81c00486100006e6400007366000072650000d1
:10d82c00653a00002030000000480000616e0000e6
:10d83c006473000066720000656500003a20000009
:10d84c00310000004e6f000020440000657600009f
:10d85c0069630000657300000044000065760000f9
:10d86c0069630000657300000050000061690000ee
:10d87c00726900006e670000204f000066660000b1
:10d88c000050000061690000726900006e670000c2
:10d89c00204f00006e00000000000000504300000c
:10d8ac004d35000031580000582000005265000032
:10d8bc00737000006f6e000064650000642000004f
:10d8cc0077690000746800002025000064000000e7
:10d8dc00504300004d350000315800005820000026
:10d8ec0052650000737000006f6e000064650000ec
:10d8fc006420000077690000746800002025000097
:10d90c006420000064750000726900006e670000fe
:10d91c00206900006e69000074690000616c0000f1
:10d92c00697a000061740000696f00006e000000ed
:10d93c00504300004d3500003158000058200000c5
:10d94c0052650000737000006f6e0000646500008b
:10d95c0064200000746f0000205000006f6c000009
:10d96c006c000000504300004d35000031580000a1
:10d97c005820000066610000696c000065640000be
:10d98c00207400006f200000706f000077650000ad
:10d99c0072200000646f0000776e0000205b0000b6
:10d9ac00256400005d000000504300004d35000070
:10d9bc00315800005820000066610000696c0000be
:10d9cc0065640000207400006f2000007365000087
:10d9dc0074200000564f00004c4c0000205b0000ef
:10d9ec00256400005d000000504300004d35000030
:10d9fc003158000058200000564f00004c4c0000dd
:10da0c002053000065740000207400006f2000009b
:10da1c003078000025300000325800000050000023
:10da2c00434d0000353100005858000020660000be
:10da3c00616900006c65000064200000746f0000d8
:10da4c002073000065740000205600004f4c00004d
:10da5c00522000005b250000645d000000500000b7
:10da6c00434d00003531000058580000205600008e
:10da7c004f4c000052200000536500007420000041
:10da8c00746f000020300000782500003032000058
:10da9c0058000000504300004d3500003158000084
:10daac005820000066610000696c0000656400008d
:10dabc00207400006f200000706f0000776500007c
:10dacc007220000075700000205b000025640000cf
:10dadc005d000000300000003434000031300000e4
:10daec0030000000320000004f46000046000000ed
:10dafc00426c000075650000427500007300000068
:10db0c004465000076690000636500002050000049
:10db1c00726f000076690000736900006f6e000080
:10db2c00656400000d0a000000520000616e0000e8
:10db3c0020550000706700007261000064650000f1
:10db4c00203100002e3100002e3100000d0a0000a3
:10db5c00004c000049430000454e000053450000b6
:10db6c0020430000564300003d33000041360000c6
:10db7c0042200000434200003930000020450000e4
:10db8c0032440000362000004643000038310000cb
:10db9c002030000030300000300000004c49000004
:10dbac00434500004e530000452000004356000042
:10dbbc00433d000033410000364200002044000089
:10dbcc0038310000322000004431000034340000b1
:10dbdc0020460000433800003120000030300000a7
:10dbec003030000000520000616e00002055000033
:10dbfc007067000072610000646500002031000055
:10dc0c002e3100002e3700000d0a000000530000da
:10dc1c004554000020480000465000005f430000bf
:10dc2c004f4e000046490000473d00004f4e00009b
:10dc3c00204f00004e2000004f4e0000204f0000ef
:10dc4c004e2000004f4e0000204f000046460000c2
:10dc5c0000520000616e000020550000706700004b
:10dc6c007261000064650000203100002e3100005c
:10dc7c002e3800000d0a000000520000616e0000fa
:10dc8c0020550000706700007261000064650000a0
:10dc9c00203100002e3100002e3900000d0a00004a
:10dcac0000520000616e00002055000070670000fb
:10dcbc007261000064650000203100002e3100000c
:10dccc002e310000300d00000a0000005200000050
:10dcdc00596f0000004500000049000000410000a1
:10dcec000042000000560000004700000044000005
:10dcfc0000590000650000005a680000005a00003e
:10dd0c0000590000004b0000004c0000004d0000ca
:10dd1c00004e0000004f000000500000000000000a
:10dd2c0053000000540000005500000046000000a5
:10dd3c004b680000005400007300000043680000b2
:10dd4c000053000068000000536800006368000086
:10dd5c0000220000002700000059000075000000a0
:10dd6c0059610000006100000062000000760000b4
:10dd7c0000670000006400000079000065000000ee
:10dd8c007a680000007a0000006900000079000049
:10dd9c00006b0000006c0000006d0000006e0000c5
:10ddac00006f0000007000000072000000730000a3
:10ddbc00007400000075000000660000006b00009d
:10ddcc00680000007473000000630000680000002d
:10dddc0073680000007300006863000068000000b6
:10ddec0065000000797500000079000061000000fa
:10ddfc00796f000000000000d4070000d407000079
:10de0c00d6070000d6070000d8070000d80700008e
:10de1c00da070000da070000dc070000dc0700006e
:10de2c00de070000de070000e0070000e00700004e
:10de3c00e2070000e2070000e4070000e40700002e
:10de4c00e6070000e6070000e8070000e80700000e
:10de5c00ea070000ea070000ec070000ec070000ee
:10de6c00ee070000ee070000f0070000f0070000ce
:10de7c00f2070000f2070000f4070000f4070000ae
:10de8c00f6070000f6070000f8070000f80700008e
:10de9c005b2500006c6c0000755d000020450000e7
:10deac00525200004f5200003a2000005541000031
:10debc00525400005b250000645d00003a20000015
:10decc00004700004552000052200000004f0000a7
:10dedc004552000052200000004600004552000050
:10deec00522000000050000045520000522000005b
:10defc00000d00000a0000000305000013150000cf
:10df0c005b2500006c6c0000755d00002025000096
:10df1c00733a000020250000730d00000a00000079
:10df2c0044450000425500004700000045520000e7
:10df3c00524f000052000000494e0000464f0000b6
:10df4c0000570000415200004e4900004e470000af
:10df5c000000000049320000432000004572000020
:10df6c00726f0000722000002d200000537400001e
:10df7c0061740000757300002069000073200000bc
:10df8c002564000000000000256400002e25000020
:10df9c00642e000025640000001200001314000021
:10dfac0015160000121300001415000016000000d6
:10dfbc002a2a00002a2a0000204200006c7500006a
:10dfcc006542000075730000202a00002a2a000018
:08dfdc002a0000000000000013
:020000040000fa
:10dfe40020019000f19f2f00810061000190a000aa
:10dff4002100980000000600c1409000f0cf5000be
:10e0040008003a008040eb0041409800a0009000d6
:10e014000188a30003003200a000900001b0a10019
:10e024002100980000000600881f78000004780092
:10e0340018009000f280200060417900e34f510005
:10e0440002003e008912070004003700b1120700e5
:10e054001800900021c6b300cb1107004f047800cc
:10e06400000006000a00fa00881f78000004780007
:10e07400a80090000070200080806000808f500015
:10e084003c003a00d0c1b3005a3c07000004e00051
:10e0940038003200684892000004e00003003400b5
:10e0a4000040e900604c9a00320037004848920072
:10e0b400e94f500027003600b84892008180fb00e9
:10e0c400ec80400081004400920020006c805700e6
:10e0d400dedc07000040eb00d0ff9f00ec8057001f
:10e0e40008007800d0ff0700384892000004e000e0
:10e0f40002003a0051c0b300614c9a0069404000ec
:10e10400c8489200814f50000500390020c0b30078
:10e11400604c9a000040eb00304c9a001500370028
:10e12400d0c1b300333c0700e24f500005003a0071
:10e13400604c9a003848920069404000304c9a0084
:10e144000c003700384892000040e800304c9a0038
:10e1540008003700384892000004e00003003a0049
:10e16400ec00440008007800afff070010c0b300c3
:10e17400304c9a004f0478000080fa00000006003a
:10e18400c0409000e2cf500002003200e1cf4000d6
:10e1940005003a0010019000f1802000e2c07800f0
:10e1a400e6cf500004003200e040900010009000e0
:10e1b400751107000300370031c6b3000200780070
:10e1c40071110700000006000600fa00889fbe00d7
:10e1d4008a9fbe008c9fbe0080057800814678002f
:10e1e40002067800834478002f07980010c6b30015
:10e1f400e04598000904e000220032000f05780091
:10e204001f0798000c0078008adc0700004478009f
:10e214008944e80088c444000980fb000080e800c9
:10e22400e01fb200808747000a0078000a0f7800d8
:10e234000881fb008c00780084dc0700894f5400bf
:10e244000600310061c0b3000880fb00017578004e
:10e254000844e80088cf5400fbff3e008984fb009b
:10e26400090545000040eb0070fd9f001b00900075
:10e274001e0178008d4078007f1107009e079000f2
:10e28400040037001b0090000c0178008d407800da
:10e2940079110700ae0790004f06be004f05be007f
:10e2a4004f04be000080fa0000000600ee8747001d
:10e2b400889fbe008a9fbe008c9fbe008e1f780080
:10e2c400800578001b00780030609300e14f500017
:10e2d40006003a008041eb00821d2e008340780046
:10e2e4000b007800b8ff0700050037008041eb0001
:10e2f400421e2e00834078000b007800b2ff070016
:10e304001b027800c46293000504e0000e00320092
:10e314000000eb008044eb00e60220000681b90017
:10e32400210320008280400081004200010032006d
:10e334008944e8000000e80080cf5200f7ff3e0067
:10e344000904e00007003a0043c0b300121f2e0086
:10e3540011c0b3000b0078009bff07008044eb0062
:10e36400050037008041eb00121f2e0011c0b300de
:10e374000b00780094ff07001b04780048609300aa
:10e384000004e0003b0032002cc0b3000045eb0069
:10e39400ee0220008a86fb000ee8b9002003b000dc
:10e3a400000044002e0032000904e00001003200a5
:10e3b4008944e9000ee8b900800678008d00440025
:10e3c400f103b000b20020007a8057001fdc070080
:10e3d4000040eb0090f79f002d03b0000d004400b7
:10e3e40088007800fddb07000000e0000d003a0023
:10e3f4007a8057000fdc0700e94f50000100360017
:10e4040090c0b3008080fb0003c2b3007a81570040
:10e4140003f178000040e8000080fb00a3c2b300d1
:10e42400037178000904e00007003a0063c0b300f8
:10e434008cc151007a8157008c4078000b00780021
:10e4440061ff0700050037008041eb007a81570027
:10e454008c4078000b0078005bff07000c46e80056
:10e464000a45e8001b047800486093008a4f500076
:10e47400c8ff3e0013c0b30002202e0071c0b300d9
:10e484000b00780050ff07001b00900051202e0065
:10e49400fc100700eb4090001b009000ba1007002e
:10e4a40030c0b300c04598004f0778004f06be0047
:10e4b4004f05be004f04be00ef00b100000006008f
:10e4c400889fbe008a9fbe00800478002a402100f5
:10e4d400db3f21000044eb00884178000324a200c4
:10e4e4008381fb008301e900cf19de005a01780023
:10e4f400db4078000900780033ff07000844e80097
:10e50400e54f5400f4ff3a0013c0b30002202e007c
:10e5140071c0b300090078002bff070019009000b8
:10e52400d1202e00d7100700e94090001900900078
:10e534009510070040c0b300c04498004f05be00ca
:10e544004f04be0000000600e7cf500001003a006f
:10e55400dbff070000000600881f78000004780035
:10e56400e0c1b300233b07000004e00006003a00ca
:10e574008041eb0062212e0083407800080078007f
:10e5840011ff0700050037008041eb0012222e0026
:10e5940083407800080078000bff0700d0c1b30067
:10e5a400143b0700e14f500006003a008041eb00a5
:10e5b40012232e0011c0b3000800780002ff0700e8
:10e5c4000d003700e24f500006003a008041eb0096
:10e5d40012242e0011c0b30008007800fafe0700d0
:10e5e400050037008041eb0012252e0011c0b30056
:10e5f40008007800f4fe070000c2b300fd3a0700eb
:10e604000004e00006003a0033c0b300f2252e00f7
:10e6140021c0b30008007800ebfe070005003700b6
:10e6240033c0b300a2262e0021c0b3000800780036
:10e63400e5fe070013c0b30002202e0071c0b30032
:10e6440008007800e0fe07001800900091272e00d3
:10e654008c100700e8409000180090004a10070052
:10e6640090c0b300404498004f04780000000600b6
:10e67400881f7800000478008041eb0072282e0087
:10e684008340780008007800cffe07008041eb004b
:10e6940052202e0011c0b30008007800cafe070003
:10e6a40063c0b300d2202e0021c0b300080078005c
:10e6b400c5fe07001800900011292e0071100700f4
:10e6c400e8409000180090002f10070010c0b3001d
:10e6d400404498004f047800000006001000fa003f
:10e6e400881f78000004780000c4b300c13a070012
:10e6f4000004e00006003a008041eb00b2292e003d
:10e704008340780008007800affe0700050037005a
:10e714008041eb00922a2e008340780008007800a4
:10e72400a9fe070010c4b300b23a070001c3b30046
:10e73400814f50000e0036000080fb000003b10042
:10e74400cf00de00008040000080d1000080fb008c
:10e75400801f7800602b2e00801f7800e1002000cd
:10e7640076805700cdde0700e4875700210037008c
:10e774000004e00007003a00402c2e00801f7800bf
:10e78400e100200074805700c4de07008f87e90091
:10e794001800370001c3b300814f500007003a004e
:10e7a400202d2e00801f7800e10020007480570087
:10e7b400bade07008f87e9000e0037000080fb00f7
:10e7c4000103200000805000cf00de0000804000e4
:10e7d4000080d1000080fb00801f7800e02d2e0017
:10e7e400801f7800e100200076805700abde070030
:10e7f400e48757000040eb00c0ff9f008041780091
:10e804007281570011c0b300080078006efe070043
:10e8140020c4b300773a0700e14f500006003a00e5
:10e8240023c0b300c22e2e00834078000800780075
:10e8340065fe07000500370023c0b300922f2e00a9
:10e8440083407800080078005ffe070013c0b3001f
:10e8540002202e0071c0b300080078005afe0700a1
:10e864001800900051302e0006100700e840900078
:10e8740018009000c40f070060c0b3004044980023
:10e884004f0478000080fa00000006001000fa002f
:10e89400881f78000004780060c3b300553a07006d
:10e8a4000004e00006003a008041eb0062312e00d3
:10e8b400834078000800780043fe07000500370015
:10e8c4008041eb0052322e0083407800080078002b
:10e8d4003dfe070090c3b300463a07000004e00081
:10e8e40006003a008041eb0032332e0011c0b30021
:10e8f4000800780034fe0700050037008041eb0073
:10e9040012342e0011c0b300080078002efe070058
:10e9140080c3b300373a0700f54f500001003600ba
:10e924000040eb000080fb00613e21006140780064
:10e934000000fb00801f7800e0342e00801f780068
:10e94400f10020007680570054de07000040eb0001
:10e9540090ff9f0033c0b3007681570021c0b300fd
:10e964000800780018fe070013c0b30002202e0030
:10e9740071c0b3000800780013fe0700180090006f
:10e98400d1352e00bf0f0700e8409000180090001a
:10e994007d0f070080c0b30040449800e48757000f
:10e9a4004f0478000080fa00000006000400fa001a
:10e9b4009000900070812000008040001080fb00d7
:10e9c400801f780000372e00801f7800410020004f
:10e9d4006880570031de0700e48757000080fa00a2
:10e9e400000006000e00fa00881f7800000478007a
:10e9f40070390700e14f500006003a008041eb00f7
:10ea040032372e008340780008007800eefd0700be
:10ea14000d003700e24f500006003a008041eb0041
:10ea240002382e008340780008007800e6fd0700d5
:10ea3400050037008041eb00d2382e008340780077
:10ea440008007800e0fd070065390700e14f500039
:10ea540006003a008041eb0072392e0011c0b30069
:10ea640008007800d8fd07000d003700e24f500081
:10ea740006003a008041eb00523a2e0011c0b30068
:10ea840008007800d0fd0700050037008041eb0046
:10ea9400323b2e0011c0b30008007800cafd070005
:10eaa40050c2b300d33907000004e00001003a006b
:10eab40010c0b3000080fb00801f7800f03b2e00e4
:10eac400801f7800c100200074805700f3dd070028
:10ead4000040eb0080ff9f00804178007481570064
:10eae40021c0b30008007800b7fd0700e139070032
:10eaf400e4875700e14f500006003a0023c0b300fa
:10eb0400c23c2e0031c0b30008007800aefd0700ff
:10eb14000d003700e24f500006003a0023c0b30056
:10eb2400923d2e0031c0b30008007800a6fd070016
:10eb34000500370023c0b300523e2e0031c0b3009d
:10eb440008007800a0fd070013c0b30002202e00c7
:10eb540071c0b300080078009bfd07001800900006
:10eb6400013f2e00470f0700e84090001800900076
:10eb7400050f070070c0b300404498004f047800ac
:10eb84000080fa0000000600889fbe008a1f7800fb
:10eb94000004780082047800030578001104e00082
:10eba40002003a0000c2b300804878001904e00073
:10ebb40002003a0000c2b300804c78001a04e0005e
:10ebc40002003a0000c2b300004d78001800900023
:10ebd400f280200060417900e64f51000f003a00b6
:10ebe4000101780011c4b300560f0700180090000b
:10ebf4000901780021c4b300520f070018009000e7
:10ec04000a01780031c4b3004e0f070018009000c9
:10ec140031c6b300dc0e07000f0037000101780095
:10ec24008040eb00110f07001800900009017800e4
:10ec340011c0b3000d0f0700180090000a017800fe
:10ec440021c0b300090f070001c6b3006144980056
:10ec540018009000cc0e07004f0578004f04be004a
:10ec6400000006008001fa00889fbe00800478003e
:10ec74000f0078004018b1003f0009000018eb00b5
:10ec84008f0078004110b1003f0009008018eb00ac
:10ec94000f0078004008b1003f0009000018eb00a5
:10eca40019047800211b200088804000f20720000e
:10ecb400c0e72f000f004000e4d907002123200003
:10ecc40088804000f2072000c0ef2f000f004000b2
:10ecd400ded90700212b200088804000f2072000a5
:10ece400c0f72f000f004000d8d907003868930000
:10ecf4000004e0000d003a00cff894000104e000a5
:10ed040025003a0030402e00c1e72f0081804700e3
:10ed14000f000900b05878000001b1000002200083
:10ed2400e0bf9e00e03f9f001b0037004ff89400b7
:10ed34000004e00006003a0030412e00c1e72f0035
:10ed4400818047000d000900b0587800e000b10050
:10ed54004ff895000004e00006003a0010422e002f
:10ed6400c1ef2f00818047000e000900b0587800e1
:10ed7400f000b1004ff896000004e00006003a00ed
:10ed840000432e00c1f72f00818047000d000900c9
:10ed9400b0587800e000b100c3f72f008f81410024
:10eda400c2ef2f000f014100c1e72f008f80400008
:10edb4000900780074ff070020c0b300c044980025
:10edc4004f04be000080fa0000000600881f78008f
:10edd40000047800a800900000702000808060008b
:10ede400808f500049003a0008489000e14f4000ed
:10edf400460032000081fb00410620000191b90069
:10ee0400411f2000810f5100e08f59003d003a005e
:10ee140048409000e44f50001f00320008003e00bc
:10ee2400e14f5000130032002a003900e24f500035
:10ee340013003200e34f50002f003a001300370054
:10ee4400e84f50001d00320005003e00e64f500020
:10ee540014003200e74f500027003a001400370036
:10ee6400e94f500018003200e14f400022003a0000
:10ee74000300370008007800fdfd07001e0037007e
:10ee84000800780077ff07001b00370008007800af
:10ee940006fd0700180037000800780088fd070009
:10eea40015003700080078000cfe07001200370038
:10eeb40008007800cbfe07000f0037000800780038
:10eec40072fe07000c00370008007800a2fd07005e
:10eed40009003700e0c1b300c6380700e14f500015
:10eee40003003a00080078005eff070002003700c4
:10eef40008007800defd070000c0eb00004c98001d
:10ef0400020037000040e800004c98004f047800ed
:10ef1400000006001600fa00881f78001004900014
:10ef2400f080200068407800e34f500013003e005a
:10ef3400420120007880570044d9070078805700a8
:10ef44003cd90700f34f500007003e0002c2b30053
:10ef54008080fb00f881570082f178000040e800cf
:10ef6400f44f5000faff3a007881570061c0b300b3
:10ef740008007800550f070007003700b200200092
:10ef84007880570031d907007881570061c0b300f9
:10ef9400080078004d0f07004f0478000080fa0045
:10efa40000000600881f780000047800e1432e006a
:10efb40008007800d7ff0700a80090000060200038
:10efc40080806000808f500003003a001800900099
:10efd40021c6b300ec0d07004f04780000000600c2
:10efe400881f780000047800a800900000702000ba
:10eff40080806000808f50000c003a001800780078
:10f00400ed00400008007800c2ff070018009000df
:10f0140021c6b300dc0d070048409000e34f5000c8
:10f0240002003a0008007800a0fc07004f047800b2
:10f03400000006000600fa00881f7800000478002b
:10f0440000c2b3006b380700e14f500017003a00cc
:10f05400a80090000060200080806000808f500035
:10f0640012003a00980090008021b0000080400017
:10f074001080fb00801f780080442e00801f7800e1
:10f08400510020006c80570084dc070018009000b9
:10f094006c81570051c0b3000c0f0700180090009a
:10f0a40021c6b300b80d0700e48757004f04780069
:10f0b4000080fa0000000600881f78000004780031
:10f0c400a80090000070200080806000808f5000b5
:10f0d4000f003a00e1432e00080078008dff07007e
:10f0e40018009000c2442e0021c0b300f70e0700a0
:10f0f4001800900021c6b300a30d070048409000fb
:10f10400e34f500002003a000800780067fc070053
:10f114004f04780000000600c0489200e9cf500078
:10f1240002003e008040eb0031489a0010489000f5
:10f13400393f0700000006000600fa00881f780027
:10f1440000047800d0c1b3002a3807000004e000ae
:10f154000400320018007800306893000004e000d6
:10f1640004003a00f1442e0008007800aefb0700ca
:10f174000200370008007800e7ff070098007800d5
:10f18400616890000004e00004003200ed8040005b
:10f19400080078005fff070003003700e1432e00fa
:10f1a400080078005bff07001800780030689300bf
:10f1b4000004e00005003a0018009000c2442e004c
:10f1c40021c0b300c10e07000400370018009000ee
:10f1d40092452e0021c0b300bc0e070000c2b3004c
:10f1e40004380700e14f500011003a0098009000e5
:10f1f40080812000614078000004e0000c003200af
:10f204000080fb00801f780080442e00801f78005f
:10f21400510020006c80570020dc0700180090008b
:10f224006c81570051c0b300a80e0700e487570053
:10f2340018009000c2452e0011c0b300a30e0700b1
:10f244001800900021c6b3004f0d07004f0478004a
:10f254000080fa0000000600881f7800000478008f
:10f26400a80090000070200080806000808f500013
:10f2740010003a0078409000e14f40000d00320049
:10f284000081fb00210320000191b9003106200018
:10f29400828f50000500310008007800a6ff0700a7
:10f2a40000c0eb0070449800020037000040e80002
:10f2b400704498004f04780000000600889fbe0048
:10f2c4008a9fbe0080047800824578000345780058
:10f2d4006c844400e20f2000080078005bd807002b
:10f2e4000800780053d80700c04c9a000040eb0097
:10f2f400b04c9a00e14f550002003a0019489000c2
:10f30400c53e0700eb4c9a004f05be004f04be00fb
:10f3140000000600881f780000047800a800900010
:10f324000060200080806000808f500017003a0049
:10f3340018007800306893000004e0000a003a00e6
:10f3440013c0b3000041eb00f1442e000800780024
:10f35400daff070018009000c2442e0021c0b30059
:10f364005a0e070006003700080078006aff0700fd
:10f374001800900092452e0021c0b300530e0700e0
:10f384001800900021c6b300ff0c07004f0478005a
:10f39400000006000001fa00881f780000047800cd
:10f3a400a80090000070200080806000808f5000d2
:10f3b4001f003a00d0c1b3008e3707000004e000fc
:10f3c4001400320018007800212b2000811f400017
:10f3d40021232000811f4000211b2000811f4000a9
:10f3e40010462e00801f7800f10f200060ef2f00e0
:10f3f4000f004000a9db070013c0b3000041eb007d
:10f4040061ef2f008f80400008007800abff0700f9
:10f41400e887570048409000e24f50000200320055
:10f42400e14f400002003a00080078000dfe07009a
:10f434004f0478000080fa0000000600881f78005e
:10f4440000047800484090000040e900e34f400089
:10f454000b003e0098009000f0802000614078008e
:10f46400e34f500006003600a800900000002f0073
:10f474008080600000002100808f500008003a0066
:10f4840008489000e14f400007003a0038489000d7
:10f49400563e07000040eb00004c98000200370085
:10f4a4000800780036fb07004f04780000000600cf
:10f4b400889fbe0000047800280090000088a30004
:10f4c40031003200e48440001940e900e14f50006b
:10f4d4000c003e0048409000e24f500003003a0008
:10f4e40000c0eb0040449800020037000040eb00ed
:10f4f40040449800a8009000f09f2f000080600016
:10f504002004980019407800ec4f500016003a008f
:10f51400a800900001b8a30008003a001800900069
:10f52400b10f07002800900000b0a000200498004c
:10f5340019407800ec4f50000b003a00280190006d
:10f544000160200001016100810f510003003200bd
:10f554000120b100810f510005003a000800780035
:10f56400b6ff070008003700e84f500002003200e1
:10f57400e44f500004003a00a8009000006020000e
:10f5840001007000200498004f04be000000060033
:10f59400881f78000004780078409000e14f400014
:10f5a40004003a0028489000103e07000040eb0099
:10f5b400704498004f047800000006000000fa0030
:10f5c400889fbe008a9fbe008c1f78000f057800bc
:10f5d40000047800e484400040ccb300994f10004c
:10f5e40005003a0028019000f0ff200000006100af
:10f5f40000c0a00020049800658040008041eb001a
:10f6040002c3b300904f110012003a00e141900090
:10f614007041510082cf510007003200f141900047
:10f6240082cf5100040032000149900013c0b3009e
:10f63400e74f510007003a00a8019000f2ff2000b4
:10f6440082816100020026000301710022049800f7
:10f654008041eb00280190000288a300670032007b
:10f664000304e00065003a008f0578000f06780077
:10f6740091419000e5c251000581fb000281e80040
:10f68400e21fb200828747000041eb000504e0005e
:10f694000f003200e6804000e6c151008381fb0088
:10f6a4000383400004c2b300d040780084cf5000ec
:10f6b40002003c000204e000030032008281fb00ef
:10f6c40081f579000241e800860f5000f6ff3a0008
:10f6d4008240e90003c2b3000042eb00020037009d
:10f6e400847578008140e9000180fb006b4178005b
:10f6f400834f5100faff32000204e000f8ff3200a9
:10f704008582fb00858245000040eb00f0fa9f00f3
:10f714008b007800e0462e00d93107000004e00099
:10f72400050032008b00780060472e00d4310700ba
:10f734000004e00005003a00a8009000f09f2f00ac
:10f7440000806000200498002b00370040ccb300f8
:10f75400994f100006003a0018009000f180200034
:10f76400e0c07800e3cf500001003600120f07001c
:10f77400a8009000006020000080600005003a00ae
:10f78400a800900000602000010070002004980090
:10f79400070037008b007800c0472e00b8310700ff
:10f7a4000004e00002003a000800780023ff07008c
:10f7b400d0c1b3008f3607000004e000040032001b
:10f7c40018007800306893000004e00004003a0058
:10f7d400f1442e000800780013fa070002003700f5
:10f7e400080078004cfe07000800780068ff070056
:10f7f4000800780011ff07008c0778008a0778005a
:10f804004f0678004f05be004f04be000080fa008a
:10f81400000006003000fa00889fbe000004780053
:10f824000e007800133607008e1f780040482e0023
:10f83400801f7800c10020006900470097da0700a4
:10f844008041eb006901470083407800080078009c
:10f854005dfa0700ce35070080447800c335070001
:10f864008984fb00891f78000080fb00801f7800da
:10f87400b0482e00801f7800d10020007600470099
:10f8840086da07008041eb007601470011c0b3001f
:10f89400080078004cfa07004a360700801f7800f9
:10f8a40080492e00801f7800b10020004002200013
:10f8b4000e00400079da070023c0b30042022000a2
:10f8c4000e01410083407800080078003efa0700ea
:10f8d40013c0b30002202e0071c0b30008007800ea
:10f8e40039fa070018009000014a2e00e50b0700c2
:10f8f400e840900018009000a30b070050c0b3002c
:10f9040040449800ee8757004f04be000080fa0080
:10f91400000006000001fa00889fbe008004780001
:10f9240001447800e14f540040003a00d0c1b300d4
:10f93400303607000004e00007003a008041eb0085
:10f9440012232e0011c0b300090078001efa07002c
:10f9540011c0b30018003700e14f500007003a000f
:10f964008041eb0012242e008840780009007800c2
:10f9740015fa070021c0b3000f0037008041eb00e7
:10f9840012252e0088407800090078000efa07003e
:10f994008040eb00d0c1b300c8360700e9409000b6
:10f9a40019009000780b0700f1442e00090078003c
:10f9b4009df907006d003700d0c1b300bf360700c2
:10f9c40019007800a07093000104e0006700320081
:10f9d400b0689300e1cf500064003a00212b20006e
:10f9e400811f400021232000811f4000211b200093
:10f9f400811f400010462e00801f7800f10f200068
:10fa040040ef2f000f00400024da07008041eb0094
:10fa14000341780041ef2f008f80400009007800f7
:10fa240026fe0700e8875700500037000804e0006e
:10fa340016003a00e0c1b300ee3507000004e00010
:10fa440009003a0011c0b300e0c1b3009b360700bf
:10fa54008041eb0012222e008340780009007800d8
:10fa6400d9f90700430037008040eb00e0c1b30040
:10fa7400923607008041eb0062212e00834078001b
:10fa840009007800d0f907003a003700e24f54002b
:10fa940031003a0000c2b300d63507000004e0008c
:10faa4001d003a0011c0b30000c2b3008336070042
:10fab4009900900080812000008040001080fb00ad
:10fac400801f780080442e00801f780051002000a1
:10fad40080ef2f000f004000f0d9070019009000bc
:10fae40082ef2f000f01410051c0b300770c0700d3
:10faf4001900900021c6b300230b07008041eb00de
:10fb0400a2262e0021c0b30009007800aef9070038
:10fb1400e4875700170037008040eb0000c2b300b1
:10fb24006636070019009000124b2e0051c0b30036
:10fb3400660c07001900900021c6b300120b0700e1
:10fb44008041eb00f2252e0021c0b30009007800ab
:10fb54009df9070007003700e74f540005003a00fd
:10fb64000900780056fa070005003700e74f5400f3
:10fb740003003200e940900019009000020b0700d6
:10fb84004f04be000080fa00000006001000fa00d6
:10fb9400889fbe0000047800e1cf500046003a0080
:10fba40010c4b3009335070080c4e80000c6b30056
:10fbb40080cf54007f003e00894078007f40500091
:10fbc4003e36070000c3b30080cf54000e00360059
:10fbd4000980fb000003b100cf00de00008040007c
:10fbe4000080d1000080fb00801f7800602b2e0075
:10fbf400801f7800e100200078805700a7d9070013
:10fc0400e4875700220037000904e00008003a00a6
:10fc1400402c2e00801f7800e100200076805700e1
:10fc24009ed907008f87e9008044eb001800370055
:10fc340000c3b30080cf540007003a00202d2e00eb
:10fc4400801f7800e10020007680570093d90700d8
:10fc54008f87e9000e0037000980fb0001032000b4
:10fc640000805000cf00de00008040000080d10002
:10fc74000080fb00801f7800e02d2e00801f78009c
:10fc8400e10020007880570084d90700e4875700fa
:10fc94000040eb00a0ff9f00804178007481570072
:10fca40011c0b3000800780047f907000940780044
:10fcb400203d07003b003700e2cf50001c003a0013
:10fcc40020c4b3004b350700e14f50000c003a004c
:10fcd4008040eb0020c4b300f83507001800900002
:10fce40011cab300ba0907008041eb00922f2e001d
:10fcf40021c0b3000800780033f907002900370059
:10fd040011c0b30020c4b300ec3507001800900004
:10fd140001cab300ae0907008041eb00c22e2e00d9
:10fd240021c0b3000800780027f907001d00370040
:10fd34000104e00016003a0000c4b3002d350700aa
:10fd44000004e00009003a0011c0b30000c4b3008d
:10fd5400da3507008041eb00922a2e0083407800b8
:10fd64000800780018f907000e0037008040eb0007
:10fd740000c4b300d13507008041eb00b2292e0046
:10fd840083407800080078000ff907000500370069
:10fd9400e7cf500003003a0008007800c8f90700d4
:10fda40008003700e840900018009000760a070029
:10fdb400040037008040eb0010c4b300bf350700d7
:10fdc40093ff37004f04be000080fa0000000600d5
:10fdd4000e00fa00889fbe00800478000144780079
:10fde400e34f540016003a00223507008040e90032
:10fdf400e3cf400002003e00e24f500008003a000a
:10fe040010c0b300d83507008041eb00c23c2e007f
:10fe140031c0b30009007800ebf807006f00370029
:10fe240020c0b300d03507008041eb00923d2e0086
:10fe340031c0b30009007800e3f807006700370019
:10fe4400e24f54001e003a0050c2b300e9340700e8
:10fe54000004e00003003200e84f500004003a00c0
:10fe64000200370010c0b300010037000040eb006f
:10fe74000044e8008840780050c2b3008f35070082
:10fe84000884fb00881f7800f03b2e00801f780058
:10fe9400c10020007680570000d907000040eb0025
:10fea400e0f79f00804178007681570021c0b300bd
:10feb40009007800c4f80700e487570047003700ba
:10fec4000804e0001e003a003a3407008040e900cc
:10fed400e1cf50000800360010c0b300073507001a
:10fee4008041eb0032372e0083407800090078000f
:10fef400b5f8070039003700e14f500008003a0018
:10ff040020c0b300fd3407008041eb0002382e000e
:10ff14008340780009007800abf807002f00370011
:10ff24000040eb00f53407008041eb00d2382e008e
:10ff34008840780009007800a3f8070025003700fe
:10ff4400e14f54001e003a00253407008040e900c8
:10ff5400e1cf50000800360010c0b300f6340700ab
:10ff64008041eb0072392e0011c0b3000900780003
:10ff740095f8070019003700e14f500008003a00d7
:10ff840020c0b300ec3407008041eb00523a2e004d
:10ff940011c0b300090078008bf807000f00370088
:10ffa4000040eb00e43407008041eb00323b2e00bc
:10ffb400884078000900780083f8070005003700be
:10ffc400e74f540005003a00090078003cf90700a7
:10ffd40005003700e74f540003003200e940900069
:10ffe40019009000e80907004f04be000080fa00e1
:10fff400000006001000fa00889fbe008a1f7800e7
:020000040001f9
:10000400000478000104e00024003a0060c3b30057
:10001400783407000004e0000f003a0011c0b30078
:1000240060c3b300253507008041eb0052322e0037
:10003400834078000800780063f8070014c0b30018
:100044008041eb0004417800844078001800780077
:100054003d0e07000e0037000042eb00844178009b
:1000640012c0b3008240780018007800360e0700f2
:100074008041eb0062312e00834078000800780054
:1000840051f807008040eb0060c3b3000b35070054
:10009400180078003c0f070055003700e2cf5000ed
:1000a40026003a0080c3b300523407008044e800bd
:1000b400f5cf5400010036008044eb0089407800fd
:1000c40080c3b300fd34070090c3b3004934070074
:1000d40000457800b0c3b30046340700804178007f
:1000e4000a41780089407800180078009f100700c2
:1000f4008984fb00603e210060c07c000000fb009e
:10010400801f7800e0342e00801f7800f10020006a
:100114007a80570061d807000040eb00d0f79f00b9
:10012400804178007a81570021c0b300080078002c
:1001340025f80700e48757002d003700e1cf500071
:1001440026003a0080c3b3002a3407000045780033
:10015400b0c3b300273407008044780090c3b300d1
:10016400243407000004e0000e003a0089417800be
:1001740012c0b3008a407800180078007b10070092
:1001840011c0b30090c3b300cc3407008041eb002e
:1001940012342e0011c0b300080078000af80700da
:1001a40013003700894178000041eb008a40780051
:1001b400180078006d1007008040eb0090c3b30076
:1001c400be3407008041eb0032332e0011c0b3006f
:1001d40008007800fcf7070005003700e7cf50005f
:1001e40003003a0008007800b5f807000300370060
:1001f400e840900018009000630907004f0578005c
:100204004f04be000080fa00000006000200fa005d
:10021400889fbe0000047800e14090002800900010
:1002240003002f008301600002002600828f51002a
:1002340004003a00e9cf50009e00360002ccb3001f
:1002440082c04000e9cf50009a003e0002602000c6
:1002540002006000820f500096003a00484090006f
:10026400e14f50000f003a000104e00003003a009f
:10027400080078007bfa07008e003700e1cf5000b9
:1002840003003a000800780008f8070089003700e6
:10029400e2cf500087003a000800780088f8070091
:1002a40084003700e24f500003003a000800780051
:1002b400eff807007f003700e34f500045003a0095
:1002c4000104e00020003a00180078003060930038
:1002d400e14f500007003a008041eb00421e2e001f
:1002e4008340780008007800b7f707008044eb00eb
:1002f4000d0037008041eb00821d2e008340780002
:1003040008007800b0f707001800780060689000d3
:1003140019c0b3000004e000030032008000eb00c9
:1003240010c6b300bd3c0700e840900018009000e0
:100334001509070018007800a060930009417800af
:10034400af0f07005b003700e1cf500007003a0011
:1003540018007800190d070018007800a20c070097
:1003640008007800d1f7070052003700e7cf5000ab
:1003740003003a0008007800bdf807004d0037007c
:1003840081c4e900a9ff9f00180478008984fb0058
:10039400e002200000c8b9002003b00000004400bf
:1003a400880078000dd407000000e000410032000e
:1003b400e002200000c8b9002003b000000444009b
:1003c4003c003200e680570000c6b300933c0700af
:1003d40038003700e44f50001e003a000104e000ea
:1003e40003003a00080078000afd070031003700d6
:1003f400e1cf500003003a0008007800b7f8070086
:100404002c003700e3cf500003003a0008007800c6
:1004140074f9070027003700e2cf500003003a00c8
:100424000800780019f9070022003700e4cf5000d3
:1004340003003a000800780047f807001d00370061
:10044400e7cf50001b003a000800780088f8070046
:1004540018003700e54f500003003a000800780008
:1004640039f8070013003700e64f500003003a0044
:1004740008007800c5fd07000e003700e74f500064
:1004840003003a000800780051fe07000900370015
:10049400e84f500003003a0008007800d5fe07003a
:1004a40004003700e94f500002003a0008007800c9
:1004b40018fd07004f04be000080fa00000006008b
:1004c400881f78000004780041409000e24f5000fb
:1004d40009003a0051409000ec4f500006003a00e9
:1004e40060c3b30043330700e14f500002003a00f9
:1004f40018009000e90b07004f0478000000060084
:10050400881f78000004780041409000e14f5000bb
:1005140013003a0018007800b0689300e1cf50004f
:1005240001003a00680e07000040eb0040449800c8
:10053400a8009000f08f2f00008060002004980035
:100544008041eb0003417800f1442e00080078005c
:100554005afb070018009000af0b07004400370057
:10056400e34f50000800320018019000e1802000a1
:10057400e2c07800e9cf500021003a00a8009000c2
:100584000188a3001e003a008041eb00034178007b
:10059400f1442e000800780048fb070000c4b300b3
:1005a40014330700e14f500003003a0018007800ac
:1005b4002c0e07000800370018007800b06893007c
:1005c400e1cf500004003a00a80090000188a30085
:1005d40001003a003c0e070018009000820b07004f
:1005e400280090000080a0002004980008007800f3
:1005f400e7fb07000800780090fb07001c003700a9
:10060400e84f50001a003a00a80090000060200053
:100614000080600016003a00a800900000602000ee
:100624000100700020049800d0c1b300f13207002b
:100634000004e000040032001800780030689300e1
:100644000004e00004003a00f1442e0008007800a1
:1006540075f607000200370008007800aefa0700bc
:1006640008007800cafb07000800780073fb070045
:100674004f04780000000600889fbe008a1f78009f
:100684000004be00280090000088a300540032003b
:10069400648544001a407800f44f50000200320090
:1006a400f14f500007003a0018007800b06893003a
:1006b400e1cf500002003a00030e070001003700aa
:1006c400e80d070050c0b3009a4f10000d003a0027
:1006d400a8009000f06f200080806000d00fb1006f
:1006e400808f500007003a0098009000d020b0009e
:1006f40061407800e64f500021003a00080078007d
:10070400dbf7070000c3b3009a4f100016003a004d
:10071400280090000088a30013003200016020002c
:10072400010060000c003a00a80090000060200066
:10073400010070002004980048409000e14f400000
:10074400020032000040eb00404498001800900082
:10075400250b070004003700a8009000f09f2f002d
:10076400008060002004980030c2b3009a4f10004b
:1007740003003a00280090000080a10020049800a3
:10078400b940900070c4b30080cf500014003a0008
:1007940019409000e54f500011003a005940900074
:1007a40081c3b300814f500006003a00a8009000b6
:1007b400f09f2f000080600000a0a000200498009b
:1007c40007003700ef4f500005003a00a8009000e2
:1007d400f09f2f00008060000090a000200498008b
:1007e40060c3b30083320700e14f50001a003a009f
:1007f400c940900080c8b30080cf50000e003a007a
:100804001800780090689300e1cf500002003a008d
:100814007d0f070010003700e2cf500002003a00bd
:100824008b0f07000c003700e3cf50000a003a009a
:10083400750f07000800370018007800106993004e
:100844000204e00004003a0082c4b30082cf5000e6
:1008540001003a00fa0b07004f0578004f04be0070
:10086400000006000401fa00881f7800e80b21004c
:10087400000c780001868800640044000048eb0006
:100884009080fb0001b0a00001d0a0000108780016
:1008940011c6b3000080e8000148780000c0eb00f6
:1008a400e7004400804878008100e8008048780030
:1008b4000041eb00f1442e00a0ef2f000f00400098
:1008c4001c2d0700a00c2100a1ef2f008180470000
:1008d400020109003158780008017800217f2700bf
:1008e40020c0b300223b070008017800e1852700ff
:1008f40040c0b3001e3b070008017800c19c2700dc
:100904000040eb001a3b070008017800417d2700f6
:1009140050c0b300163b070008017800c1982700b7
:1009240010c0b300123b070008017800e13328002f
:1009340050c2b3000e3b07000801780021282800ac
:1009440020c2b3000a3b07000801780021262800d2
:10095400e0c3b300063b070008017800c18127000b
:10096400c0c3b300023b07000801780081102800cf
:1009740060c2b300fe3a07000801780021ff260098
:10098400c0c2b300fa3a07000801780001ae27009c
:1009940080c2b300f63a070008017800814d2700b1
:1009a40050c3b300f23a070008017800e1ff2600c3
:1009b40090c2b300ee3a070008017800a1a5270011
:1009c40070c2b300ea3a07002203200088007800ce
:1009d400e0922700d6380700ea00440080487800f7
:1009e4004206200088007800806e2700d038070077
:1009f400eb00440080487800421f20008800780003
:100a040040032700ca380700e90044008048780002
:100a14004f0478000080fa0000000600217f2700c0
:100a240020c0b300e23a0700e185270040c0b300cc
:100a3400df3a0700c19c27000040eb00dc3a0700c6
:100a4400417d270050c0b300d93a0700c198270060
:100a540010c0b300d63a0700e133280050c2b300f7
:100a6400d33a07002128280020c2b300d03a070057
:100a7400c1812700c0c3b300cd3a07002126280056
:100a8400e0c3b300ca3a07008110280060c2b30073
:100a9400c73a070021ff2600c0c2b300c43a0700ca
:100aa40001ae270080c2b300c13a0700814d270080
:100ab40050c3b300be3a0700e1ff260090c2b30062
:100ac400bb3a0700a1a5270070c2b300b83a0700db
:100ad400e0922700a5380700806e2700a33807009e
:100ae40040032700a1380700e00b2100870009001c
:100af4000018eb0000000600904190008040eb00dd
:100b0400e2cf4100070032000001e8008341e80021
:100b14008381fb0003014100b0c06800820f5000d4
:100b2400fdff3a000180fb000000e9004f00de00f9
:100b340000000600889fbe0001047800e30444001e
:100b440019417800e24f510004003a00880078000f
:100b540060c3b300b13a07009c003700a84090007e
:100b6400f8cf50001f003a00e14f510004003a0052
:100b740088007800d0c3b300a83a07009300370078
:100b840081c3b300814f510090003a00c8409000e7
:100b9400e1cf500004003a0022c0b300e1802000fd
:100ba40002f078000b003700e2cf500004003a0056
:100bb400c2c0b300e180200002f0780005003700d5
:100bc400e3cf500003003a0092c0b300e18020005c
:100bd40002f078008800780020c2b3008f3a070042
:100be4007a003700f0c3b30080cf50002e003a00e3
:100bf40018409000e84f50002b00360000cab300a4
:100c0400804f510048003a00d84a9000484a90006a
:100c1400f849900078419000e840900058409000d6
:100c24008582fb00ef9f6200c42ade00851f7800e6
:100c34000482fb00ef1f62004422de00841f780060
:100c44008381fb00ef9f6100c419de00831f7800dd
:100c5400884990008381fb00831f78000281fb0098
:100c6400ef1f61004411de00821f78008180fb00c9
:100c7400ef9f6000c408de00811f78000080fb0045
:100c8400ef1f60004400de00801f780048409000a1
:100c9400ef1f6000604d2e00801f78009038070021
:100ca400fe87570049003700a0c6b30080cf50002c
:100cb40007003a0060c3b300804f510043003a007c
:100cc400880078006b404000543a07003f0037002a
:100cd400b0c3b30080cf500013003a006b40400013
:100ce400804f510003003a00880078007f40500094
:100cf4004a3a070030c2b300994f100003003a008b
:100d04008800780065404000443a070070c3b3008f
:100d1400994f10002d003a00880078006b40500075
:100d24003e3a070029003700e1cf400013003a00a3
:100d3400b0c3b300804f510003003a00880078002c
:100d440078405000353a070030c2b300994f100084
:100d540003003a0088007800654040002f3a0700fd
:100d640060c3b300994f100018003a00880078005f
:100d74006b404000293a07001400370000ccb30050
:100d840080cf500011003a0030c2b300804f5100b0
:100d940008003a00c840900000ccb30080cf500057
:100da4000a003a0088007800d0c2b3001b3a07005a
:100db4000600370010c2b300804f510003003a0010
:100dc400880078006d404000143a07004f04be00cc
:100dd4000000060030419000e24f510004003a0048
:100de4008000780060c3b3000c3a07000e0037009f
:100df40091cbb30081404100e1cf500004003e009c
:100e04008000780050c2b300043a0700060037009f
:100e140021c3b300814f510003003a0080007800e1
:100e240030c4b300fd3907000000060031409000d3
:100e3400e24f500003003a0060c3b300f7390700e3
:100e4400170037002141900083c6b300834f51003f
:100e540006003a0012c3b300824f500010003a005b
:100e640030c3b300ed3907000d003700e14f4100f6
:100e740006003a0002c2b300824f500008003a0054
:100e840040c3b300e53907000500370022c3b300af
:100e9400824f500002003a0030c4b300df3907002b
:100ea40000000600889fbe0001047800e3044400ab
:100eb40019407800b1c3b300814f500006003200de
:100ec4002841900081ccb300814f510005003a00c5
:100ed400e14f500003003a0088007800b0c2b3002c
:100ee400ce39070020c3b300994f100002003a0026
:100ef40088007800c93907004f04be0000000600ce
:100f0400b0409000e2cf500003003a008000780027
:100f140060c3b300c13907000000060030419000ef
:100f2400a1c7b300814f510003003a00800078004c
:100f3400f0c3b300b9390700000006003041900047
:100f4400e14f510004003a0080007800d0c3b300a0
:100f5400b23907000600370021c3b300814f5100a6
:100f640003003a008000780020c4b300ab390700c6
:100f740000000600889fbe000004780017c0b3007c
:100f840076c6b30055c0b30074c0b30033c0b30019
:100f9400c2c0b3008740780008007800632e0700c1
:100fa40021c0b300e0802000017478006400400098
:100fb400000044008044eb00094878006f300700cb
:100fc400f180200000f47800aa300700018120009d
:100fd40000f47800493007001181200000f4780003
:100fe40030812000000044000948780000c0eb0074
:100ff400e380400000f478008100e80081004400b0
:10100400894878006181200000f478007081200014
:10101400000044000948780080812000000044005a
:101024000948780020512000000044000948780055
:1010340060802000000044000008eb0030107800bd
:1010440040802000000044000948780030802000df
:10105400000044000948780050802000000044004b
:10106400094878000d3707000001be00a180200068
:10107400810044008288be00080078004f04be004e
:10108400000006000000fa00889fbe008a1f780056
:101094000f04780084447800644542008a82fb008f
:1010a4008582e800e51fb200858747008803780041
:1010b400014c780084c0e800114498002244980050
:1010c4000400e0000a0032008002eb0032c0b300ea
:1010d4000283fb00e3c27a0085737b000241e800cf
:1010e400e34251008582fb00850f5200f8ff3e0069
:1010f4008041eb00e14f5500070032000701780002
:101104008180fb008100e80081804300b2c1690056
:10111400810f5100fdff3a008a80fb00818043006b
:10112400f3f89f000a04e000110032008700780001
:1011340052802000020140009281fb00f202200054
:101144000299b9001451200002014200020140003a
:101154000201e800e3c144008381fb008301e8004d
:101164008381400031697800838f5000fdff3a008d
:1011740051802000e0c07800efcf500004003a0016
:1011840051802000010040000048eb0003003700bc
:1011940052802000020040000148e80088077800df
:1011a4004f0578004f04be000080fa0000000600de
:1011b4000000fa00889fbe008a9fbe008c1f780042
:1011c40000067800814578008204780003457800a1
:1011d4000f0478000900780096d007008080fb0097
:1011e40064824000e6804000e11fb200818747002e
:1011f4008801780051cab300014c780031c6b300ad
:10120400114498002a4498003b4498000004e000ec
:1012140008003200e30044000901e8000040e9004e
:101224000080fb0000004100b9687800808f540002
:10123400fdff3a00b2c3b30081c6b3000c007800ce
:1012440090ff0700880778004f0678004f05be001e
:101254004f04be000080fa00000006000000fa00ff
:10126400889fbe008a9fbe008c1f7800800578008e
:101274000145780002047800834478000f06780062
:10128400080078006bd00700f74f500001003600cb
:1012940070c1b3008080fb0065824000e78040009d
:1012a400e11fb2008f0178008187470011c2b300ab
:1012b40081497800994198008040eb00a141980051
:1012c4000a44b000ba4198000004e000080032006b
:1012d400e38041000801e8000040e9000080fb00d1
:1012e40000004100b8687800800f5400fdff3a0008
:1012f4000480410061c0b30071f89f00b2c3b30021
:1013040081c6b3000b0078005eff07008c077800ed
:101314004f0678004f05be004f04be000080fa005f
:1013240000000600104890000000060020489000cd
:101334000000060080017800134290000040eb009a
:10134400e14f52000800320041c0b3006342420042
:101354000181fb0063417900024068008140e8009c
:10136400814f5200faff3a0000000600889fbe0039
:101374008004780009007800ecff0700004478003e
:1013840009007800e7ff0700804478000980fb002b
:10139400801f78000880fb00801f7800b0512e0069
:1013a400801f7800ce360700e6875700ef4f5400c1
:1013b40007003e0060532e00801f780030c0b30049
:1013c400153707008f87e90010c0b30047003700c6
:1013d400f04f540007003a00a0542e00801f7800fc
:1013e40030c0b3000c3707008f87e90020c0b3007a
:1013f4003e003700f14f540007003a00c0552e005c
:10140400801f780030c0b300033707008f87e900de
:1014140030c0b30035003700f24f540009003a00e1
:10142400f6cf54000a003a0000572e00801f7800bf
:1014340030c0b300f83607008f87e90040c0b3001e
:101444002a00370072405400e14f500009003e006a
:10145400f7cf540007003a0050582e00801f780040
:1014640030c0b300ec3607008f87e90050c0b300ea
:101474001e003700f44f540007003a00b0592e0004
:10148400801f780030c0b300e33607008f87e9007f
:1014940060c0b3001500370000ceb3000040440024
:1014a400ef4f500007003e00005b2e00801f7800c5
:1014b40030c0b300d83607008f87e90070c0b3008e
:1014c4000a0037000040eb0001c3b300814f540011
:1014d40006003a00205c2e00801f780030c0b30064
:1014e400cd3607008f87e90080c0b3004f04be00eb
:1014f400000006000200fa00889fbe008a9fbe001a
:1015040080057800010578003a409000e24f5000d1
:1015140004003a008a00780060c3b3003f38070033
:101524007a003700aa409000f2cbb30082cf50007b
:101534000e003a00b2c5b300824f500004003a00d6
:101544008a007800f0c2b300343807006f00370017
:10155400c2c5b300824f500054003a008a0078009c
:1015640000c3b3002d38070068003700f2c3b3008e
:1015740082cf50004d003a0002cab300824f50009f
:101584004a003a009a409000f9cf500004003a0013
:10159400408120006a5590008a7578005b0037000e
:1015a4001a41900031c2b300814f510038003a0013
:1015b40030812000ba489000817578000000e8006e
:1015c400ba509000817578000000e800ca5090007d
:1015d400817578000000e800ea5090008175780079
:1015e400660050006b407800e24f50004700320024
:1015f4007a5090000004e000440032000080fb00b8
:10160400cf80de00bbcd070002562e0003c52300a9
:1016140065ce07000004be000a5890000080fb005d
:10162400cf80de00b3cd070072712b001385230039
:101634005dce07000001be000800be0035cd0700e6
:1016440002ce0700c21728006328240056ce0700e4
:1016540002002000b33924002ecd07008acd0700f4
:1016640071812000ebc0780080cf50002700320049
:101674007181200080f5780010c0b300e0f79f006e
:10168400ea80570050c3b300e43707001f00370057
:101694009a409000e3cf50000e003a008a00780090
:1016a40000c4b300dd3707001800370042c5b3009b
:1016b400824f500004003a008a00780080c3b300cf
:1016c400d637070011003700f2c3b30082cf5000b1
:1016d4000e003a0001cab300814f50000b003a00db
:1016e4001a409000ef4f500008003a000a007800ba
:1016f4001eff0700e0f79f001181200080f57800ad
:10170400ea80570040c4b300c43707004f05be0049
:101714004f04be000080fa00000006000400fa0036
:101724008050900070489000c0ff9f00d1ff9f0040
:101734000040eb00e0ff9f0064805700ca290700c7
:101744000080fa00000006000400fa00c04890007f
:1017540030489000c0ff9f00d1ff9f000040eb0085
:10176400e0ff9f0064805700bf2907000080fa0053
:10177400000006000400fa00a060900010609000d1
:10178400c0ff9f00d1ff9f000040eb00e0ff9f00df
:1017940064805700b42907000080fa0000000600a6
:1017a400889fbe008004780009007800dbff0700f2
:1017b400e34f500006003e0028c0b300884f50009d
:1017c4001d003100e14f500006003a0007003700c9
:1017d400e44f50001100320058c0b300e64f5000ef
:1017e400150036000044eb001300370009007800b0
:1017f400e0ff070018c0b300050037000040e9000f
:1018040061c2b300814f50000100360068c0b300cc
:10181400084078004f04be0000000600090078006c
:10182400d4ff070048c0b30071c2b300814f500019
:10183400f7ff3e000500370009007800cdff0700e0
:10184400e54f5400edff3200f1ff370038c0b3001c
:10185400efff37000200fa00889fbe008a9fbe0097
:101864008c1f7800800478000104780038409000d0
:10187400e24f500004003a008800780060c3b300cf
:10188400663707007a0037009840900022c2b30000
:1018940082cf50004d003a0028419000f1c3b300bc
:1018a400814f510057003a0001cab300814f5000e4
:1018b40054003a0008007800a3ff07008045780030
:1018c40008007800abff07000045780008007800a6
:1018d40092ff07000046780008007800b0ff070078
:1018e400c0f79f000004e00033003200685090000d
:1018f4000080fb00801f7800585090000080fb009f
:10190400801f7800485090000080fb00801f780002
:10191400385090000080fb00801f78000a85fb008f
:101924008a1f78008b85fb008b1f78000c86fb00d8
:101934008c1f7800284890000080fb00801f7800ee
:10194400184890000080fb00801f78000848900031
:101954000080fb00801f7800784090000080fb002e
:10196400801f7800684090000080fb00801f780092
:10197400584090000080fb00801f78004840900091
:101984000080fb00801f7800605d2e00801f7800bf
:1019940053350700f0802000efd097008174780061
:1019a40061fd2f008f804000714040001b3707000d
:1019b400fe8757002e003700d0612e00801f78006c
:1019c400873507008f87e90029003700ecc05000f5
:1019d400f5cf50000b003e0028419000f1c3b30046
:1019e400814f510007003a0001cab300814f5000f3
:1019f40004003a0088007800a0c3b300073707004a
:101a04001b00370011c3b300814f500004003a009b
:101a14008800780060c2b300003707001400370064
:101a240051c4b300814f500004003a00880078008c
:101a340090c2b300f93607000d00370001c2b300ad
:101a4400814f500004003a0088007800e0c3b300de
:101a5400f23607000600370081c4b300814f5000fe
:101a640003003a008800780050c2b300eb36070048
:101a74004f0678004f05be004f04be000080fa00f8
:101a840000000600c04090008180fb00c408de0016
:101a940020c0b300efcf50000400320010c0b300e8
:101aa400eacf500001003a0020c0b3000000060055
:101ab4000200fa00889fbe008004780001047800c8
:101ac40038409000e24f500004003a00880078004b
:101ad40060c3b300d13607002e003700f14f500029
:101ae4000e003a0048409000a0ff9f000004e00070
:101af40003003a0021c0b300e08020008174780024
:101b0400e680570040c2b300c4360700208120009d
:101b1400aff89700817478001e003700f54f50002d
:101b240008003a0008007800d6ff07000181200071
:101b340080f478008800780070c3b300b7360700db
:101b440014003700f84f500004003a008800780071
:101b5400b0c3b300b13607000e003700f94f500090
:101b64000c003a005840900081812000e9c07800c0
:101b740080cf5000070032000004e000050035006b
:101b84008181200080f4780088007800c0c3b3000d
:101b9400a23607004f04be000080fa0000000600d1
:101ba4000c00fa00889fbe008a9fbe008c9fbe0076
:101bb400000478002f0798001800e00001013200ab
:101bc40029512000890444001945780088067800ca
:101bd40008007800233607000a81fb000201440054
:101be4002141200000f178000a45e8008a4c780081
:101bf400e14f5500e400360030412000000044006d
:101c040090c5e800f0c2b30080cf55003300360021
:101c14002234070032412000020144001281fb00fb
:101c2400821f78008b85fb008b1f78006011b80041
:101c3400809fbe00829fbe0040642e00801f7800fb
:101c440030c0b300bb340700ee875700205120009a
:101c5400684078000004e000110032008044eb008a
:101c64002a4120008b672e002c5120000c064400d2
:101c74000980fb000a004000684078000080fb00f7
:101c8400801f78008b1f780030c0b300a934070090
:101c94008944e800e48757009ccf1400f4ff3e0019
:101ca400e0672e00801f780030c0b300a134070025
:101cb40020512000000044000048eb002041200097
:101cc400800044007f0009008018eb000d007800bc
:101cd400043607008f87e900ab0037008b4f5500af
:101ce400a9003a008f0478003f0798008a86fb0019
:101cf4000d80e800e01fb200808747008904e800f7
:101d04000900a100e53307000d0f78008d1f78004e
:101d14006011b800809fbe00829fbe0010682e0034
:101d2400801f780030c0b30082340700ec8757006e
:101d34000a04e000110032001c4120000c0644009b
:101d440059079800090578005c407800005d780028
:101d54000080fb00801f780085672e00851f7800b7
:101d640030c0b30073340700ae4b900007405500f9
:101d7400e487570080cf5500f3ff3e003a5120001e
:101d84000a05440030802000000044009080fb00dd
:101d9400f00220000088b900000045000d01780021
:101da4008900780066cd07000000e00018003a00c2
:101db400e0692e00801f780030c0b3005d34070056
:101dc4003b8020008b0544009b80fb00f002200038
:101dd4000088b900000045000d0178008000eb0088
:101de40077cd07001b4078008f87e900ef4f500044
:101df40004003a0030802000000044000048eb005a
:101e04000300370031802000810044008048e8004e
:101e1400e0672e00801f780030c0b300453407000f
:101e2400090578000900780033fb07008f87e90073
:101e3400e14f50003f003a009945780080c6b30056
:101e440080cf550003003a000800be0039fb0700ac
:101e54000b003700f0cf450003003a00090078007a
:101e6400dcfb07000d00370000c8b30080cf55002d
:101e740003003a000800be000dff07000e00370003
:101e8400b0c3b30080cf550004003a008a00780044
:101e9400080078006ffe07000e00370000cdb30085
:101ea40080cf550004003a008a00780008007800ca
:101eb40090fd07000e00370000ccb30080cf550022
:101ec40004003a008a00780008007800d7fb070075
:101ed4000d00370000c5b30080cf550004003a0060
:101ee4008a00780008007800eefb07000a0037003b
:101ef400a0c6b30080cf550003003a000a00780062
:101f0400fffb0700040037000b04e00002003a0066
:101f14000a00780001fc0700a940900080ccb300bf
:101f240080cf500010003a000a00780003fc07003c
:101f34000d003700194090000080fb00801f7800de
:101f44009e1f7800294090000080fb00801f7800cd
:101f54001980fb00801f7800506a2e00801f7800d3
:101f64001f340700ea875700204120008006440000
:101f74007f000900801eeb000010b0000000440048
:101f84000048eb00be079000608020000000440081
:101f94001000be00e00f5000e08f580003003a002c
:101fa4008000eb0090c3b3009c3507003b3307006f
:101fb4000001be0061802000810044008288be00d0
:101fc400550037004080200000004400518020006c
:101fd400e8c0780090cf50004f0032002f33070044
:101fe4000045eb005c8020000c0644005c07980070
:101ff4004980200089044400ab8020008b05440004
:102004000081fb008001eb00028fbe003c00370022
:10201400223307003b015000ab815800e60f51000a
:10202400e08f5900360036009981fb00f20220004f
:102034000299b90034512000020142000201440017
:1020440012429000a006ab0023003a0004c2e8004c
:10205400170032000001eb0003412000830144001b
:10206400f602200025512000130078009980fb001f
:10207400068eb9003c0798004d0798008c0041007b
:102084008580400081004400914090008180fb00e5
:102094002100980093007800110090000098a3009c
:1020a400fdff3a000201e800824f5200eeff3e00bd
:1020b40019407800ef4f500002003a00804ceb00ca
:1020c40001003700804ce800f4320700808dbe0028
:1020d4002ac0b3000a003700e24f5500080032005e
:1020e4001e01be000200500083805800a30f200090
:1020f400830f5000e08f5800010036001ac0b3006f
:102104005e02900014427800994f5200020032009f
:10211400e14f5500beff3a0020512000684078008e
:102124000004e0003b003200dc3207000001be0086
:10213400618020008100440031065100a1865900cd
:102144000c00be006d0420008d0f5000e08f58007d
:1021540004003e002051200068407800e14f400018
:102164002c003a00cd320700295120008904440094
:102174001981fb00821f78006011b800809fbe00a7
:10218400829fbe00606d2e00801f780030c0b300b7
:1021940068330700ec8757001904e000110032008f
:1021a4008044eb002a4120008b672e002c51200034
:1021b4000c0644000980fb000a00400068407800d7
:1021c4000080fb00801f78008b1f780030c0b300b4
:1021d400583307008944e800e48757009ccf140073
:1021e400f4ff3e00e0672e00801f780030c0b3008b
:1021f4005033070020512000000044000048eb0049
:1022040020412000800044007f0009008018eb007a
:102214008f87e90008007800c92a0700ae079000fc
:102224004f06be004f05be004f04be000080fa00fa
:10223400000006000200fa0021c0b300e1ff9f0085
:1022440011c0b300f1ff9f00240020008f81e9003a
:1022540000c1eb0081c1b3008afb07000080fa00d3
:10226400000006000200fa0021c0b300e1ff9f0055
:102274008040eb00f1ff9f00240020008f81e900e3
:1022840082c6b30081c1b3007efb07000080fa0060
:10229400000006000c00fa0094c3b300c4f79f00ca
:1022a400d1f79f0001c8b30001414100e2f79f004c
:1022b4008040eb00f1f79f0083ff9f0091ff9f0098
:1022c40012c0b300a2ff9f00b2ff9f00c1ff9f0096
:1022d400d2ff9f00e2ff9f00f2ff9f00c400200096
:1022e400ec81570082c6b30081c1b30065fb0700cf
:1022f4000080fa00000006000400fa0084c0b30065
:10230400c4ff9f000042eb00d4ff9f00e2ff9f0048
:10231400f3ff9f0014002000e4815700014178007e
:10232400f1c3b30057fb07000080fa000000060069
:102334000200fa000041eb00e2ff9f0014002000bd
:102344008f81e90001417800f1c3b3004dfb070020
:102354000080fa00000006000200fa00b2c0b300d8
:10236400e2ff9f00140020008f81e9000141780002
:10237400f1c3b30043fb07000080fa00000006002d
:102384000200fa0012c1b300e2ff9f001400200013
:102394008f81e90001417800f1c3b30039fb0700e4
:1023a4000080fa00000006000200fa00f2c9b3003f
:1023b400e2ff9f00140020008f81e90001417800b2
:1023c400f1c3b3002ffb07000080fa0000000600f1
:1023d4000200fa0062c3b300e2ff9f00f1ff9f0016
:1023e400240020008f81e900a2c6b30081c6b30097
:1023f40024fb07000080fa00000006000200fa0037
:1024040013c0b300e3ff9f00140020008f81e90094
:102414001cfb07000080fa00000006000200fa001e
:1024240024c0b300e4ff9f00f3ff9f0024002000ba
:102434008f81e90013fb07000080fa00000006000a
:102444000400fa0001812000e0c07800e2cf5000cf
:102454000c003a00c1c0b300c1ff9f0031c0b300fb
:10246400d1ff9f0011c0b300e1ff9f0034002000a2
:10247400e48157000041eb00f1c3b30001fb070006
:102484000b003700e1cf500009003a00e480570008
:1024940092722e0003000900b25878004400200014
:1024a400e48157000041eb00f1c3b300f5fa0700e3
:1024b4000080fa00000006000400fa0001812000f8
:1024c400e0c07800e2cf50000c003a00c1c0b30075
:1024d400c1ff9f0051c4b300d1ff9f0011c0b300de
:1024e400e1ff9f0034002000e48157000041eb002d
:1024f400f1c3b300e3fa07000b003700e1cf50004b
:1025040009003a00e480570052722e0003000900cb
:10251400b258780044002000e48157000041eb00e9
:10252400f1c3b300d7fa07000080fa0000000600e8
:102534000400fa0001812000e0c07800e2cf5000de
:102544000c003a00c1c0b300c1ff9f0071c3b300c7
:10255400d1ff9f0011c0b300e1ff9f0034002000b1
:10256400e48157000041eb00f1c3b300c5fa070052
:102574000b003700e1cf500009003a00e480570017
:1025840012722e0003000900b258780044002000a3
:10259400e48157000041eb00f1c3b300b9fa07002e
:1025a4000080fa00000006000400fa000181200007
:1025b400e0c07800e2cf50000c003a00c1c0b30084
:1025c400c1ff9f0041c3b300d1ff9f0011c0b300fe
:1025d400e1ff9f0034002000e48157000041eb003c
:1025e400f1c3b300a7fa07000b003700e1cf500096
:1025f40009003a00e4805700d2712e00030009005c
:10260400b258780044002000e48157000041eb00f8
:10261400f1c3b3009bfa07000080fa000000060033
:102624000400fa0001812000e0c07800e2cf5000ed
:102634000c003a00c1c0b300c1ff9f0041c3b30006
:10264400d1ff9f0011c0b300e1ff9f0034002000c0
:10265400e48157000041eb00f1c3b30089fa07009d
:102664000b003700e1cf500009003a00e480570026
:1026740092712e0003000900b25878004400200033
:10268400e48157000041eb00f1c3b3007dfa070079
:102694000080fa00000006000400fa000181200016
:1026a400e0c07800e2cf50000c003a00c1c0b30093
:1026b400c1ff9f0051c4b300d1ff9f0011c0b300fc
:1026c400e1ff9f0034002000e48157000041eb004b
:1026d400f1c3b3006bfa07000b003700e1cf5000e1
:1026e40009003a00e480570052712e0003000900eb
:1026f400b258780044002000e48157000041eb0008
:10270400f1c3b3005ffa07000080fa00000006007e
:102714000400fa0001812000e0c07800e2cf5000fc
:102724000c003a00c1c0b300c1ff9f0041c3b30015
:10273400d1ff9f0011c0b300e1ff9f0034002000cf
:10274400e48157000041eb00f1c3b3004dfa0700e8
:102754000b003700e1cf500009003a00e480570035
:1027640012712e0003000900b258780044002000c2
:10277400e48157000041eb00f1c3b30041fa0700c4
:102784000080fa00000006000400fa0052cab300f8
:10279400c2ff9f00d1ff9f0011c0b300e1ff9f0063
:1027a4008040eb00f1ff9f0044002000e4815700cb
:1027b400b2c3b30081c6b30032fa07000080fa0046
:1027c400000006000000fa00889fbe008a1f7800ff
:1027d40080047800010478000f0578000800780070
:1027e40014cb0700eb4f500001003600b0c0b3001b
:1027f4008080fb0063824000e5804000e11fb2005e
:102804008f0178008187470031c2b3008149780085
:10281400fdc0400091419800f0c05000a1419800d3
:102824000004e000080032008380e8000801e800aa
:102834000040e9000080fb0000004100b868780017
:10284400800f5400fdff3a00b2c3b30081c6b30049
:10285400090078000bfa07008a0778004f05780012
:102864004f04be000080fa000000060003c6b30057
:102874007afa07000000060013c6b30077fa0700cf
:10288400000006000000fa00889fbe008a1f78003e
:1028940080047800010478000f05780008007800af
:1028a400e4ca0700f44f50000100360040c1b300f1
:1028b4008080fb0066824000e8804000e11fb20097
:1028c4008f0178008187470011c2b30081497800e5
:1028d40011c6b300914198008040eb00a1419800db
:1028e40091c0b300b14198000004e0000800320038
:1028f400e38041000801e8000040e9000080fb009b
:1029040000004100b8687800800f5400fdff3a00d1
:102914000480410061c0b30061f89f0071f89f001a
:10292400b2c3b30081c6b30009007800d5f907002b
:102934008a0778004f0578004f04be000080fa0033
:10294400000006000800fa00889fbe008a9fbe00af
:102954008c9fbe002007980021479800020478004d
:102964000f0f780008007800b2ca0700804678008c
:1029740080c2b30080cf5600010036008046780044
:102984000d04e000330032008045eb000b46780074
:102994003f0798008bc45600f4cf54000100360062
:1029a40049c1b3000981fb000201e8000280e8008c
:1029b400e03fb2000f057800808747008000eb00fd
:1029c4000a0078007eca07000904e0000e00320005
:1029d4008a0078008a01e8000940e9000080fb00d1
:1029e400808141000b4078003e0290000081fb0092
:1029f400e85879000040e800838f5000fbff3a005c
:102a04003407980089c545000c04e00006003a002c
:102a140013c0b3000a017800ae4090002e0090006d
:102a2400e3f90700050037008c4178000a017800bb
:102a3400ae4090002e009000ddf90700be07900024
:102a44008bcf5600030036008944e800094646004f
:102a5400cfff37009e0778004f06be004f05be002b
:102a64004f04be000080fa00000006000000fa00d7
:102a7400889fbe008a1f78008004780001047800d3
:102a84000f057800080078006aca0700e94f500073
:102a94000100360090c0b3008080fb0063824000d8
:102aa400e5804000e11fb2008f0178008187470074
:102ab40031c2b3008149780021c6b3009141980026
:102ac40001c3b300a14198000004e00008003200f3
:102ad4008380e8000801e8000040e9000080fb0072
:102ae40000004100b8687800800f5400fdff3a00f0
:102af400b2c3b30081c6b3000900780061f90700ce
:102b04008a0778004f0578004f04be000080fa0061
:102b1400000006000000fa00889fbe008a1f7800ab
:102b240080047800010478000f057800080078001c
:102b340040ca0700e94f50000100360090c0b300be
:102b44008080fb0064824000e6804000e11fb20008
:102b54008f0178008187470011c2b3008149780052
:102b640021c6b3009141980011c0b300a14198005f
:102b740001c4b300b14198000004e0000800320031
:102b8400e38041000801e8000040e9000080fb0008
:102b940000004100b8687800800f5400fdff3a003f
:102ba400b2c3b30081c6b3000900780035f9070049
:102bb4008a0778004f0578004f04be000080fa00b1
:102bc400000006000000fa00889fbe008a1f7800fb
:102bd40080047800010478000f057800080078006c
:102be40014ca0700eb4f500001003600b0c0b30018
:102bf4008080fb0068824000ea804000e11fb20050
:102c04008f0178008187470031c2b3008149780081
:102c1400fdc040009141980001c2b300a141980059
:102c24008040eb000004e000090032008380e800eb
:102c34008802e8000041e9000281fb0002814200b1
:102c4400b8687800820f5400fdff3a008040780095
:102c54000180fb000080410042c0b3003240980074
:102c64008140e8000181fb000281410000c2b30001
:102c7400304198008140e8000181fb00028141005d
:102c8400304198008140e8000181fb00028141004d
:102c9400304198008140e8008180fb008180410040
:102ca40000c1b300b0409800b2c3b30081c6b30002
:102cb40009007800f3f807008a0778004f057800c8
:102cc4004f04be000080fa00000006000000fa0075
:102cd400889fbe008a9fbe0000057800814478006a
:102ce400020478008f05780008007800d1c9070035
:102cf400eb4f500001003600b0c0b3008080fb00f1
:102d040064824000e6804000e11fb2008f01780039
:102d14008187470051cab3008149780021c6b300b6
:102d24009141980011c0b300a1419800b9419800a5
:102d34000004e00008003200e38041000801e800dc
:102d44000040e9000080fb0000004100b868780002
:102d5400800f5400fdff3a00b2c3b30081c6b30034
:102d64000a007800c7f807008b0778004f05be00fb
:102d74004f04be000080fa00000006000200fa00c2
:102d840001c1b300e1ff9f00140020008f81e9001e
:102d940002c8b30081c1b300baf807000080fa008a
:102da400000006000200fa0041c1b300e1ff9f00e9
:102db400140020008f81e90002c8b30081c6b3006b
:102dc400b0f807000080fa00000006000400fa00d2
:102dd40003c4b300c3ff9f0013c0b300d3ff9f001d
:102de400e1ff9f00f2ff9f0044002000e4815700b0
:102df40002c8b300b1c3b300a2f807000080fa0010
:102e0400000006000200fa00889fbe008a9fbe00f0
:102e14008c9fbe00000f7800010578000f06780033
:102e24000a00780083c90700e306400065004000fb
:102e34000000a100808747008c05780030c2b300f1
:102e4400004e78007f4040001046980070405000cb
:102e5400204698000044eb00050037000880fb0082
:102e640000804500eac47c00394098000844e8002a
:102e74008884fb000a0078006ec90700808f540024
:102e8400f6ff39000d0278008b01780002c8b30008
:102e940081ccb3001e0078007af807008c07780014
:102ea4004f06be004f05be004f04be000080fa006e
:102eb400000006008000eb00d2ff070000000600bf
:102ec4001000fa001281200060417900e14f5100a6
:102ed4001d003a0082cf50000400320022c0b3002b
:102ee40082cf50000100320000c1eb00418120007c
:102ef400e0c17800c1c0b30081f79f0092f79f0042
:102f04008040eb00a1f79f00b1f79f00c1f79f003d
:102f1400d1f79f00e1f79f00f1f79f0083ff9f0027
:102f240091ff9f00a1ff9f00b1ff9f00c1ff9f0081
:102f3400d4002000f081570002cdb300f1c3b300e8
:102f440050f807007000370082c1e900e1cf51005a
:102f540020003e0012c0b30082cf500004003200b3
:102f640022c0b30082cf50000100320000c1eb0048
:102f74004181200060c278008100e800e0c178004f
:102f8400c1c0b30081f79f008040eb0091f79f0020
:102f9400a2f79f00b1f79f00c1f79f00d1f79f00f0
:102fa400e1f79f00f1f79f0081ff9f0091ff9f00d1
:102fb400a4ff9f00b3ff9f00c1ff9f00d400200027
:102fc400f081570002cdb300f1c3b3002df8070020
:102fd4004d003700e4415100e2cf510020003e0093
:102fe40002c8b300e1cf50000400320002c4b300b1
:102ff400e2cf50000100320000c1eb00418120000b
:1030040060c278008100e800e0c17800c1c0b3006c
:1030140081f79f008040eb0091f79f00a1f79f008c
:10302400b2f79f00c1f79f00d1f79f00e1f79f001f
:10303400f1f79f0081ff9f0091ff9f00a4ff9f0075
:10304400b3ff9f00c1ff9f00d4002000f081570010
:1030540002cdb300f1c3b3000af807002a00370019
:1030640067415100e14f510027003e0002c5b30003
:10307400e1cf50000400320002c8b300e2cf500098
:103084000100320000c1eb003181200060c37800f0
:103094008100e800e0c278008100e80060c27800a6
:1030a4008100e800e0c17800c1c0b30081f79f004f
:1030b4008040eb0091f79f00a1f79f0080c3eb00d5
:1030c400b7f79f00c2f79f00d1f79f00e1f79f0079
:1030d400f1f79f0086ff9f0091ff9f00a5ff9f00cf
:1030e400b4ff9f00c3ff9f00d1ff9f00e1ff9f003b
:1030f400f1ff9f0004012000f081570002cdb300ce
:10310400f1c3b300dff707000080fa0000000600f7
:103114000200fa0031c5b300e1ff9f001400200053
:103124008f81e90002cdb30001c8b300d5f70700d1
:103134000080fa00000006000000fa00889fbe002c
:103144008a9fbe008c1f78000006780081047800f6
:103154000f05780009007800b6c80700e4054000b0
:10316400660040000000a100808747000a04780040
:1031740030c2b300004d780000ccb3001045980075
:1031840000c2b3002045980009007800a9c80700d0
:10319400eb4f50000400360070c1b3000881e80012
:1031a4008040eb00040037008040eb000004e000a6
:1031b400faff3a0004003700396978008140e800da
:1031c40080cf5000fcff39008180fb008100440067
:1031d40000c1b300b04098000b0278008801780069
:1031e40002ccb30081c6b3000c007800a5f7070039
:1031f4008a0778004f0678004f05be004f04be00d2
:103204000080fa00000006000000fa00889fbe005b
:103214008a1f780080047800010478000f05780084
:103224000800780083c80700f74f500001003600fb
:1032340070c1b3008080fb0064824000e6804000df
:10324400e11fb2008f0178008187470031c2b300cb
:1032540081497800fdc040009141980001c2b3004b
:10326400a14198008040eb000004e0000900320016
:103274008380e8008802e8000041e9000281fb0045
:1032840002814200b8687800820f5400fdff3a00c2
:10329400804078008180fb008180410000c1b30040
:1032a400b040980002ccb30001c8b3000900780014
:1032b40074f707008a0778004f0578004f04be00b2
:1032c4000080fa00000006000000fa00889fbe009b
:1032d4008a9fbe00000578008144780002047800cb
:1032e4008f0578000800780052c80700e44f5000aa
:1032f4000100360040c0b3008080fb0064824000bf
:10330400e6804000e11fb2008f017800818747000a
:1033140011c2b3008149780031ccb30091419800c7
:103324008040eb00a14198000944b000b9419800e5
:103334000004e00008003200e38041000801e800d6
:103344000040e9000080fb0000004100b8687800fc
:10335400800f5400fdff3a0002ccb30081c6b300d5
:103364000a00780047f707008b0778004f05be0076
:103374004f04be000080fa00000006000400fa00ba
:1033840012c2b300c2ff9f0002ccb300d2ff9f0061
:103394000041eb00e2ff9f00f1ff9f00440020008a
:1033a400e4815700b2c3b30081c6b30035f7070008
:1033b4000080fa00000006000200fa0061c4b300b5
:1033c400e1ff9f00a1c0b300f1ff9f002400200093
:1033d4008f81e900b2c3b30081c6b30029f70700a7
:1033e4000080fa00000006000200fa0051c4b30095
:1033f400e1ff9f0021c0b300f1ff9f0024002000e3
:103404008f81e90082c6b300b1c3b3001df7070082
:103414000080fa00000006000200fa0051c4b30064
:10342400e1ff9f008040eb00f1ff9f00240020009b
:103434008f81e90082c6b300b1c3b30011f707005e
:103444000080fa00000006000200fa0051c4b30034
:10345400e1ff9f0011c9b300f1ff9f002400200089
:103464008f81e90082c6b300b1c3b30005f707003a
:103474000080fa00000006000200fa0024c3b30032
:10348400e4ff9f00f3ff9f00240020008f81e900e8
:10349400fcf607000080fa00000006000400fa00b1
:1034a400e4805700d2702e0003000900b25878005f
:1034b40044002000e4815700b2c3b30081ccb300c0
:1034c400f0f607000080fa00000006000200fa008f
:1034d400b2c2b300e2ff9f00f1ff9f00240020006e
:1034e4008f81e90072ceb30081ccb300e5f607000a
:1034f4000080fa00000006000200fa00c2c2b30015
:10350400e2ff9f00f1ff9f00240020008f81e9006b
:1035140072ceb30081ccb300daf607000080fa0063
:10352400000006000200fa0012c1b300e2ff9f008f
:10353400f1ff9f00240020008f81e900f2cbb3004b
:1035440001c8b300cff607000080fa0000000600af
:103554000600fa00e680570082702e00040009007d
:10356400b258780054002000e6815700f2cbb30033
:1035740001cdb300c3f607000080fa000000060086
:103584000600fa00e680570032702e00040009009d
:10359400b258780054002000e6815700f2cbb30003
:1035a40001cdb300b7f607000080fa000000060062
:1035b40080007800211bb0003f0009008018eb0058
:1035c40021232000808040003f0009008018eb0088
:1035d4000108b100202bb0003f0009000018eb00e7
:1035e4000008b10000000600c06093000104e00080
:1035f4000e0032008040eb00e40220000181fb0059
:103604000491b9002203b00002014000030032001b
:103614002d0009000059eb00e202b1008140e800ee
:1036240040619300814f5100f4ff3e008000780018
:10363400511ab000030009008058eb008040eb00f1
:1036440041609b000000060080007800511ab00021
:10365400030009008058eb00000006000200fa0095
:1036640010407800e0ff9f000040eb00f0ff9f0057
:103674000f80e900fc2107000080fa00000006002a
:10368400889fbe008a9fbe008c1f780000067800c9
:10369400010578008a1f780020712d00801f7800b2
:1036a40020c0b3003d2e0700e48757008044eb00a0
:1036b400cb5320008b05460004003700ea407c0011
:1036c4000b0078004f2f07008944e8000984fb00b1
:1036d4000a00780057c70700800f5400f7ff39002d
:1036e400c053200000004600d1c0b300452f07009e
:1036f40020742000000646001c80fb0011002000fe
:10370400042a07004f0678004f05be004f04be0090
:10371400000006000600fa007225250093442500e7
:10372400d2bf9f00e3bf9f0051042000f1bf9f0060
:10373400e6805700d2ff07000080fa000000060070
:103744001000fa00881f780000047800821f7800b7
:103754008180fb00811f780080722d00801f78001b
:10376400f100200078805700ccca0700f880570089
:1037740008007800c2ff0700e68757004f0478006e
:103784000080fa00000006000800fa0062552400d8
:1037940023352500c2bf9f00d3bf9f0092f42400ad
:1037a400e3042000e2bf9f00f3bf9f00e8805700be
:1037b400b3ff07000080fa0000000600ea87470014
:1037c4008e1f78006a87570052e5240003152400f1
:1037d400029fbe0091242500010f780064875700e2
:1037e400004feb00ea805700a5ff07004f07780061
:1037f400af00b100000006008000fa00881f7800c6
:1038040000047800811f780050732d00801f780019
:1038140001082000a0f72f000f0040009fca0700f6
:10382400a1f72f008f8040000800780094ff070064
:10383400e48757004f0478000080fa000000060077
:103844001000fa00881f78000004780018709000b7
:103854000004e0000c0032000080fb00801f7800b0
:10386400d0732d00801f780001012000768057005e
:103874008aca0700f68057000800780080ff070016
:10388400e487570004003700a0742d00801f7800df
:10389400f22d07008f87e9004f0478000080fa00ba
:1038a40000000600ea8747008e1f78006a875700e9
:1038b4003245250013442500029fbe0051352500e2
:1038c400010f780064875700004feb00ea8057002f
:1038d4006bff07004f077800af00b100000006003f
:1038e4001e00fa00881f7800000478000482fb00a0
:1038f400841f7800811f78000200be006011b800a8
:10390400809fbe00829fbe0060772d00801f7800dc
:10391400d101200020fd2f000f0040005fca0700e6
:1039240021fd2f008f8040000800780054ff07001d
:103934000800780077ff0700ee8757004f047800ef
:103944000080fa00000006002600fa00881f7800b4
:10395400000478008381fb00831f78000281fb0050
:10396400821f78008180fb00811f78000482fb00a5
:10397400841f780010792d00801f780051022000e8
:10398400e0fc2f000f00400044ca0700e1fc2f00b8
:103994008f8040000800780039ff07000800780095
:1039a4005cff0700ea8757004f0478000080fa00a4
:1039b400000006000e00fa00881f7800000478005a
:1039c400811f7800a07b2d00801f7800d10020008b
:1039d4007480570031ca0700f4805700080078004b
:1039e40027ff0700080078004aff0700e487570014
:1039f4004f0478000080fa00000006004a00fa0034
:103a0400889fbe008a1f7800800478000105780032
:103a14008a1f7800507c2d00801f7800a1022000ae
:103a2400c0fa2f000f0040001cca0700c1fa2f0083
:103a34008f8040000900780011ff0700738457004d
:103a4400820020008a007800080078007fc6070002
:103a5400881f7800107d2d00801f780071012000e0
:103a640020fd2f000f0040000cca070021fd2f008d
:103a74008f8040000900780001ff070009007800ea
:103a840024ff0700e88757004f0578004f04be0065
:103a94000080fa00000006001800fa00881f780071
:103aa400000478000104e00009003a00307e2d0093
:103ab400fa80570017000900b05878008001b1005f
:103ac400fa80570008007800edfe07000a0037006e
:103ad400e1cf500008003a00b07f2d00fa80570073
:103ae40016000900b05878007001b100fa80570040
:103af40008007800e2fe07000800780005ff0700d0
:103b04004f0478000080fa00000006001200fa005a
:103b1400881f780000047800821f78008180fb00f1
:103b2400811f780020812d00801f78001101200062
:103b34007a805700d9c90700fa8057000800780036
:103b4400cffe070008007800f2fe0700e687570062
:103b54004f0478000080fa00000006001e00fa00fe
:103b6400881f7800000478000482fb00841f78001a
:103b74008381fb00831f78000281fb00821f780091
:103b84008180fb00811f780020822d00801f780037
:103b9400e101200060fd2f000f004000bfc90700b5
:103ba40061fd2f008f80400008007800b4fe0700fc
:103bb40008007800d7fe0700ea8757004f04780012
:103bc4000080fa00000006001800fa00881f780040
:103bd400000478000281fb00821f78008180fb00d2
:103be400811f780000842d00801f7800810120004f
:103bf40000fe2f000f004000a8c9070001fe2f009f
:103c04008f804000080078009dfe070008007800bf
:103c1400c0fe0700e68757004f0478000080fa00d2
:103c2400000006001000fa00881f780000047800e5
:103c34008180fb00811f7800a0852d00801f780003
:103c4400f10020007680570094c90700f6805700e1
:103c5400080078008afe070008007800adfe07001f
:103c6400e48757004f0478000080fa000000060043
:103c74002800fa00881f780000047800841f780068
:103c8400831f7800821f7800811f7800a0862d0092
:103c9400801f780081022000c0fc2f000f0040002c
:103ca4007ec90700c1fc2f008f8040000800780007
:103cb40073fe07000800780096fe0700ea875700a5
:103cc4004f0478000080fa00000006001e00fa008d
:103cd400881f780000047800841f78008381fb002b
:103ce400831f78000281fb00821f78008180fb0023
:103cf400811f7800c0882d00801f7800d10120002a
:103d040060fd2f000f00400064c9070061fd2f0013
:103d14008f8040000800780059fe070008007800f2
:103d24007cfe0700ea8757004f0478000080fa0001
:103d3400000006000e00fa00881f780000047800d6
:103d44000281fb00821f78008180fb00811f7800c4
:103d5400908a2d00801f7800e100200076805700b3
:103d64004ec90700f68057000800780044fe07009b
:103d74000800780067fe0700e68757004f047800c4
:103d84000080fa00000006000600fa002255240014
:103d940033552400d2bf9f00e3bf9f00410520009c
:103da400f1bf9f00e680570035fe07000080fa004f
:103db400000006001800fa00889fbe008a1f7800e1
:103dc400000578008104780002047800c200200015
:103dd400890078000a0078009cc50700881f7800d5
:103de400891f7800908b2d00801f780081012000ae
:103df400c0fd2f000f00400028c90700c1fd2f009f
:103e04008f8040000a0078001dfe0700e6875700f7
:103e14004f0578004f04be000080fa000000060041
:103e24000a00fa00881f7800000478008180fb00f3
:103e3400811f7800408c2d00801f7800a100200095
:103e44007080570015c90700f080570008007800fb
:103e54000bfe0700e48757004f0478000080fa0047
:103e6400000006001000fa00881f780000047800a3
:103e7400786890000004e0000c0032000080fb0031
:103e8400801f7800d08c2d00801f7800f100200066
:103e94007680570001c90700f680570008007800b3
:103ea400f7fd0700e487570004003700b08d2d00ac
:103eb400801f7800692c07008f87e9004f04780081
:103ec4000080fa00000006001000fa00881f780045
:103ed40000047800786890000004e0000c003200d0
:103ee4000080fb00801f780040902d00801f780028
:103ef4000101200076805700e8c80700f6805700cb
:103f040008007800defd0700e4875700040037004e
:103f140030912d00801f7800502c07008f87e90016
:103f24004f0478000080fa00000006000600fa0042
:103f3400881f780000047800d0932d00801f78003b
:103f4400510020006a805700d4c80700ea80570057
:103f540008007800cafd07008f87e9004f04780045
:103f64000080fa00000006002800fa00881f78008c
:103f7400000478000100e0000e003a000200e000b6
:103f840028003a0020942d00801f78008100200032
:103f940040fd2f000f004000c0c8070041fd2f0066
:103fa4008f80400008007800b5fd07008f87e90086
:103fb4001c0037000200e0000d003a00811f780069
:103fc400a0942d00801f7800d100200020fd2f0038
:103fd4000f004000b1c8070021fd2f008f80400072
:103fe40008007800a6fd0700e48757000d0037009d
:103ff400821f7800811f780050952d00801f780063
:104004007102200000fd2f000f004000a3c807002c
:1040140001fd2f008f8040000800780098fd070004
:10402400e68757004f0478000080fa00000006007d
:104034001400fa00881f7800000478007868900063
:104044000004e0000c0032000080fb00801f7800b8
:1040540030962d00801f7800310120007a805700af
:104064008ec80700fa8057000800780084fd070016
:10407400e48757000400370060972d00801f780004
:10408400f62b07008f87e9004f0478000080fa00c0
:10409400000006001200fa00881f7800000478006f
:1040a400811f7800709a2d00801f78002101200064
:1040b4007880570079c80700f88057000800780016
:1040c4006ffd0700e48757004f0478000080fa0072
:1040d400000006001400fa00881f7800000478002d
:1040e400786890000004e0000c0032000080fb00bf
:1040f400801f7800f09a2d00801f78004101200075
:104104007a80570065c80700fa80570008007800d5
:104114005bfd0700e487570004003700309c2d0046
:10412400801f7800cd2b07008f87e9004f047800ab
:104134000080fa00000006001200fa00881f7800d0
:1041440000047800786890000004e0000c0032005d
:104154000080fb00801f7800409f2d00801f7800a6
:1041640021012000788057004cc80700f8805700d0
:104174000800780042fd0700e48757000400370078
:10418400309c2d00801f7800b42b07008f87e90036
:104194004f0478000080fa00000006001200fa00c4
:1041a400881f780000047800786890000004e0001c
:1041b4000c0032000080fb00801f780060a02d00fe
:1041c400801f7800110120007880570033c8070051
:1041d400f88057000800780029fd0700e48757009d
:1041e4000400370070a12d00801f78009b2b07006e
:1041f4008f87e9004f0478000080fa000000060071
:104204001a00fa00881f78000004780021649b00db
:1042140032649b00e1cf500004003a00f0e4240033
:1042240001002000008fbe00050037000104e000fb
:1042340003003a00f064240061042000008fbe00f3
:10424400e14f510005003a00f0e424000100200091
:104254002007980031079800060037000204e000a8
:1042640004003a00f0642400610420002007980050
:1042740031079800e41f47008e1f780030a42d00fa
:10428400801f7800110120006800470003c8070060
:10429400e800470008007800f9fc0700e6875700ab
:1042a4004f0478000080fa00000006000001fa00c4
:1042b400881f780000047800811f780020a52d0055
:1042c400801f7800f10f2000a0ef2f000f004000a6
:1042d400f2c70700a1ef2f008f804000080078008c
:1042e400e7fc0700e48757004f0478000080fa00d9
:1042f400000006001000fa00881f7800000478000f
:104304000304e00008003a00811f780050a52d0046
:10431400801f78000101200076805700dfc7070066
:10432400e48757000b0037008381fb00831f78006c
:104334000281fb00821f7800811f780000a62d00f7
:10434400801f7800010120007a805700d3c707003e
:10435400e8875700f280570008007800c8fc07007f
:104364004f0478000080fa00000006004600fa00be
:10437400889fbe008a9fbe008c1f7800800478004e
:10438400814578000246780008ccb30008c4450093
:10439400e1cf510032003200e3c0b3000041eb0032
:1043a40011a72d0009007800d2ff07000885fb0043
:1043b4008a1f78000004eb00881f78008a1f7800a9
:1043c400881f7800881f780040a72d00801f780080
:1043d4006104200040fa2f000f004000afc707001f
:1043e40041fa2f008f80400009007800afff0700da
:1043f400e3c0b3000041eb0041ac2d00090078009c
:10440400bcff07008a1f7800881f78008a1f780085
:10441400881f7800881f780070ac2d00801f7800fa
:104424006104200080f92f000f0040009bc70700a3
:1044340081f92f008f804000090078009bff07005e
:104444008b40e80074b12d008c417800f2c0b300b9
:10445400090078001dfe0700f88757003100370077
:10446400e3c0b3000041eb0011a72d000900780060
:10447400a0ff07000885fb008a1f780008082000b9
:10448400881f78008a1f7800881f7800881f7800aa
:1044940040a72d00801f78006104200040fa2f00ff
:1044a4000f0040007dc7070041fa2f008f804000b5
:1044b400090078007dff0700e3c0b3000041eb0072
:1044c40041ac2d00090078008aff07008a1f78009c
:1044d400881f78008a1f7800881f7800881f78005a
:1044e40070ac2d00801f78006104200080f92f003b
:1044f4000f00400069c7070081f92f008f8040003a
:104504000900780069ff07008b40e800b4b12d0072
:104514008c417800f2c0b30009007800ebfd07007d
:10452400f88757004f0678004f05be004f04be00c1
:104534000080fa0000000600ec874700881f78001e
:104544008e1f780000047800e1cf40000d003a008f
:104554006e87570030c42400f1342500009fbe004c
:104564005004220011c42400009fbe00c004200097
:10457400000f7800ee8057000800780040fc070028
:104584000b0037008180fb00811f7800408c2d00d8
:10459400801f780091002000728057003fc70700f9
:1045a400f28057000800780035fc0700e4875700c4
:1045b4004f0778004f047800cf00b10000000600d8
:1045c4001000fa00881f780000047800187090002a
:1045d4000080fb00801f7800e0b12d00801f780070
:1045e400f1002000768057002cc70700f6805700a2
:1045f4000800780022fc0700e48757004f04780085
:104604000080fa00000006000c00fa00881f780001
:1046140000047800187090000080fb00801f780070
:10462400d0b22d00801f7800c10020007280570096
:104634001ac70700f28057000800780010fc070032
:10464400e48757004f0478000080fa000000060059
:104654001000fa00881f7800000478001870900099
:104664000080fb00801f780090b32d00801f78002d
:10467400f10020007680570008c70700f680570035
:1046840008007800fefb0700e48757004f04780019
:104694000080fa00000006001600fa00881f780067
:1046a40000047800786890000080fb00801f780088
:1046b40080b42d00801f7800510120007c805700b9
:1046c400f6c60700fc80570008007800ecfb0700e2
:1046d400e48757004f0478000080fa0000000600c9
:1046e4001400fa00881f78000004780078689000ad
:1046f4000080fb00801f7800d0b52d00801f78005b
:10470400310120007a805700e4c60700fa80570080
:1047140008007800dafb0700e48757004f047800ac
:104724000080fa00000006001200fa00881f7800da
:1047340000047800786890000080fb00801f7800f7
:1047440000b72d00801f78002101200078805700d9
:10475400d2c60700f880570008007800c8fb07009d
:10476400e48757004f0478000080fa000000060038
:10477400881f780000047800c05320000000440023
:10478400d1c0b3001f2b0700207420000004440094
:104794001880fb0011002000de2507004f0478007c
:1047a400000006002f03b000889fbe008a9fbe0051
:1047b4008c9fbe008e1f78000005be0082bf9f0044
:1047c400ca6493000904e000120032000004eb0004
:1047d4008046eb00ec0220001ec0b3000cc0b90000
:1047e4002103200080804000810045000b007800f8
:1047f400fac207000000e00001003a008e4678008b
:104804000804e80088cf5400f4ff3e000d04e000e3
:104814001a003a00d20020008b00780020fc2f0000
:104824000f00400009c307000f0078001003b10017
:10483400200009000058eb00020220008fb8970006
:10484400f0fc2f000f00400000c307008980fb002c
:10485400e00220000088b900000045002103200088
:104864008100400022fc2f0002814700160009004d
:10487400b21878008944e80049659b004f07780026
:104884004f06be004f05be004f04be002f03b1000b
:1048940000000600889fbe008a9fbe008c9fbe0059
:1048a40080047800c96693000040eb00c0649b005c
:1048b4000d04e0001e0032000004eb00eb022000b7
:1048c4000bc0b9002a032000000545000a854400f6
:1048d400140032002c032000000646000c8644001d
:1048e400890078000c007800bcc207000000e000da
:1048f40009003a000804e0000a0032000bc1b900c4
:1049040002814400f203b0008c00780009007800b2
:10491400a4ff0700030037002d000900005deb0031
:10492400ea02b1000804e80088cf5600e4ff3e0024
:1049340009007800501ab000030009000058eb0089
:104944004f06be004f05be004f04be000000060027
:10495400889fbe008a9fbe008c9fbe008e1f780079
:104964000005780001067800ca6693000044eb0055
:104974000007eb00eb0220008884fb000bc8b900a1
:104984002103200080804000810045000c00780055
:1049940092c207000000e00003003a000bc8b9000f
:1049a40000074500fe03b0000844e8008d4f5400a2
:1049b400f1ff36000e0078004f0778004f06be0066
:1049c4004f05be004f04be00000006003200fa008e
:1049d4008f0078002103b100050009008018eb0066
:1049e4008058eb008f0078005102b10020000900cc
:1049f4008058eb008040eb00c1ff9f00e1ff9f0067
:104a0400d1ff9f00f1ff9f00e1fc2f008180470050
:104a140031000900315878002003b1000080fa0009
:104a2400000006003200fa00881f780000047800b5
:104a3400c0fc2f000f004000e4ff0700c0fc2f0063
:104a44000080470031000900305c78002803b10081
:104a54004f0478000080fa00000006008c0bfa0076
:104a6400889fbe008004780080bb2f00008447002c
:104a740008007800d5ff070001472f000181470097
:104a840031000900385978002803b10011c0b3007f
:104a940023612f0081f7790032612f00817779003b
:104aa4000040eb0066014100807779000142780004
:104ab4000201e8008477790041612f0080f77800d3
:104ac40000417800b4612f0082777a0041c0b300be
:104ad400c3612f0081f779006011b80063024200be
:104ae4000f024200021a78000312780051612f006d
:104af40001814700030009000059eb0000472f0023
:104b04000f004000aafa0700a3be2f000384470049
:104b14008043eb0026c2b30055c0b30064c0b300a9
:104b2400a3c1b30052c1b30021c0b3000800780090
:104b34007e1f0700647a2f00048047002141200073
:104b440008020900381878000100500001045400dc
:104b540002472f0082814700443a8000a3030900e2
:104b6400b31c780084845400090078004f04be000c
:104b74000080fa0000000600889fbe000004be000a
:104b840021b82d000900780014c207000000e000dd
:104b940002003a00007498001100370071b82d002b
:104ba400090078000dc207000000e00002003a008e
:104bb400706c980006003700d1b82d000900780009
:104bc40006c207000000e00001003a0010749800db
:104bd4008870900010c0b3000104e0000a003a009d
:104be400f868900010c0b3000104e00006003a0029
:104bf400987090000104e00003003a000040eb00cc
:104c0400606c980020c0b3004f04be000000060092
:104c1400889fbe008a1f7800000578000104780090
:104c24008244780021b82d0008007800ebc1070009
:104c34000000e00002003a00097598000d003700fa
:104c440071b82d0008007800e4c107000000e000fe
:104c540002003a00796d980006003700d1b82d00a3
:104c640008007800ddc107000000e00001003a0000
:104c7400197598004f0578004f04be000000060027
:104c8400dc01fa00889fbe008a9fbe008c9fbe0094
:104c9400000578004faf99006b3320008a854500ea
:104ca400d1c0b3000b007800162a070080047800f6
:104cb4000900e000d10232008f0678003faf99006e
:104cc4000980e8000000a10080874700120020004e
:104cd40052af99000004eb000cc2b3000b00780043
:104ce400e02907008c4f500004003a00dea8910030
:104cf4008100e80051af990002003700ed4f5000e9
:104d04000200320080767c00020037000041eb0094
:104d140082767c000804e800888f5400efff3e0090
:104d24008984e8000900a1000f04780089874700fe
:104d34000804e8000800a1002daf99008d00780058
:104d440008007800b5c10700dea89100018040008a
:104d54000080e8000000a1000f067800808747006b
:104d64000c06e8000c00a10011b92d000800780021
:104d7400dac107000000e000090032000c047800ea
:104d840019b92d008005eb00001c7800890078001b
:104d94000b007800d1c107000000e000faff3a00e0
:104da4002ea99100821f780030b92d00801f780051
:104db40020c0b300792807001c047800a1b92d0095
:104dc4000800780085c10700e48757000000e00070
:104dd40057003a002c04900061ba2d0008007800b6
:104de4007ec107000000e00013003a000a007800ca
:104df400eff9070010c0b300206d9b000e0078008f
:104e04001002b0007f0109000058eb00f680460054
:104e1400100220000e004000e31d0700201b2000ac
:104e24000a004000f2072000110220008e8040009a
:104e340086c107003a003700d1ba2d000800780077
:104e440066c107000000e0000f003a008e00780001
:104e54001102b0007f0109008058eb00f780460082
:104e6400100220000e004000cf1d07002023200068
:104e74000a004000f2072000110220008e8040004a
:104e840072c107002600370051bb2d0008007800ce
:104e940052c107000000e0000e003a000e01780045
:104ea4001202b0007f0109000059eb00f6804600b1
:104eb400100220000e004000bb1d0700202b200024
:104ec4000a004000f2072000110220008e804000fa
:104ed4005ec107002a689300e14f500010003a00b9
:104ee400202b2000801f450021232000811f450026
:104ef400221b2000821f4500c0bb2d00801f7800ac
